:100000000C94A7140C94D1140C94D1140C94D11406
:100010000C94D1140C94D1140C94D1140C94D114CC
:100020000C94D1140C94D1140C94D1140C94D114BC
:100030000C94D1140C94D6220C94D1140C94D11499
:100040000C94D1140C942CC50C9492BE0C94D11425
:100050000C9407A20C94FDA10C94D1140C94D1140F
:100060000C94D1140C94D1140C94D1140C94D1147C
:100070000C94D1140C94D1140C94D1140C94D1146C
:100080000C9488750C94D1140C94D1144E414E49A3
:100090004E495459494E46CDCCCC3D0AD7233C1746
:1000A000B7D13877CC2B329595E6241FB14F0A0093
:1000B0000020410000C84200401C4620BCBE4CCA83
:1000C0001B0E5AAEC59D7400407A10F35A00A07200
:1000D0004E18090010A5D4E80000E8764817000083
:1000E000E40B54020000CA9A3B000000E1F5050051
:1000F0000080969800000040420F000000A086019A
:10010000000000102700000000E803000000006469
:1001100000000000000A00000000000100000000D4
:10012000002C76D888DC674F0823DFC1DFAE59E1A9
:10013000B1B796E5E3E453C63AE651997696E8E618
:10014000C28426EB898C9B62ED407C6FFCEFBC9CEB
:100150009F40F2BAA56FA5F490055A2AF75C936BFD
:100160006CF9676DC11BFCE0E40D47FEF520E6B5B8
:1001700000D0ED902E0300943577050080841E0892
:100180000000204E0A000000C80C333333330F98B0
:100190006E12831141EF8D2114893BE65516CFFE77
:1001A000E6DB18D1844B381BF77C1D901DA4BBE403
:1001B00024203284725E228100C9F124ECA1E53D45
:1001C0002741425300504C4100FFE0FFD140A0C8FE
:1001D000A6A22FF80023AC00AF10FFFEFF05FFD052
:1001E000FFE0FFC1FFD1E240A0C8A6A22FF8002384
:1001F0008127AC00AFFFD0FF64FFD1A5FFD0FF6423
:10020000FF64FFD1A4FFD0FF16FFFE4265640045E6
:100210006E636C6F73757265002568753A253032B0
:1002200068750025303268753A25303268750020CF
:100230002020202020200020202020003FFFF03818
:10024000007030FC3020FC102078102030102C0082
:10025000D02E31D02F7BD02F7BD02E31D02C00D080
:1002600020301020781020FC1030FC303800703F17
:10027000FFF03FFFF038007031863023871027876A
:10028000902F87D02F03D0203010207810207810A6
:100290002030102F03D02F87D0278790238710314D
:1002A00086303800703FFFF004104002082002083A
:1002B00020041040082080104100104100082080D8
:1002C0000410400000001FFFF81FFFF86E6F7469F4
:1002D0006669636174696F6E200063616E63656C4B
:1002E000005072696E742041626F727465640044DC
:1002F00069736D6973730055492041626F7274654B
:100300006400706175736500526573756D650055A5
:10031000492050617573650050617573696E672E71
:100320002E2E00726573756D65006E6F7469666957
:10033000636174696F6E200050726F6265205A208D
:100340004F66667365740046696C2E204469612EA1
:10035000004520696E206D6D5E33002008204661E7
:100360006374002008204D6178002008204D696EDC
:10037000004F6666004F6E004175746F74656D7056
:10038000005654726176204D696E00566D696E009C
:10039000566D6178204500566D6178205A00566D83
:1003A0006178205900566D6178205800416D617860
:1003B000204500416D6178205A00416D61782059D7
:1003C00000416D6178205800412D54726176656C52
:1003D00000412D5265747261637400416363656C02
:1003E0000056652D4A65726B00565A2D4A65726B30
:1003F0000056592D4A65726B0056582D4A65726B2E
:100400000050726F6265205A204F666673657400F3
:1004100050726F62652059204F6666736574005094
:10042000726F62652058204F6666736574004520C0
:1004300073746570732F6D6D005A205374657073FB
:100440002F6D6D00592053746570732F6D6D0058BA
:100450002053746570732F6D6D00416476616E6317
:1004600065642053657474696E6773003F0043616F
:100470006E63656C00496E6974004D343238004912
:100480006E697469616C697A6520454550524F4DBB
:100490000046696C616D656E740054656D706572BF
:1004A00061747572650053746570732F6D6D0050C3
:1004B000726F6265204F666673657473004A657279
:1004C0006B00416363656C65726174696F6E0056A1
:1004D000656C6F636974790053657420486F6D654E
:1004E000204F66667365747300436F6E6669677547
:1004F000726174696F6E0053746F77004465706C3D
:100500006F790053572D4D6F64650053656C662DF0
:100510005465737400526573657400426564004EDF
:100520006F7A7A6C650046616E2053706565640071
:10053000436F6E66696775726174696F6E005265AC
:1005400073746F72652044656661756C7473004CDA
:100550006F61642053657474696E67730053746FC0
:1005600072652053657474696E67730050726568B4
:10057000656174202420436F6E66004C4344204321
:100580006F6E747261737400424C546F75636800CF
:1005900050726F6265205A204F6666736574004121
:1005A0006476616E6365642053657474696E677305
:1005B000004D61696E004D3139305335350A47328F
:1005C000380A4732390A4D3430300A4D313034530D
:1005D0003231350A4732380A4D31303953323135EC
:1005E0000A4D34323053310A4731583130305931A5
:1005F000303046353030300A47315A300A4D3530C8
:10060000300A4D31313720536574205A204F6666C9
:10061000736574004D313036533132380A4D333002
:10062000334338533231354530550A4D3530300A71
:100630004D313137205049442054756E6520446F48
:100640006E65004D3139305335350A4D31303453F4
:100650003231350A4732380A4732394C310A47318C
:1006600020583130305931303046353030300A473B
:10067000315A30004D3530300A4D31313720536515
:100680007474696E67732053746F72656400537479
:100690006F72652053657474696E6773005072657C
:1006A0007020666F72205A2041646A75737400501E
:1006B00049442054756E65005365747570004D6132
:1006C000696E003F004261636B0053746F700043BA
:1006D0006F6E66696775726174696F6E0054656DDF
:1006E0007065726174757265004D6F74696F6E002C
:1006F000486F737420537461727400526573756D22
:1007000065205072696E740054756E650053746F85
:1007100070205072696E740050617573652050725C
:10072000696E74004C6576656C696E6720546F6FF6
:100730006C7300496E666F2053637265656E0021AD
:1007400000486F74656E6420746F6F20636F6C6413
:10075000004261636B0050726F63656564004D6FAA
:1007600074696F6E0044697361626C6520537465CF
:100770007070657273004D3834004F6666004F6EBE
:1007800000426564204C6576656C696E67004C6557
:1007900076656C20426564004732394E00417574BD
:1007A0006F20486F6D6500473238004D61696E00FB
:1007B00050726568656174202420456E6400507233
:1007C00065686561742024204265640054656D701D
:1007D0006572617475726500C501C101436F6F6C0C
:1007E000646F776E005072656865617420240046FE
:1007F000616E20537065656400426564004E6F7AD7
:100800007A6C65004D61696E0050726F6265205AA6
:10081000204F666673657400466C6F770046616EA4
:1008200020537065656400426564004E6F7A7A6C8F
:1008300065005370656564004D61696E00486F6DB9
:10084000696E67204661696C6564006F70656E0053
:10085000545249474745524544003A20007A5F6D5B
:10086000696E00795F6D696E00785F6D696E005228
:1008700065706F7274696E6720656E6473746F70F3
:10088000207374617475730A0020746F6F206C6F2D
:100890006E6720657874727573696F6E207072650B
:1008A00076656E7465640A0020636F6C64206578F9
:1008B00074727573696F6E2070726576656E74659B
:1008C000640A00486F6D65202573257325732046E3
:1008D00069727374005761726E696E673A20486F6F
:1008E0006D696E672042756D702044697669736F1B
:1008F00072203C20310A00020204000000000000C7
:100900000000000000000000164300001643000035
:10091000484300000041000000410000004000008A
:100920000001000000010000800055555500000046
:10093000400033333300AAAA2A0049922400000061
:100940002000C7711C0099991900D1451700555511
:1009500015003BB1130024491200111111000000D1
:1009600010000F0F0F00E3380E0043790D00CCCCC0
:100970000C00C3300C00E8A20B0064210B00AAAAF3
:100980000A00703D0A009DD80900427B09009224AC
:100990000900DCD308008888080010420800000025
:1009A0000800F0C107008787070075500700711C19
:1009B00007003EEB0600A1BC0600699006006666D3
:1009C0000600703E06006118060017F4050074D199
:1009D00005005BB00500B290050062720500555538
:1009E000050078390500B81E0500050505004EEC28
:1009F000040087D40400A1BD040090A7040049921C
:100A00000400C17D0400EE690400C756040044449C
:100A100004005C32040008210400411004000000BE
:100A200004003FF00300F8E0030026D20300C3C334
:100A30000300CCB503003AA803000A9B0300388EDC
:100A40000300C08103009F750300D0690300505E5E
:100A500003001D53030034480300913D030033336A
:100A6000030016290300381F030097150300300CFC
:100A70000300030303000BFA020049F10200BAE885
:100A800002005CE002002DD802002DD0020059C8FF
:100A90000200B0C0020031B90200DAB10200AAAA15
:100AA0000200A0A30200BC9C0200FA9502005C8F29
:100AB0000200DF88020082820200457C0200277665
:100AC000020027700200436A02007C640200D05ECC
:100AD00002003F590200C8530200FFFDFCFAF8F67D
:100AE000F4F2F0EEECEAE9E7E5E3E1E0DEDCDAD9A6
:100AF000D7D5D4D2D0CFCDCBCAC8C7C5C3C2C0BF4B
:100B0000BDBCBAB9B7B6B4B3B2B0AFADACAAA9A8C0
:100B1000A6A5A4A2A1A09E9D9C9A9998979594930E
:100B200092908F8E8D8B8A8988878684838281803C
:100B30007F7E7D7B7A797877767574737271706F4A
:100B40006E6D6C6B6A696867666564636261605F3D
:100B50005E5D5C5B5A595858575655545352515024
:100B6000504F4E4D4C4B4A4A4948474646454443F0
:100B7000424241403F3E3E3D3C3B3B3A39383837AC
:100B8000363535343332323130302F2E2E2D2C2B5A
:100B90002B2A2929282727262525242323222121FA
:100BA00020201F1E1E1D1C1C1B1B1A19191818178C
:100BB0001616151514131312121111100F0F0E0E15
:100BC0000D0D0C0C0B0A0A09090808070706060593
:100BD00005040403030202010000000016430000A4
:100BE0001643000048430000000000000000000021
:100BF000000053657474696E67732053746F726577
:100C00006400454550524F4D20496E697469616CCE
:100C1000697A65640A0000803B4400803B44000020
:100C20002041000096420000A0420000A0420000C7
:100C3000C8430000BE42D0070000D0070000640097
:100C400000004B000000434F4D4D554E4943415469
:100C5000494F4E0044525952554E004552524F5240
:100C60005300494E464F004543484F00486F746556
:100C70006E642049646C652054696D656F757400FD
:100C8000486F74656E642049646C652054696D65B5
:100C90006F75740A002121204B494C4C206361750B
:100CA00073656420627920746F6F206D75636820AE
:100CB000696E6163746976652074696D65202D20A5
:100CC00063757272656E7420636F6D6D616E643AE8
:100CD000200053544F505045442E20005072696EEE
:100CE0007465722073746F7070656420647565201C
:100CF000746F206572726F72732E2046697820744B
:100D00006865206572726F7220616E64207573650C
:100D1000204D39393920746F207265737461727493
:100D20002E202854656D7065726174757265206936
:100D3000732072657365742E205365742069742066
:100D400061667465722072657374617274696E672E
:100D5000290A004E6F20436865636B73756D2077B9
:100D6000697468206C696E65206E756D6265722CA1
:100D7000204C617374204C696E653A20006368658D
:100D8000636B73756D206D69736D617463682C207E
:100D90004C617374204C696E653A20004C696E6535
:100DA000204E756D626572206973206E6F74204CE1
:100DB000617374204C696E65204E756D6265722B8F
:100DC000312C204C617374204C696E653A20004DC3
:100DD0003131300053657269616C207374617475D0
:100DE00073206D69736D617463680A00776169745B
:100DF0000A00506C6561736520526573657400501C
:100E000052494E5445522048414C544544002553C4
:100E10003A20255300706F7765726F6666004B4904
:100E20004C4C45442E20005072696E7465722068E7
:100E3000616C7465642E206B696C6C282920636179
:100E40006C6C6564210A0053544F505045442E2069
:100E5000005072696E7465722073746F707065648F
:100E60002064756520746F206572726F72732E2016
:100E700046697820746865206572726F7220616EB1
:100E80006420757365204D39393920746F2072657F
:100E900073746172742E202854656D70657261746C
:100EA0007572652069732072657365742E205365B1
:100EB0007420697420616674657220726573746150
:100EC0007274696E67290A006563686F3A0045723B
:100ED000726F723A0042696C696E656172204C658E
:100EE00076656C696E6720477269643A0A00212151
:100EF0002053544F502063616C6C656420626563BD
:100F000061757365206F6620424C546F756368206D
:100F10006572726F72202D20726573746172742015
:100F200077697468204D3939390A002121205354DA
:100F30004F502063616C6C656420626563617573FA
:100F400065206F6620424C546F756368206572722D
:100F50006F72202D207265737461727420776974CA
:100F600068204D3939390A002F2F616374696F6E1B
:100F70003A0073746172740050726F62696E672018
:100F8000506F696E740025532025692F2569002E46
:100F90000A002F0050726F62696E67206D6573687A
:100FA00020706F696E742000202844525952554EAB
:100FB0002900473239204175746F20426564204C06
:100FC0006576656C696E67003F20284C2C522C4674
:100FD0002C4229206F7574206F6620626F756E64D5
:100FE000732E0A003F2856296572626F7365206C64
:100FF0006576656C20696D706C61757369626C658E
:101000002028302D34292E0A00426164205A20768F
:10101000616C75650A004E6F2062696C696E65616E
:101020007220677269640A0020496E76616C696497
:101030002065787472756465722000536C65657004
:101040002E2E2E005A2050726F62652050617374EC
:10105000204265640A005A2050726F626520506118
:10106000737420426564004732384C3000205A3A8D
:10107000200020593A200042656420583A20004D53
:1010800065736820706F696E74206F7574206F6669
:101090002072616E67650A004D302053746F7000D6
:1010A0004D312053746F7000436F6E74696E7565B7
:1010B00000436C69636B20746F20526573756D65B6
:1010C0002E2E2E004E6F204D6F76652E00256973F3
:1010D0000025696D20256973002569682025696DE3
:1010E0002025697300256964202569682025696DBC
:1010F00020256973002569792025696420256968A0
:101100002025696D20256973005072696E74207402
:10111000696D653A20006F6B006F666600670C6250
:101120000C5B0C540C460C44454255473A00544D58
:10113000334420456E64657232204F46462E0020AF
:101140004500204D39322058004649524D574152F2
:10115000455F4E414D453A4D61726C696E20322EAD
:10116000302E375F4457372E3320544D33442045BB
:1011700032534D4442422028417072203234203292
:101180003032312032313A31363A32362920534F1B
:10119000555243455F434F44455F55524C3A68743E
:1011A0007470733A2F2F6769746875622E636F6D60
:1011B0002F496E73616E6974794175746F6D6174D6
:1011C000696F6E2F4D61726C696E2F747265652F39
:1011D000437265616C6974794477696E5F322E3051
:1011E0002050524F544F434F4C5F56455253494F36
:1011F0004E3A312E30204D414348494E455F5459B7
:1012000050453A544D334420456E64657232204552
:10121000585452554445525F434F554E543A31202D
:10122000555549443A63656465326132662D3431FF
:1012300061322D343734382D396231322D633535F2
:101240006336326633363766660A002F2F004D311B
:10125000343520533C696E6465783E206F75742088
:101260006F662072616E67652028302D31290A0073
:10127000205400205200416363656C65726174699B
:101280006F6E3A2050005741524E494E4721204C34
:101290006F77205A204A65726B206D6179206C65EA
:1012A000616420746F20756E77616E746564207060
:1012B00061757365732E0A004D3230362058002058
:1012C000580020204D61783A2000200020204D69F0
:1012D0006E3A2000536F667420656E6473746F708D
:1012E000733A200046523A0020466C6F773A20004D
:1012F0003A200020536572766F2000206F757420AD
:101300006F662072616E67650A00536572766F20A2
:101310000050726F6265204F6666736574205A00D4
:1013200050726F6265204F6666736574205A0020A4
:10133000643A0020693A0020703A00496E76616C88
:1013400069642065787472756465720A0020643A75
:101350000020693A0020703A004C434420436F6EED
:1013600074726173743A200064697300656E00439F
:10137000290A0061626C656420286D696E207465BD
:101380006D702000436F6C642065787472756465BD
:10139000732061726520004F4646004F4E00426543
:1013A00064204C6576656C696E6720004661696CE7
:1013B000656420746F20656E61626C6520426564AF
:1013C000204C6576656C696E670A00496E76616CC3
:1013D0006964206D6573682E0A004D3432312069CE
:1013E0006E636F727265637420706172616D657493
:1013F00065722075736167650A004D6573682070BA
:101400006F696E74206F7574206F662072616E67ED
:10141000650A004F666673657473204170706C696D
:101420006564004572723A20546F6F2066617221C4
:1014300000546F6F206661722066726F6D20726556
:10144000666572656E636520706F696E740A00452B
:101450004550524F4D204F4B0A00290A0020746F0F
:1014600020003F5A206F7574206F662072616E678E
:1014700065202800290A0020746F20003F59206F42
:101480007574206F662072616E676520282D0029B3
:101490000A0020746F20003F58206F7574206F661B
:1014A0002072616E676520282D00205A00205900A7
:1014B00050726F6265204F666673657420580049EC
:1014C0006E76616C69642065787472756465720A01
:1014D000002042002050006F6B0020573A00436FFD
:1014E0006F6C696E672E2E2E0048656174696E6799
:1014F0002E2E2E00452025530020573A00426564C9
:1015000020436F6F6C696E672E2E2E00426564203B
:1015100048656174696E672E2E2E002364656669C6
:101520006E652044454641554C545F006265640039
:101530004B6420004B6920004B7020005049442030
:101540004175746F74756E652066696E6973686540
:1015500064212050757420746865206C6173742058
:101560004B702C204B6920616E64204B6420636FAC
:101570006E7374616E74732066726F6D2062656C39
:101580006F7720696E746F20436F6E66696775723E
:101590006174696F6E2E680A005049442041757469
:1015A0006F74756E65206661696C6564212074696D
:1015B0006D656F75740A00504944204175746F74ED
:1015C000756E65206661696C6564212054656D7077
:1015D0006572617475726520746F6F2068696768E1
:1015E0000A00204B643A2000204B693A2000204B2F
:1015F000703A200020436C61737369632050494442
:10160000200A00204E6F206F76657273686F6F74CA
:101610000A002054753A2000204B753A2000206DB6
:1016200061783A2000206D696E3A200020643A20EB
:101630000020626961733A2000504944204175746A
:101640006F74756E652073746172740A005049443A
:10165000204175746F74756E65206661696C656490
:10166000212054656D706572617475726520746FA8
:101670006F20686967680A00504944204175746F9B
:1016800074756E6500504944204175746F74756EB1
:1016900065206661696C656421204261642068652B
:1016A000617465722069640A004572723A2075742B
:1016B000663820666F6E74206E6F7420696E697470
:1016C00069616C697A65642E004572723A2075749E
:1016D000663820666F6E74206E6F7420696E697450
:1016E00069616C697A65642E004572723A2075747E
:1016F000663820666F6E74206E6F7420696E697430
:1017000069616C697A65642E00000C0F00FE0702A7
:101710002503BB017FFE08FE08FE05080806000041
:1017200040F0C88888987810050808060000C0F8BE
:101730008888888888F80505050600012030F8307B
:10174000200508080600002070F820202020E00571
:1017500009090600FF2070A8A8B88888702007052E
:1017600005070001D86C366CD80509090600FFF89A
:10177000A88888888888A8F8050A0A0600FE2050EC
:1017800050505088A8A8887003030306000340A0A7
:1017900040FFFFFFFFFFFFFFFFFFFFFFFFFFFFFF18
:1017A000FFFFFFFFFFFFFF0000000605FF01070727
:1017B000060200808080808000800303030601050C
:1017C000A0A0A005060606000050F85050F85005ED
:1017D00009090600FF2070A8A07028A8702005073E
:1017E00007060000C8C810204098980507070600A3
:1017F0000040A0A040A89068010303060205808075
:10180000800309090601FF2040408080804040207D
:101810000309090601FF8040402020204040800548
:10182000070706000020A8702070A82005050506FF
:1018300000012020F820200203030601FFC04080A1
:10184000050101060003F8020202060100C0C005FE
:101850000707060000081010204040800507070613
:101860000000708898A8C888700307070601004028
:10187000C040404040E0050707060000708808109F
:101880002040F8050707060000F8081030088870A7
:1018900005070706000010305090F81010050707E4
:1018A000060000F880F008088870050707060000A9
:1018B000304080F0888870050707060000F808109F
:1018C000102020200507070600007088887088888F
:1018D0007005070706000070888878081060020508
:1018E00005060100C0C000C0C00206060601FFC018
:1018F000C000C04080030505060101204080402053
:10190000050303060002F800F8030505060101803F
:101910004020408005070706000070881020200046
:10192000200507070600007088B8A8B88070050772
:1019300007060000708888F8888888050707060071
:1019400000F04848704848F0050707060000708816
:101950008080808870050707060000F048484848E6
:1019600048F0050707060000F88080F08080F80541
:101970000707060000F88080F080808005070706D2
:10198000000070888080988870050707060000882E
:101990008888F8888888030707060100E0404040EF
:1019A0004040E00507070600003810101010906056
:1019B0000507070600008890A0C0A09088050707CB
:1019C000060000808080808080F805070706000000
:1019D00088D8A8888888880507070600008888C8EE
:1019E000A898888805070706000070888888888876
:1019F00070050707060000F08888F08080800507E2
:101A00000706000070888888A89068050707060008
:101A100000F08888F0A0908805070706000070880D
:101A20008070088870050707060000F82020202035
:101A300020200507070600008888888888887005A8
:101A40000707060000888888885050200507070689
:101A5000000088888888A8A8500507070600008825
:101A60008850205088880507070600008888502085
:101A7000202020050707060000F80810204080F805
:101A80000309090601FFE080808080808080E005F6
:101A900007070600008040402010100803090906CF
:101AA00001FFE020202020202020E0050303060085
:101AB000052050880501010600FEF8030303060116
:101AC0000580402005050506000070087888780527
:101AD00007070600008080F0888888F00505050665
:101AE00000007080808870050707060000080878ED
:101AF000888888780505050600007088F0807005E4
:101B00000707060000304840E04040400507070650
:101B100000FE708888887808700507070600008036
:101B200080F0888888880307070601004000C040CD
:101B30004040E00409090601FE10003010101010AA
:101B4000906005070706000080808890E090880379
:101B50000707060100C04040404040E0050505067B
:101B60000000D0A8A8A8A8050505060000B0C888F0
:101B700088880505050600007088888870050707B5
:101B80000600FEF0888888F080800507070600FEC2
:101B900078888888780808050505060000B0C880A0
:101BA000808005050506000078807008F0050707AD
:101BB0000600002020F8202020180505050600005A
:101BC0008888889868050505060000888888502060
:101BD0000505050600008888A8A85005050506002B
:101BE0000088502050880507070600FE8888885026
:101BF000204080050505060000F8102040F8030984
:101C0000090601FF20404040804040402001090972
:101C10000602FF8080808080808080800309090622
:101C200001FF804040402040404080050303060003
:101C30000248A890FF24F4D43050C38E20C2A240A2
:101C400017828B7011127A910D816CD90AA861E10B
:101C500008C7586607615143061E4B5D05C145A77D
:101C6000041A411104093D9803713931034036DBF0
:101C70000265339102D4305402802E1D02632CEE93
:101C800001752AC501B028A001102781018F2564A4
:101C9000012B244B01E0223401AC211F018D200DCA
:101CA00001801FFC00841EED00971DDF00B81CD2D0
:101CB00000E61BC600201BBC00641AB200B219A8C3
:101CC000000A19A0006A189900D117910040178BDB
:101CD00000B516840031167E00B31579003A1573ED
:101CE00000C7146F0058146A00EE1366008813636F
:101CF0000025135E00C7125B006C125700151254CA
:101D000000C111510070114F0021114B00D6104934
:101D1000008D1047004610440002104200C00F40E2
:101D200000800F3E00420F3C00060F3B00CB0E38F8
:101D300000930E37005C0E3500270E3400F30D3291
:101D400000C10D3100900D3000600D2E00320D2DC0
:101D500000050D2C00D90C2B00AE0C2900850C2998
:101D6000005C0C2700350C27000E0C2600E80B2425
:101D700000C40B2400A00B23007D0B23005A0B2171
:101D800000390B2100180B2000F80A1F00D90A1E89
:101D900000BB0A1E009D0A1D00800A1D00630A1C6C
:101DA00000470A1B002C0A1B00110A1A00F7091A27
:101DB00000DD091900C4091900AB091900920917BF
:101DC000007B091800630917004C09160036091634
:101DD00000200916000A091500F5081500E008148E
:101DE00000CC081400B8081400A4081400900813CC
:101DF000007D0812006B08130058081200460812F4
:101E00000034081100230811001208110001081104
:101E100000F0071000E0071000D0071000C0071006
:101E200000B0070F00A107100091070E0083070FF5
:101E30000074070F0065070E0057070E0049070ED4
:101E4000003B070D002E070E0020070D0013070DA5
:101E50000006070D00F9060C00ED060D00E0060C6B
:101E600000D4060C00C8060C00BC060C00B0060C22
:101E700000A4060B0099060C008D060B0082060BD1
:101E80000077060B006C060B0061060A0057060B74
:101E9000004C060A0042060A0038060A002E060A0E
:101EA0000024060A001A060A001006090007060A9E
:101EB00000FD050900F4050900EB050900E205092C
:101EC00000D9050900D0050900C7050900BE0509AC
:101ED00000B5050800AD050800A50509009C05082A
:101EE00000940508008C050800840508007C05089E
:101EF00000740508006C050700650508005D05070E
:101F000000560508004E0507004705070040050874
:101F10000038050700310507002A050700230507DB
:101F2000001C050600160507000F0507000805063A
:101F30000002050700FB040600F5040700EE040696
:101F400000E8040600E2040700DB040600D50406EE
:101F500000CF040600C9040600C3040600BD040641
:101F600000B7040600B1040500AC040600A6040690
:101F700000A00405009B04060095040500900406DB
:101F8000008A04050085040500800406007A040523
:101F90000075040500700405006B04050066040567
:101FA00000610405005C04050057040500520405A7
:101FB000004D04050048040500430405003E0404E8
:101FC000003A04050035040500300404002C040523
:101FD0000027040400230405001E0404001A04045E
:101FE0000016040500110404000D04040009040592
:101FF000000404040000040400FC030400F80304CB
:1020000000F4030400F0030400EC030400E80304FC
:1020100000E4030400E0030400DC030400D803042C
:1020200000D4030400D0030400CC030400C803035D
:1020300000C503030024F404D9201BC40C5C0E98D3
:1020400004C4095F0265077101F405F900FB04B3DC
:102050000048048700C10369005803550003034585
:1020600000BE023A008402310053022A00290225F0
:102070000004022000E4011C00C8011900AF011790
:102080000098011400840113007101100061011017
:102090000051010E0043010D0036010B002B010B16
:1020A0000020010B00150109000C010900030108C3
:1020B00000FB000800F3000800EB000700E4000646
:1020C00000DE000600D8000600D2000600CC0005A5
:1020D00000C7000500C2000500BD000400B90004EF
:1020E00000B5000400B1000400AD000400A9000424
:1020F00000A5000300A20003009F0004009B000352
:102100000098000300950002009300030090000374
:10211000008D0002008B0003008800020086000290
:102120000084000300810002007F0002007D0002A5
:10213000007B0002007900020077000100760002B7
:10214000007400020072000100710002006F0002C2
:10215000006D0001006C0002006A000100690002CD
:1021600000670001006600010065000100640002D4
:10217000006200010061000100600001005F0002D8
:10218000005D0001005C0001005B0001005A0001DD
:1021900000590001005800010057000100560001DD
:1021A00000550001005400010053000000530001DD
:1021B000005200010051000100500001004F0001D9
:1021C000004E0000004E0001004D0001004C0001D7
:1021D000004B0000004B0001004A000100490001D3
:1021E00000480000004800010047000100460000D0
:1021F00000460001004500000045000100440001C8
:1022000000430000004300010042000000420001C2
:10221000004100000041000100400001003F0000BB
:10222000003F0001003E0000003E0001003D0000B4
:10223000003D0001003C0000003C0000003C0001AB
:10224000003B0000003B0001003A0000003A0001A2
:10225000003900000039000100380000003800009B
:102260000038000100370000003700010036000090
:102270000036000000360001003500000035000087
:10228000003500010034000000340000003400017B
:102290000033000000330000003300010032000072
:1022A0000032000000320001003100000031000067
:1022B000003100010030000000300000003000015B
:1022C000002F0000002F0000002F0000002F000151
:1022D000002E0000002E0000002E0001002D000046
:1022E000002D0000002D0000002D0001002C00003A
:1022F000002C0000002C0000002C0001002B00002E
:10230000002B0000002B0000002B0001002A000021
:10231000002A0000002A0000002A00010029000015
:102320000029000000290000002900000029000108
:1023300000280000002800000028000000280000FD
:1023400000280001002700000027000000270000EF
:1023500000270000002700010026000000260000E2
:1023600000260000002600000026000100250000D5
:1023700000250000002500000025000000250000C9
:1023800000250001002400000024000000240000BB
:1023900000240000002400010023000000230000AE
:1023A00000230000002300000023000000230000A1
:1023B0000023000100220000002200000022000093
:1023C0000022000000220000002200010021000085
:1023D0000021000000210000002100000021000079
:1023E000002100000021000100200000002000006A
:1023F000002000000020000000200000002000005D
:102400000020000000200001001F0000001F00004D
:10241000001F0000001F0000001F0000001F000040
:10242000001F0001001E0000001E0000001E000032
:10243000001E00000039300000332500008719001D
:1024400000B00F0000DB080000BD040000740200B3
:10245000003F01000020436F756E7420583A00421F
:10246000656400453100626564002C2073797374E3
:10247000656D2073746F70706564212048656174A8
:1024800065725F49443A200048656174696E67204F
:102490004661696C65640048656174696E672066B1
:1024A00061696C6564004D31313220536875746424
:1024B0006F776E001000C90210012C01400122014B
:1024C00070011801B0010E01F00104015002FA0080
:1024D000B002F0003003E600D003DC009004D2002C
:1024E0007005C800A006BE000008B400B009AA002C
:1024F000D00BA000600E960060118C0000158200C9
:1025000020197800C01D6E00A0226400B0275A0078
:10251000902C500000314600E0343C00103832006E
:10252000903A2800603C1E00A03D1400803E0A0046
:10253000203F0000544845524D414C2052554E41D9
:1025400057415900546865726D616C2052756E6117
:10255000776179004572723A204D415854454D508B
:10256000004D415854454D5020747269676765723B
:102570006564004572723A204D494E54454D5000F5
:102580004D494E54454D50207472696767657265B8
:102590006400202F002042403A0020403A006001B1
:1025A000F4017001EA019001E001B001D601D0010F
:1025B000CC010002C2013002B8016002AE019002FB
:1025C000A401D0029A012003900170038601C00388
:1025D0007C0130047201A004680120055E01B00591
:1025E000540160064A0120074001F0073601F00857
:1025F0002C01100A2201500B1801C00C0E01500EC4
:1026000004013010FA002012F0005014E600C01649
:10261000DC007019D200501CC800501FBE00702290
:10262000B400B025AA00F028A000202C9600302F7E
:102630008C0010328200A0347800F0366E00E03852
:102640006400803A5A00403B5500E03B5000F03CAB
:102650004600C03D3C00603E3200E03E2800303F76
:102660001E00503F1900703F1400A03F0A00C03FF9
:102670000000D03FF6FFE03FECFF2020506C616E81
:102680006E657242756666657242797465733A204A
:10269000002046726565204D656D6F72793A2000A5
:1026A000436F6D70696C65643A20417072203234FA
:1026B00020323032310A00204C617374205570642E
:1026C000617465643A20323032312D30342D313826
:1026D000207C20417574686F723A2054696E794D80
:1026E000616368696E657333440A00322E302E3799
:1026F0005F4457372E330A004D61726C696E0020BB
:10270000536F6674776172652052657365740A0051
:10271000205761746368646F672052657365740A3B
:10272000002042726F776E206F757420526573655A
:10273000740A002045787465726E616C205265736E
:1027400065740A00506F77657255700A0073746182
:1027500072740A00456E6473746F707300255320A1
:10276000256320256320256320256300205A3A0035
:1027700020593A0020583A00656E6473746F707384
:10278000206869743A2000000000010200090A0074
:102790000000000403080700000000000000000023
:1027A00000000000000000004D6F76652025736D6D
:1027B0006D004D6F766520302E316D6D004D6F765A
:1027C0006520316D6D004D6F76652031306D6D0087
:1027D0004D6F766520417869730045787472756431
:1027E0006572004D6F7665205A004D6F76652059F1
:1027F000004D6F7665205800FFFFFF50726F6269D1
:102800006E67204661696C65640A0050726F626988
:102810006E67204661696C656400205A3A2000208A
:10282000593A200042656420583A200073686F7757
:1028300000627574746F6E0070726F6D70745F00FB
:10284000656E6400626567696E00220A00556E6BF2
:102850006E6F776E20636F6D6D616E643A2022003B
:10286000544D334420456E64657232205265616474
:10287000792E005072696E74696E672E2E2E00508C
:1028800072696E74205061757365640020453A006A
:10289000205A3A0020593A00583A004572726F7235
:1028A0002077726974696E6720746F2045455052B5
:1028B0004F4D210A0020746F6F206C6F6E6720658A
:1028C0007874727573696F6E2070726576656E7458
:1028D00065640A0020636F6C642065787472757398
:1028E000696F6E2070726576656E7465640A005259
:1028F0006573656E643A2000000022002500280000
:102900002B0000002100240027002A0002020202FE
:102910000202020204040404040404040303030383
:102920000303030301010101010101010102040884
:102930001020408001020408102040800102040899
:10294000102040808040201008040201EFD811249C
:102950001FBECFEFD0E4DEBFCDBF12E0A0E0B1E0FC
:10296000E8E8F6ED01E00BBF02C007900D92AE3132
:10297000B107D9F724E1AEE1B2E001C01D92A03A5F
:10298000B207E1F714E1C7EAD4E104C02197FE01E0
:102990000E94F1E8C63AD107C9F70E948ED90C947B
:1029A00042EB0C9400009F92AF92BF92CF92DF92C5
:1029B000EF92FF920F931F93CF93DF9300D000D03D
:1029C0001F92CDB7DEB7EAEDFAE00027BB27462F0E
:1029D000572FA82FAA2341F4A52F542FB85FAA235D
:1029E00019F4A52F5527B85FA03138F45295A29558
:1029F000452F4F70507FA42BBC5FA03428F4550F97
:102A0000AA1F550FAA1FBE5FA03818F4550FAA1FA2
:102A1000B395550FAA1FEA0FF01F449151E0AA2762
:102A2000B85081F1C8F0B0FF02C0440F551FB1FF8C
:102A300004C0440F551F440F551FB2FF06C05295E6
:102A40004295142F1F70407F512BB3FF1BC0A52F41
:102A5000542F44270C944215B195B0FF02C05595F0
:102A60004795B1FF04C05595479555954795B2FFD9
:102A700005C05295407F4295452B5F70B3FF02C061
:102A8000452F5527DD24CC24BB24B2E0649FD01809
:102A9000C108B00AB00B749FC018B108B00B849F76
:102AA000B018B109659FC018B108B00B759FB01878
:102AB000B109859FB0196A9FB018B1097A9FB01902
:102AC0004D9DA12C99243327992722275D9DA00C89
:102AD000911C301F901F201FAD9D900C311D901F29
:102AE000201F4C9DA00C911C301F901F201F5C9D2F
:102AF000900C311D901F201FAC9D300D911D201F8B
:102B00004B9D900C311D901F201F5B9D300D911D22
:102B1000201FAB9D900D211D4B9F300D911D201F3F
:102B20005B9F900D211DAB9F200DB1E0BB24CC24F9
:102B3000DD24639FD018C108B00AB00B739FC01882
:102B4000B108B00B839FB018B109699FC018B108D4
:102B5000B00B799FB018B109899FB019629FB01866
:102B6000B109729FB019D61AC70AB80A20F0B1E0AD
:102B70003B0F901F201F1124792F632F90E0822F8D
:102B80000F900F900F900F900F90DF91CF911F91AA
:102B90000F91FF90EF90DF90CF90BF90AF909F90FC
:102BA0000895CF92DF92EF92FF9280917602882370
:102BB00009F457C0C0907202D0907302E090740282
:102BC000F090750220E030E0A901C701B6010E9433
:102BD00004E2882309F445C020E030E040E05FE3F0
:102BE000C701B6010E946AE29B01AC010E946AE241
:102BF0002BED3FE049E450E40E946AE29B01AC0106
:102C000060E070E080E89FE30E947EE96B017C0158
:102C1000C0926D02D0926E02E0926F02F09270024A
:102C20006091240170912501072E000C880B990BEF
:102C30000E940BE22AE037ED43E25CE30E946AE285
:102C4000A70196010E946AE260937001709371017E
:102C50008093720190937301FF90EF90DF90CF907B
:102C60000895C12CD12C80E8E82E8FE3F82ED0CF28
:102C7000CF92DF92EF92FF92FC01C080D180E28080
:102C8000F38020E030E0A901C701B6010E9404E210
:102C900087FF68C0C701B601905820E030E040E2ED
:102CA00051E40E946AE220E030E040EA50E40E94F1
:102CB000FBE820E030E040E251E40E947EE90E941F
:102CC000F0E99B0160E22031F7E23F0730F0C901F3
:102CD00060E177E20E94C9E8605D6093A00B283E46
:102CE00083E0380708F445C0C90168EE73E00E942C
:102CF000C9E8CB016AE070E00E94C9E8805D80937A
:102D0000A10B80E22436310558F0C90164E670E079
:102D10000E94C9E8CB016AE070E00E94C9E8805DCA
:102D20008093A20B80E22A30310558F0EAE0F0E00F
:102D3000C901BF010E94C9E8CB01BF010E94C9E8D7
:102D4000805D8093A30BC9016AE070E00E94C9E82E
:102D5000805D8093A40B80EA9BE0FF90EF90DF9072
:102D6000CF90089520E030E040E251E4C701B60181
:102D700098CF80E2C4CF8F929F92AF92BF92CF92B2
:102D8000DF92EF92FF92FC01C080D180E280F3805D
:102D900020E030E040E251E4C701B6010E946AE25F
:102DA00020E030E040E251E40E946AE24B015C0125
:102DB00020E030E0A901C701B6010E9404E220E052
:102DC00030E040EA50E487FF04C020E030E040EA11
:102DD00050ECC501B4010E94FBE820E030E040E285
:102DE00051E40E947EE90E94F0E99B018BE237FFEB
:102DF00005C022273327261B370B8DE280939F0BBC
:102E0000C90168EE73E00E94DDE8CB01EAE0F0E082
:102E1000BF010E94DDE8805D8093A00BC90164E6DC
:102E200070E00E94DDE8CB01BF010E94DDE8805D1B
:102E30008093A10BC901BF010E94DDE8282FCB01BF
:102E4000BF010E94DDE8805D8093A20B8EE280933B
:102E5000A30B205D2093A40B8FE99BE0FF90EF90E4
:102E6000DF90CF90BF90AF909F908F9008958F92FA
:102E70009F92AF92BF92CF92DF92EF92FF92CF9349
:102E8000FC01C080D180E280F38020E030E040E2AD
:102E900051E4C701B6010E946AE220E030E048EC4C
:102EA00052E40E946AE24B015C0120E030E040E223
:102EB00051ECC701B6010E9404E2181654F420E058
:102EC00030E048EC52E4C701B6010E947EEA87FD7B
:102ED00086C020E030E0A901C701B6010E9404E2EB
:102EE00087FF6EC060E070E080EA90ECA50194017D
:102EF0000E94FBE820E030E040E251E40E947EE9DD
:102F00000E94F0E96B017C01F7FC5FC020E137E231
:102F100040E050E00E946EE8CA01B9012AE030E0CA
:102F200040E050E00E946EE8605D60939F0BC70137
:102F3000B60128EE33E040E050E00E946EE89AE0EF
:102F4000892E912CA12CB12CCA01B901A5019401A3
:102F50000E946EE8605D6093A00BC701B60124E695
:102F600030E040E050E00E946EE8CA01B901A501DE
:102F700094010E946EE8605D6093A10B8EE28093E5
:102F8000A20BC701B601A50194010E946EE8C62FED
:102F9000CA01B901A50194010E946EE8605D6093C9
:102FA000A30BC05DC093A40B8FE99BE0CF91FF9072
:102FB000EF90DF90CF90BF90AF909F908F9008954B
:102FC00060E070E080EA90E491CFF094E094D094D7
:102FD000C094C11CD11CE11CF11C6DE2A6CF20E005
:102FE00030E0A901C701B6010E9404E287FF6AC070
:102FF00060E070E080EA90ECA50194010E94FBE89B
:1030000020E030E040E251E40E947EE90E94F0E9D5
:103010004B015C0120E030E0A901C701B6010E942C
:103020007EEA87FD0BC020E030E040E251E4C701BA
:10303000B6010E9404E260E287FD13C0B7FC47C0FE
:10304000C501B40128EE33E040E050E00E946EE894
:10305000CA01B9012AE030E040E050E00E946EE889
:10306000605D6093A00BC501B40124E630E040E050
:1030700050E00E946EE88AE0C82ED12CE12CF12CA1
:10308000CA01B901A70196010E946EE8605D6093D4
:10309000A10B8EE28093A20BC501B401A70196019A
:1030A0000E946EE8C62FCA01B901A70196010E94CD
:1030B0006EE8605D6093A30BC05DC093A40B80EAD3
:1030C0009BE074CF60E070E080EA90E495CFB0942C
:1030D000A09490948094811C911CA11CB11C6DE261
:1030E000C0CF9C0197FF26C0EE27FF27E81BF90BF6
:1030F0002D398FEF38070CF05DC08DE28093A10B66
:10310000CF0164E670E00E94DDE8CB012AE030E008
:10311000B9010E94DDE8805D8093A20BCF01B90167
:103120000E94DDE8CB01B9010E94DDE8805D80935B
:10313000A30B2AC0283E83E03807B4F1C90168EE2A
:1031400073E00E94DDE8CB01EAE0F0E0BF010E94FD
:10315000DDE8805D8093A10BC90164E670E00E9408
:10316000DDE8CB01BF010E94DDE8805D8093A20B0A
:10317000C901BF010E94DDE8CB01BF010E94DDE86B
:10318000805D8093A30BF901CF016AE070E00E949B
:10319000DDE8805D8093A40B81EA9BE008958DE2D9
:1031A00037FDC5CF80E2C3CFF90180E22436310577
:1031B0000CF0A4CF80E28093A10B8093A20BEA30A5
:1031C000F1056CF38DE237FF80E28093A20BCF0113
:1031D0006AE070E00E94DDE8605D6093A30BD4CFED
:1031E0009C0197FD2DC080E2243631055CF0C901B9
:1031F00064E670E00E94DDE8CB016AE070E00E94C6
:10320000DDE8805D8093A20B80E22A3031055CF01E
:10321000EAE0F0E0C901BF010E94DDE8CB01BF0197
:103220000E94DDE8805D8093A30BC9016AE070E035
:103230000E94DDE8805D8093A40B82EA9BE0089504
:103240003195219531098DE2DDCF24E6829FC001C1
:10325000112481589F4F6FEF70E00E94DDE8262F08
:1032600081E3643609F080E28093A10B90E22A307A
:1032700040F03AE0822F632F0E94AFE80E94AFE84F
:10328000905D9093A20B822F6AE00E94AFE8905D60
:103290009093A30B85E28093A40B81EA9BE00895B1
:1032A0006091240170912501072E000C880B990B69
:1032B0000E940BE22AE037ED43E25CE30E946AE2FF
:1032C00020916D0230916E0240916F025091700218
:1032D0000E946AE2609370017093710180937201A1
:1032E0009093730108958091AC0B811104C080917B
:1032F0008E0B8093020C0895CF93DF93EC01CB01EA
:10330000BA010E940BE229EC38EC48EC5EE30E9423
:103310007EE920E030E040E05FE30E94FBE80E94AD
:10332000F7E96883DF91CF9108950E940BE229ECC1
:1033300038EC48EC5EE30E947EE920E030E040E0BB
:103340005FE30E94FBE80E94F7E9862F0C942519A1
:1033500080914001909141010C94216BE091AC0B64
:1033600086E0E802F0011124E458F44F80918E0BBE
:1033700090E0958384830895CF93DF9300D000D0AD
:10338000CDB7DEB70E94F7E90E9409E269837A832C
:103390008B839C83CE0101960E9438160F900F906C
:1033A0000F900F90DF91CF9108958F929F92AF92DF
:1033B000BF92CF92DF92EF92FF92CF936B017C018D
:1033C00020E030E0A9010E9404E287FD9FC06DEB80
:1033D00077E386E095E3A70196010E94FBE86B0185
:1033E0007C0120E030E040E251E40E946AE220E00B
:1033F00030E048EC52E40E946AE24B015C0120E0BC
:1034000030E0A901C701B6010E9404E220E030E0EB
:1034100040EA50E487FF04C020E030E040EA50EC8E
:10342000C501B4010E94FBE820E030E040E251E435
:103430000E947EE90E94F0E96B017C018BE2F7FEBD
:1034400009C0F094E094D094C094C11CD11CE11C3C
:10345000F11C8DE280939E0BC701B60120E137E29B
:1034600040E050E00E946EE88AE0882E912CA12C6A
:10347000B12CCA01B901A50194010E946EE8605DFA
:1034800060939F0BC701B60128EE33E040E050E0A7
:103490000E946EE8CA01B901A50194010E946EE87C
:1034A000605D6093A00BC701B60124E630E040E008
:1034B00050E00E946EE8CA01B901A50194010E9482
:1034C0006EE8605D6093A10B8EE28093A20BC70152
:1034D000B601A50194010E946EE8C62FCA01B90188
:1034E000A50194010E946EE8605D6093A30BC05D2E
:1034F000C093A40B8EE99BE0CF91FF90EF90DF90FB
:10350000CF90BF90AF909F908F9008956DEB77E331
:1035100086E095EB60CF8F929F92AF92BF92CF9251
:10352000DF92EF92FF926B017C0120E030E0A90175
:103530000E9404E287FD6BC06DEB77E386E095E3C4
:10354000A70196010E94FBE86B017C0120E030E0BE
:1035500040E251E40E946AE220E030E040E251E4BF
:103560000E946AE24B015C0120E030E0A901C70142
:10357000B6010E9404E220E030E040EA50E487FF18
:1035800004C020E030E040EA50ECC501B4010E94E4
:10359000FBE820E030E040E251E40E947EE90E9436
:1035A000F0E99B018BE237FF05C022273327261B5A
:1035B000370B8DE28093A00BC90164E670E00E9496
:1035C000DDE8CB01EAE0F0E0BF010E94DDE8805DCC
:1035D0008093A10BC901BF010E94DDE8282FCB0118
:1035E000BF010E94DDE8805D8093A20B8EE2809394
:1035F000A30B205D2093A40B80EA9BE0FF90EF904B
:10360000DF90CF90BF90AF909F908F9008956DEB1B
:1036100077E386E095EB94CF8F929F92AF92BF9223
:10362000CF92DF92EF92FF92CF936B017C0120E06B
:1036300030E0A9010E9404E287FDAAC06DEB77E3A8
:1036400086E095E3A70196010E94FBE86B017C01EF
:1036500020E030E0A9010E9404E287FF9EC0C7017C
:10366000B601905820E030E040E251E40E946AE266
:1036700020E030E040E251E40E946AE220E030E0E5
:1036800040EA50E40E94FBE820E030E040E251E4F0
:103690000E947EE90E94F0E96B017C0180E2809348
:1036A0009E0B60E280E1C81687E2D806E104F104CF
:1036B0008CF0C701B60120E137E240E050E00E9403
:1036C0006EE8CA01B9012AE030E040E050E00E9413
:1036D0006EE8605D60939F0B60E288EEC81683E041
:1036E000D806E104F1048CF0C701B60128EE33E0FE
:1036F00040E050E00E946EE8CA01B9012AE030E0E3
:1037000040E050E00E946EE8605D6093A00B60E2D4
:1037100084E6C816D104E104F1048CF0C701B601B7
:1037200024E630E040E050E00E946EE8CA01B901B2
:103730002AE030E040E050E00E946EE8605D609377
:10374000A10B8AE0882E912CA12CB12CC701B601C7
:10375000A50194010E946EE8C62FCA01B901A50116
:1037600094010E946EE8605D6093A20B8EE28093EC
:10377000A30BC05DC093A40B8EE99BE0CF91FF909B
:10378000EF90DF90CF90BF90AF909F908F90089573
:103790006DEB77E386E095EB55CF20E030E040E23B
:1037A00051E4C701B60162CFCF92DF92EF92FF9250
:1037B000CF93DF9300D000D0CDB7DEB76B017C0193
:1037C00020E030E0A9010E9404E287FD1BC06DEB00
:1037D00077E386E095E3A70196010E94FBE8698301
:1037E0007A838B839C83CE0101960E9438160F90BA
:1037F0000F900F900F90DF91CF91FF90EF90DF909F
:10380000CF9008956DEB77E386E095EBE4CFCF9210
:10381000DF92EF92FF926B017C0120E030E0A90182
:103820000E9404E287FD26C06DEB77E386E095E316
:10383000A70196010E94FBE86B017C0120E030E0CB
:10384000A9010E9404E220E030E040E05FE387FF4E
:1038500004C020E030E040E05FEBC701B6010E9409
:10386000FBE80E94F0E9CB01FF90EF90DF90CF9052
:103870000C94F0186DEB77E386E095EBD9CFCF93FE
:10388000DF93EC01CB01BA010E940BE220E030E0B3
:1038900040E251E40E947EE920E030E0A9010E946C
:1038A000FBE8688379838A839B83DF91CF910895B6
:1038B000CF93DF93EC01CB01BA010E940BE220E031
:1038C00030E040E251E40E947EE920E030E0A901CE
:1038D0000E94FBE8688379838A839B83DF91CF9181
:1038E00008950E940BE220E030E040E251E40E94A3
:1038F0007EE920E030E0A9010E94FBE80C940C1B5B
:103900000E940BE220E030E040E251E40E947EE9B8
:1039100020E030E0A9010E94FBE80C948B1ACF93C1
:10392000DF93EC01CB01BA010E940BE220E030E012
:1039300048EC52E40E947EE920E030E0A9010E94B8
:10394000FBE8688379838A839B83DF91CF91089515
:10395000CF93DF93EC01CB01BA010E940BE220E090
:1039600030E048EC52E40E947EE920E030E0A9011A
:103970000E94FBE8688379838A839B83DF91CF91E0
:1039800008950E940BE220E030E048EC52E40E94EF
:103990007EE920E030E0A9010E94FBE80C94D519F3
:1039A000CF93DF93EC01CB01BA010E940BE220E040
:1039B00030E0A9010E94FBE8688379838A839B83B6
:1039C000DF91CF910895CF93DF93EC01CB01BA0142
:1039D0000E940BE220E030E0A9010E94FBE868832E
:1039E00079838A839B83DF91CF9108950E940BE2B4
:1039F00020E030E0A9010E94FBE80C94071CCF9363
:103A0000DF93EC01CB01BA010E940BE22AE037ED13
:103A100043E25DE30E947EE920E030E0A9010E94DC
:103A2000FBE80E94F7E9688379838A839B83DF91AF
:103A3000CF9108950E940BE22AE037ED43E25DE367
:103A40000E947EE920E030E0A9010E94FBE80C948E
:103A5000BC19CF93DF93EC01CB01BA010E940BE2BA
:103A60002AE037ED43E25DE30E947EE920E030E0AA
:103A7000A9010E94FBE8688379838A839B83DF9195
:103A8000CF9108950E940BE22AE037ED43E25DE317
:103A90000E947EE920E030E0A9010E94FBE80C943E
:103AA000D41B0E940BE220E030E0A9010E94FBE859
:103AB0000C94D41BCF92DF92EF92FF92CF93DF93BF
:103AC00000D000D0CDB7DEB70E940BE220E030E09E
:103AD00048EC52E40E947EE920E030E0A9010E9417
:103AE000FBE86B017C0120E030E0A9010E9404E2C8
:103AF0002DEB37E346E055E387FF04C02DEB37E3BA
:103B000046E055EBC701B6010E94FBE869837A8362
:103B10008B839C83CE0101960E9437170F900F90E4
:103B20000F900F90DF91CF91FF90EF90DF90CF90AB
:103B30000895CF93DF93EC01CB01BA010E940BE211
:103B400020E030E0A9010E94FBE80E94F0E97983BF
:103B50006883DF91CF9108950E940BE220E030E06E
:103B6000A9010E94FBE80E94F0E9CB010C94F01837
:103B7000CF93DF93EC01CB01BA010E940BE220E06E
:103B800030E04AE754E40E947EE920E030E0A901F9
:103B90000E94FBE8688379838A839B83DF91CF91BE
:103BA000089580914C1390914D13891B8F7039F4B7
:103BB00081E09091BB0B913019F080E0089581E095
:103BC0000895E0917E04E63010F581E08E0F809339
:103BD0007E0440919A0B50919B0B60919C0B7091CD
:103BE0009D0B9091950B8091960B28E0E29FF00140
:103BF0001124E25CFB4F20915E1330915F133183FF
:103C000020834283538364837583968387830895D7
:103C1000FC0184910895FC018081089590917102C6
:103C200081E089270C94B3724091EB0221E0422796
:103C30006CE070E00C94C9B44091EB0221E04227A3
:103C400064E070E00C94C9B44091EB0221E042279B
:103C500061E070E00C94C9B44091EB0221E042278E
:103C600062E070E00C94C9B44091EB0221E042277D
:103C700061E070E00C94C9B44091EB0221E042276E
:103C800068E070E00C94C9B44091EB0221E0422757
:103C90006CE070E00C94C9B441E061E070E00C9419
:103CA000C9B44091EB0221E042270C94C9B462E010
:103CB00070E00C9434BD6CE070E00C9434BD64E0B2
:103CC00070E00C9434BD61E070E00C9434BD61E0B0
:103CD00070E00C9434BD6CE070E00C9434BD0C9436
:103CE000A8BD0C94A8BDCF93DF9380914C13909105
:103CF0004D13891B80958F7019F40E94267EF5CF95
:103D000080914C138F5F8F70A0914C139BE5A99FFE
:103D1000D0011124FD01EA5EF34FEF0119929A954B
:103D2000E9F798E09083A55DB34F90E1EEE4F3E10D
:103D300001900D929A95E1F720914C1390914D13BB
:103D4000291303C094E69093491380934C13DF9199
:103D5000CF910C94A273CF92DF92EF92FF920F93C8
:103D60001F93C12CD12C76018C0126ED3BE042ED56
:103D70005BE06EEC7BE08AEC9BE00E9421B41F913B
:103D80000F91FF90EF90DF90CF9008958F929F92C8
:103D9000AF92BF92EF92FF920F931F93CF93DF9357
:103DA000EC018B01E42EF22E80915E1390915F1353
:103DB0008C179D0709F43EC020914B0227FD1092FD
:103DC0004B022BE5CB39D20709F03FC0855791460E
:103DD00071F40E949CBD6E517B4F8F4F9F4F60933B
:103DE0007F04709380048093810490938204D09325
:103DF0005F13C0935E1330E020E000939A0B1093A2
:103E00009B0B20939C0B30939D0BE092950BF092B3
:103E1000960BC557D14621F41092940B10927E0454
:103E200082E08093670181E08093970B10927D047C
:103E30001092930BDF91CF911F910F91FF90EF9014
:103E4000BF90AF909F908F90089521E6C537D2071D
:103E500071F68B599B4519F0C5E7D1E6C8CF0E9492
:103E60009CBD80907F0490908004A0908104B090CD
:103E70008204681979098A099B0997FFEDCF80911F
:103E8000AF0B8770873041F7CAEDD2E5B0CF20E0A5
:103E900040E070E060E08FE690E20C94C61E8091F6
:103EA000130C811114C080917401909175010197D8
:103EB00020910013309101132817390744F420E0B2
:103EC00040E070E060E084E790E20C94C61E0C9441
:103ED000471F21E02093940BFC0180819181A281F6
:103EE000B3818093120190931301A0931401B093B6
:103EF000150120E040E070E060E080918C0B909133
:103F00008D0B0C94C61ECF93DF9300D000D0CDB79D
:103F1000DEB78DEC9CECACECBCE389839A83AB837D
:103F2000BC83CE0101960E94691F0F900F900F90E5
:103F30000F90DF91CF910895CF93DF9300D000D001
:103F4000CDB7DEB78DEC9CECACECBDE389839A83F6
:103F5000AB83BC83CE0101960E94691F0F900F9026
:103F60000F900F90DF91CF910895CF93DF9300D002
:103F700000D0CDB7DEB780E090E0A0E8BFE3898352
:103F80009A83AB83BC83CE0101960E94691F0F9078
:103F90000F900F900F90DF91CF910895CF93DF9303
:103FA00000D000D0CDB7DEB780E090E0A0E2B1E471
:103FB00089839A83AB83BC83CE0101960E94691FDB
:103FC0000F900F900F900F90DF91CF910895CF92A7
:103FD000DF92EF92FF92CF93C82F0E949CBD6B019E
:103FE0007C0124EA30E74DE75FE3609112017091B4
:103FF000130180911401909115010E9404E287FD44
:1040000018C08AEF90E0A0E0B0E08C0D9D1DAE1DC1
:10401000BF1D80931F0490932004A0932104B093AC
:104020002204C0931001CF91FF90EF90DF90CF90CA
:10403000089580E090E0DC01E8CFCF93DF9300D0DB
:1040400000D0CDB7DEB784EF91E0A0E0B0E0898387
:104050009A83AB83BC83BE016F5F7F4F88E70E946A
:10406000FD740F900F900F900F90DF91CF910895F6
:10407000CF93C82FCB010E94F3768AE598E00E9487
:10408000F3768BE498E0CC2311F080E598E00E9471
:10409000F3768AE0CF910C944776CF93DF93CDB738
:1040A000DEB720E24F8158856E818D810E94F8B87D
:1040B000DF91CF9108956FEF80918E0B0C9448BEE5
:1040C00061E372E482E00C94D6D666E372E481E0A8
:1040D0000C94D6D66BE372E480E00C94D6D660E400
:1040E00072E483E00C94D6D6EF92FF920F931F9365
:1040F0008FE3E82E87E0F82E01E417E02BE530E4AB
:1041000047E45FE161E577E086E597E00E9405C15D
:104110001F910F91FF90EF900895EF92FF920F93F0
:104120001F9383ECE82E86E0F82E0DE017E02BE5D8
:1041300030E44EEC5DE565EC76E08AEC96E00E94BA
:1041400005C11F910F91FF90EF900895EF92FF929C
:104150000F931F938CE6E82E84E0F82E0FE714E00F
:1041600030E020E04CE55BE56EE674E085E794E046
:104170000E9405C11F910F91FF90EF9008958091CB
:104180006701882341F0609183047091840441E0C9
:1041900081E00C949BB80895CF92DF92EF92FF924A
:1041A000CF93DF9300D000D0CDB7DEB76B017C0199
:1041B00020E030E0A9010E9404E287FD1BC06DEB06
:1041C00077E386E095E3A70196010E94FBE8698307
:1041D0007A838B839C83CE0101960E9479B90F90DC
:1041E0000F900F900F90DF91CF91FF90EF90DF90A5
:1041F000CF9008956DEB77E386E095EBE4CF0E94D6
:104200000BE220E030E04AE754E40E947EE920E03F
:1042100030E0A9010E94FBE80C94CC20EF92FF92C1
:104220000F931F93CF93DF93EC018B017A018A8563
:104230009B858617970731F0888199810E94A7C2D4
:104240001B870A87B701888199810E9439B92E811D
:104250003F81820F932F911D9F838E8390E080E09A
:10426000DF91CF911F910F91FF90EF9008959F9252
:10427000AF92BF92CF92DF92EF92FF920F931F9374
:10428000CF93DF93EC018B01942EA52E8A859B851D
:104290008617970731F0888199810E94A7C21B87F2
:1042A0000A8788859985019649F5BC800A818E81A7
:1042B000080FC880D980D6015596ED91FC91C601B2
:1042C0000995B80EE92CFA2C10E0F70121917F0135
:1042D000211127C08E819F81810F911D9F838E8325
:1042E00090E080E0DF91CF911F910F91FF90EF90D0
:1042F000DF90CF90BF90AF909F9008950E811F8167
:10430000692D7A2D888199810E9439B9800F912F6A
:10431000911D288539852817390738F681E090E006
:10432000E1CF4B2D602FC6010E94FFC2080F180F6E
:10433000CCCFAF92BF92DF92EF92FF920F931F9379
:10434000CF93DF938C01EB01D42E79018FE04817D6
:1043500009F486C0A5E14A17B1F1BAE04B130EC0CB
:10436000EC81FD8130E020E042E061E0C801099588
:104370004EED51E0BE01C8010E94AAC30A80DB8154
:10438000C02DF2E3DF1609F4E2C0FD1508F491C078
:1043900085E1D81609F4E0C0A7E1DA1609F4EFC008
:1043A000B4E1DB127BC0EE81FF818D8190E0880F4C
:1043B000991F8E0F9F1F11928E179F07E1F7CE0155
:1043C0000E94F2BE6BC0AA80BB8049EC51E0C801DC
:1043D0000E94AAC3F5014481440F406BBE01C8018D
:1043E0000E9492C341E0BE01C8010E949AC3D50158
:1043F00016962D913C911797EC81FD8115964C9165
:1044000066E0C801099540E0BE01C8010E94A2C350
:1044100049EC51E0BE01C8010E94AAC3F5014481E4
:10442000440F4F5F406BBE01C8010E9492C341E040
:10443000BE01C8010E949AC3D50115964C911597EB
:1044400016962D913C91240F311DEC81FD8166E083
:10445000C801099540E0BE01C8010E94A2C38ECFE9
:1044600041E0C8010E94A2C340E0BE01C8010E9411
:104470009AC341E8BE01C8010E9492C3F70140817E
:1044800050E05595479555954795BE01C8010E9446
:1044900092C340E0BE01C8010E94A2C381E0DF9147
:1044A000CF911F910F91FF90EF90DF90BF90AF9051
:1044B0000895E6E4DE1609F471C0F7E4DF1609F4A6
:1044C00071C08BE3D812EACFD70111969C91119756
:1044D00013968C9138E0390F813031F0833011F030
:1044E000392F02C0392F985021E04B81491708F429
:1044F00020E041E0391708F040E091E05A8135179B
:1045000008F490E0322F342B932311F4242331F25A
:10451000F701128100E0D12C843048F490E0FC01D6
:10452000ED53FE4FD08081549E4FDC010C9117FF5C
:1045300004C0B701CE010E94F9BEF70180818D0D44
:1045400080838181800F8183110F89F7A7CFB70105
:10455000CE010E94F9BEA2CFCE010E94DCBE88230C
:1045600009F49DCFEE81FF818D8190E0880F991F26
:104570008E0F9F1F11928E179F07E1F78FCFD701E4
:104580001C928A8111968C9311978D81815012967D
:104590008C9312978B8113968C9380CF8D81F7012A
:1045A00080837CCF8981D7018C9378CF0F930FB70D
:1045B0000F9300916E000F930B7F00936E0000919C
:1045C0006F000D7F00936F000F930BB70F930CB725
:1045D0000F921F922F933F934F935F936F937F930D
:1045E0008F939F93AF93BF93EF93FF9311240E94F8
:1045F000BBCCFF91EF91BF91AF919F918F917F9134
:104600006F915F914F913F912F911F900F900CBF31
:104610000F910BBF0F910260F89400936F000F9100
:1046200000936E000F910FBF0F911895EF92FF92BC
:104630000F931F93E092EC02F092ED020093EE02D2
:104640001093EF0260931A0570931B0580931C056D
:104650009FEFFF27621B730B840B30F480957095DE
:104660006195790B890B99279093BA04A6E06A9F0C
:104670000092AE04512DEE277A9F500DE11D8A9FC6
:10468000E00D5093AF04E093B004AFE06A9F009256
:10469000B204512DEE277A9F500DE11D8A9FE00D47
:1046A0005093B304E093B404AAE06A9F0092B60466
:1046B000512DEE277A9F500DE11D8A9FE00D5093FA
:1046C000B704E093B8041F910F91FF90EF90089505
:1046D00000000000000000008091420580FF27C01C
:1046E000459A8FEF8093160580914205869580FF4D
:1046F00021C0479A8FEF80931705809142058695D8
:10470000869580FF1AC02A988FEF809318058091B4
:10471000420586958695869580FF12C0289A8FEF70
:1047200080931905000000000000000008954598DE
:1047300081E0D8CF479881E0DECF2A9A81E0E5CFAB
:10474000289881E0EDCF833B21E0920714F083EBC2
:1047500091E090930313809302130C94A8BDAF9241
:10476000BF92CF92DF92EF92FF920F931F93CF935E
:10477000DF93C7ECD1E10AEE1BE087EDA82E81E1C3
:10478000B82EC12CD12C7601C3946991799189916D
:1047900099910E9409E2288939894A895B890E9496
:1047A0006AE20E94F7E9F801619371938193919312
:1047B0008F01C616D706E806F90610F46B017C01D6
:1047C000AC16BD0611F76FEF7FEFCB01A701960185
:1047D0000E944CE82093FA0B3093FB0B4093FC0BA8
:1047E0005093FD0BDF91CF911F910F91FF90EF90B0
:1047F000DF90CF90BF90AF9008950F931F93CF930A
:10480000DF930BED11E1C3E0DCE0F8012191319180
:10481000419151918F0160E070E080E89FE30E9438
:104820007EE96993799389939993FCE0C331DF071B
:1048300061F70E9483B4DF91CF911F910F910C9487
:10484000AF230C94FD230C94FD230C94FD230C94B6
:10485000FD230C94AF230C94AF230C94AF230C9442
:10486000AF2390914C1380914D13981306C0809103
:10487000140C9091150C892B19F00E94267EF1CF13
:10488000089590914C1380914D13981308C0809116
:10489000140C9091150C892B11F40C94E3730E9465
:1048A000267EEFCFCF93DF9320917102222379F000
:1048B000EC010E94C6709B01AC01688579858A85F0
:1048C0009B850E94FAE8688779878A879B87DF91B2
:1048D000CF910895CF93DF9320917102222379F035
:1048E000EC010E94C6709B01AC01688579858A85C0
:1048F0009B850E94FBE8688779878A879B87DF9181
:10490000CF910895CF9383E50E947270882331F090
:104910000E941370909323018093220182E40E94ED
:104920007270882331F00E9413709093210180935C
:10493000200186E40E9441708823B9F00E9417701C
:1049400060931C0170931D0180931E0190931F01C1
:10495000C1E020E030E0A9010E9404E2811101C021
:10496000C0E0C0933D05CF91089560E070E0CB01B9
:10497000E7CF2F923F924F925F926F927F928F92EA
:104980009F92AF92BF92CF92DF92EF92FF920F93DE
:104990001F93CF93DF93CDB7DEB76C970FB6F89424
:1049A000DEBF0FBECDBF8C015B015A834983FC0182
:1049B000EA5BFF4F208131814281538129873A8709
:1049C0004B875C87CA01B9010E9409E26B017C0137
:1049D000D5012D913D914D915C910E946AE20E941A
:1049E00067E92B013C01E981FA8120813181428113
:1049F0005381C701B6010E946AE20E9467E94B0138
:104A00005C01C301B2010E94F7E9698B7A8B8B8B41
:104A10009C8B683771058105910540F428E730E0EB
:104A200040E050E0298B3A8B4B8B5C8BC501B40185
:104A30000E94F7E96D877E878F87988B68377105AD
:104A40008105910540F448E750E060E070E04D8753
:104A50005E876F87788BF801EE5AFF4F4080518058
:104A600062807380C301B2010E940BE269837A8382
:104A70008B839C8369897A898B899C890E9409E24E
:104A80006D8B7E8B8F8B988F20E030E0A901698140
:104A90007A818B819C810E9404E2882309F4E1C120
:104AA000A7019601C701B6010E946AE24B015C01B1
:104AB0002D893E894F89588DCA01B9010E946AE249
:104AC0009B01AC01C501B4010E94FAE84B015C01F5
:104AD00029813A814B815C81CA01B9010E94FBE8BE
:104AE0009B01AC01C501B4010E947EE90E9467E907
:104AF0000E94F7E96D837E838F83988766277727E7
:104B0000CB0164197509860997090E940BE24B01D4
:104B10005C016D857E858F8598890E9409E22B0155
:104B20003C0120E030E0A901C501B4010E9404E28B
:104B3000882309F49AC1A3019201C301B2010E9422
:104B40006AE2698F7A8F8B8F9C8FA7019601C701CC
:104B5000B6010E946AE29B01AC01698D7A8D8B8D52
:104B60009C8D0E94FAE86B017C01A5019401C501AE
:104B7000B4010E94FBE89B01AC01C701B6010E9491
:104B80007EE90E9426EAD80195968D909D90AD9081
:104B9000BC909897750164012D813E814F815885A5
:104BA000C21AD30AE40AF50A0E94F7E9C61AD70A1C
:104BB000E80AF90AF7FE8EC02D893E894F89588D83
:104BC000CA01B9010E946AE26B017C0129813A8124
:104BD0004B815C81CA01B9010E94FBE869877A8731
:104BE0008B879C8720E030E0A90169817A818B81E5
:104BF0009C810E9404E2882309F43BC1C501B401F1
:104C00000E9409E229853A854B855C850E946AE20B
:104C1000A70196010E94FAE86D837E838F839887AF
:104C2000A3019201C301B2010E946AE29B01AC019F
:104C30006D817E818F8198850E94FBE82B013C016C
:104C400020E030E040E850E469817A818B819C81EA
:104C50000E946AE29B01AC01C301B2010E947EE99D
:104C60000E9467E92B013C0120E030E0A9010E948D
:104C70007EEA18161CF0412C512C3201C301B201FE
:104C80000E94F7E96D837E838F8398878616970647
:104C9000A806B90620F48D829E82AF82B8866D8107
:104CA0007E818F8198850E9409E229853A854B850E
:104CB0005C850E946AE2A70196010E94FBE80E94BF
:104CC000BCEA0E94F7E969877A878B879C87C12CA9
:104CD000D12C760169857A858B859C8529893A89CD
:104CE0004B895C89621B730B840B950B0E9409E254
:104CF00029813A814B815C810E947EE920E034E287
:104D000044EF59E40E946AE20E94F7E94B015C011A
:104D100069857A858B859C852D853E854F8558894B
:104D2000621B730B840B950B0E9409E229813A8167
:104D30004B815C810E947EE920E034E244EF59E43B
:104D40000E946AE20E94F7E92B013C013FE68316CC
:104D50009104A104B10408F090C0F401EE0FFF1F0C
:104D6000EE0FFF1FE25EF64F85919591A591B491EC
:104D70008983292E3A2EBD8B4FE6441651046104D7
:104D8000710408F083C0F201EE0FFF1FEE0FFF1F4A
:104D9000E25EF64F45915591659174919A01CB0170
:104DA0004D815E816F817885D80199964D935D9391
:104DB0006D937C939C974C0D5D1D6E1D7F1DF801BE
:104DC00045A756A767A770ABE65BFF4F49895A898D
:104DD0006B897C894083518362837383D5968D92DE
:104DE0009D92AD92BC92D897F80141AE52AE63AE9F
:104DF00074AEFD9649814083218232825D8953835E
:104E00003496208331838283938369857A858B8569
:104E10009C85D1966D937D938D939C93D4973D966D
:104E20002D853E854F855889208331834283538366
:104E30006C960FB6F894DEBF0FBECDBFDF91CF9159
:104E40001F910F91FF90EF90DF90CF90BF90AF90A8
:104E50009F908F907F906F905F904F903F902F909A
:104E6000089560E070E0CB0141CE60E070E0CB01DE
:104E700088CE60E070E0CB01F3CEC501B4010E94A2
:104E8000D3146983272E382E9D8B76CFC301B201B0
:104E90000E94D3149B0184CF90916F0081E091FD1B
:104EA00002C080E0089590916F009D7F90936F0005
:104EB00008950E944C271092FE0B1092FF0B109247
:104EC000000C1092010C81110C94A27308950F93A1
:104ED0001F9380914C1390914D13891B8F7009F48F
:104EE00049C090914913992361F0833040F48FEFCA
:104EF000890F29F08093491390E080E038C0109228
:104F0000491380914D132BE5829FC00111248A5EC5
:104F1000934FFC01208120FDEFCF4091FE0B50917B
:104F2000FF0B6091000C7091010CE95AFF4F00815A
:104F3000118122813381401B510B620B730B409313
:104F4000FE0B5093FF0B6093000C7093010C2091AB
:104F50004D132F5F2F7020934A1330914D132091E2
:104F60004B13321304C020914A1320934B131F910B
:104F70000F9108950E945927BFCFFC0120813181F4
:104F8000428153816091E7117091E8118091E9119C
:104F90009091EA110E946AE20E9483EA60935A1398
:104FA00070935B1380935C1390935D1390914C13FB
:104FB00080914D1398130C94731E0E9431240E940B
:104FC0004C2740915A1350915B1360915C13709180
:104FD0005D134093370550933805609339057093FE
:104FE0003A0581110C94A27308954F925F926F92CB
:104FF0007F928F929F92AF92BF92CF92DF92EF9269
:10500000FF920F931F93CF93DF93EC018B015A0113
:10501000F9012091E7113091E8114091E911509187
:10502000EA1160817181828193810E946AE20E940B
:1050300083EA6B017C012091E3113091E4114091EE
:10504000E5115091E611F5016081718182819381B2
:105050000E946AE20E9483EA4B015C012091DF1109
:105060003091E0114091E1115091E211F80160811D
:105070007181828193810E946AE20E9483EA2B01FE
:105080003C012091DB113091DC114091DD115091F8
:10509000DE11688179818A819B810E946AE20E9487
:1050A00083EA60934E1370934F1380935013909341
:1050B00051134092521350925313609254137092B2
:1050C00055138092561390925713A0925813B09292
:1050D0005913C0925A13D0925B13E0925C13F09272
:1050E0005D1390914C1380914D13981791F0DF91BF
:1050F000CF911F910F91FF90EF90DF90CF90BF90D5
:10510000AF909F908F907F906F905F904F900C9496
:10511000731E0E9431240E944C27409156135091D7
:1051200057136091581370915913009152131091B5
:1051300053132091541330915513C0904E13D090B7
:105140004F13E0905013F0905113C0922B05D09262
:105150002C05E0922D05F0922E0500932F0510935B
:105160003005209331053093320540933305509339
:105170003405609335057093360540915A1350916C
:105180005B1360915C1370915D13409337055093EE
:1051900038056093390570933A05882391F0DF91C3
:1051A000CF911F910F91FF90EF90DF90CF90BF9024
:1051B000AF909F908F907F906F905F904F900C94E6
:1051C000A273DF91CF911F910F91FF90EF90DF902D
:1051D000CF90BF90AF909F908F907F906F905F9097
:1051E0004F900895CF92DF92EF92FF92CF93DF938B
:1051F000C82F0E944C2794E0C99FE0011124FE01B2
:10520000E55DFA4FC080D180E280F38081110E9479
:10521000A273CD5FD34FC701B6010E940BE2288174
:1052200039814A815B810E946AE2DF91CF91FF90D0
:10523000EF90DF90CF900895CF92DF92EF92FF92A0
:10524000CF93DF93C82F0E944C2794E0C99FE001C1
:105250001124FE01E15EFA4FC080D180E280F3802C
:1052600081110E94A273CD5FD34FC701B6010E9486
:105270000BE2288139814A815B810E946AE2DF91D9
:10528000CF91FF90EF90DF90CF900895CF93DF9371
:1052900024E0829FC0011124EC01C454D44FFC01CE
:1052A000EB5BFA4F8F599D4FDC012D913D914D9154
:1052B0005C9160817181828193810E94FBE86883A7
:1052C00079838A839B83DF91CF91089580FF04C007
:1052D0009091A00490FD8E7F81FF05C09091A00465
:1052E000969590FD8D7F82FF06C09091A0049695C3
:1052F000969590FD8B7F08952F923F924F925F92EB
:105300006F927F928F929F92AF92BF92CF92DF92D5
:10531000EF92FF920F931F93CF93DF93CDB7DEB73A
:10532000A6970FB6F894DEBF0FBECDBF80912601C1
:10533000882309F4CDC08091A004C82ED12CF12C73
:10534000E12C80FF3CC08090280190902901A09022
:105350002A01B0902B0120915102309152024091CC
:10536000530250915402C501B4010E947EEA1816FE
:1053700044F48092510290925202A0925302B09251
:1053800054028090340190903501A0903601B09085
:1053900037012091510230915202409153025091B5
:1053A0005402C501B4010E9404E287FF08C0809244
:1053B000510290925202A0925302B0925402D7012D
:1053C000C601B695A7959795879580FF3CC08090BC
:1053D0002C0190902D01A0902E01B0902F012091D2
:1053E0005502309156024091570250915802C50122
:1053F000B4010E947EEA181644F4809255029092FD
:105400005602A0925702B0925802809038019090B4
:105410003901A0903A01B0903B01209155023091A2
:1054200056024091570250915802C501B4010E94A2
:1054300004E287FF08C08092550290925602A09223
:105440005702B092580292E0F694E794D794C7942A
:105450009A95D1F7C0FE3CC0C0903001D090310188
:10546000E0903201F09033012091590230915A02BC
:1054700040915B0250915C02C701B6010E947EEA36
:10548000181644F4C0925902D0925A02E0925B027C
:10549000F0925C02C0903C01D0903D01E0903E0152
:1054A000F0903F012091590230915A0240915B02E5
:1054B00050915C02C701B6010E9404E287FF08C058
:1054C000C0925902D0925A02E0925B02F0925C02C2
:1054D0008091C61183FD7EC02091D60B3091D70BF1
:1054E0004091D80B5091D90B60915D0270915E0292
:1054F00080915F02909160020E9404E2882309F487
:1055000069C01091130C111161C0809174019091C8
:105510007501019720910013309101132817390765
:105520003CF40E94BB7C88EA98E00E94F37611E08C
:105530002091D60B3091D70B4091D80B5091D90BBD
:1055400060915D0270915E0280915F0290916002B5
:105550000E94FAE86B017C0120E030E0A9010E9482
:105560007EEA87FF04C0F7FAF094F7F8F0942091F0
:105570007001309171014091720150917301C70126
:10558000B6010E946AE220E030E84BE354E40E9456
:105590007EEA1816ECF40E94BB7C89E898E00E9431
:1055A000F37680915D0290915E02A0915F02B091CE
:1055B00060028093D60B9093D70BA093D80BB09337
:1055C000D90B8DE592E00E94BD2704C010E0B0CF5A
:1055D0001111E7CF2AE037ED43E25CE36091180157
:1055E0007091190180911A0190911B010E946AE249
:1055F0006B017C016091160170911701072E000C60
:10560000880B990B0E940BE29B01AC01C701B6010C
:105610000E946AE2698B7A8B8B8B9C8B80917102E2
:10562000882309F46CC02091CA0B3091CB0B4091B8
:10563000CC0B5091CD0B6091510270915202809130
:105640005302909154020E94FAE86D8B7E8B8F8BEF
:10565000988F2091CE0B3091CF0B4091D00B509171
:10566000D10B609155027091560280915702909132
:1056700058020E94FAE8698F7A8F8B8F9C8F209155
:10568000D20B3091D30B4091D40B5091D50B60913C
:10569000590270915A0280915B0290915C020E94C3
:1056A000FAE86D8F7E8F8F8F98A32091D60B309163
:1056B000D70B4091D80B5091D90B60915D0270913E
:1056C0005E0280915F02909160020E94FAE86B0195
:1056D0007C0120E030E0A9016D897E898F89988D59
:1056E0000E9404E281110FC020E030E0A901698D21
:1056F0007A8D8B8D9C8D0E9404E2811104C0C12C97
:10570000D12C76012CC12D893E894F89588DCA0133
:10571000B9010E946AE24B015C01298D3A8D4B8DE3
:105720005C8DCA01B9010E946AE29B01AC01C5010E
:10573000B4010E94FBE84B015C012D8D3E8D4F8D25
:1057400058A1CA01B9010E946AE29B01AC01C501DE
:10575000B4010E94FBE84B015C01A7019601C7015F
:10576000B6010E946AE29B01AC01C501B4010E942E
:10577000FBE80E94BCEA4B015C012DEB37E346E8F5
:1057800055E30E9404E287FF0FC020E030E0A9014A
:10579000C701B6010E947EEA4601570187FF04C097
:1057A000B7FAB094B7F8B0942DEB37E346E855E379
:1057B000C501B4010E9404E287FDDEC020E030E0B4
:1057C00040EA51E4C501B4010E947EE90E94F7E974
:1057D0001B01672B19F422242394312CB10190E092
:1057E00080E00E9409E29B01AC0160E070E080E88B
:1057F0009FE30E947EE92B013C01AC019B01C501A6
:10580000B4010E946AE24B015C01A30192016D891F
:105810007E898F89988D0E946AE26D8B7E8B8F8B3B
:10582000988FA3019201698D7A8D8B8D9C8D0E943A
:105830006AE2698F7A8F8B8F9C8FA30192016D8DA5
:105840007E8D8F8D98A10E946AE26D8F7E8F8F8FE3
:1058500098A3A3019201C701B6010E946AE269A35D
:105860007AA38BA39CA380E1EAECFBE08E010F5F9F
:105870001F4FD80101900D928A95E1F70E949CBDBF
:105880002B013C0128EC420E511C611C711C0DA324
:105890001EA381E0281A310809F45FC00E949CBD54
:1058A0008B019C01041915092609370937FD86C0AB
:1058B0002B013C0128EC420E511C611C711C0E9402
:1058C000267E2D893E894F89588D69817A818B8109
:1058D0009C810E94FBE869837A838B839C83298D5A
:1058E0003A8D4B8D5C8D6D817E818F8198850E9474
:1058F000FBE86D837E838F8398872D8D3E8D4F8D42
:1059000058A169857A858B859C850E94FBE869870B
:105910007A878B879C8729A13AA14BA15CA16D85D1
:105920007E858F8598890E94FBE86D877E878F87AB
:10593000988B750164018E010F5E1F4F9E01235FDE
:105940003F4FAE01475F5F4FBE016B5F7F4F8DA141
:105950009EA10E9421B481119CCF750164018E012A
:105960000F5E1F4F2DE532E049E552E065E572E03C
:1059700081E592E00E9421B480E1E1E5F2E0AAEC49
:10598000BBE001900D928A95E1F7A6960FB6F894C8
:10599000DEBF0FBECDBFDF91CF911F910F91FF9062
:1059A000EF90DF90CF90BF90AF909F908F907F90BF
:1059B0006F905F904F903F902F9008950E945DC828
:1059C00080CF80919C0490919D04A0919E04B09101
:1059D0009F048093180190931901A0931A01B0932A
:1059E0001B0180919A0490919B04909317018093DE
:1059F000160108958091180190911901A0911A0142
:105A0000B0911B0180939C0490939D04A0939E04ED
:105A1000B0939F04809116019091170190939B047D
:105A200080939A0484E690E0909317018093160186
:105A300008954F925F926F927F928F929F92AF9252
:105A4000BF92CF92DF92EF92FF920F931F93CF936B
:105A5000DF93CDB7DEB72C970FB6F894DEBF0FBE3D
:105A6000CDBF2B013C0129873A874B875C874701D3
:105A70005801F601E080F1800281138120E030E0DE
:105A8000A901B701C8010E9404E2882309F488C073
:105A90005E2D4F2D302F212F852F942FA32FB22F26
:105AA00089839A83AB83BC8320E030E0A901B701EE
:105AB000C8010E9404E2811108C0E0906801F090E2
:105AC000690100916A0110916B01C701D8018D83B2
:105AD0009E83AF83B887A50194016091D20B70912A
:105AE000D30B8091D40B9091D50B0E9404E287FFD9
:105AF0000CC08092D20B9092D30BA092D40BB09298
:105B0000D50BCE0101960E94AB1E4092CA0B50925B
:105B1000CB0B6092CC0B7092CD0B89859A85AB85AF
:105B2000BC858093CE0B9093CF0BA093D00BB093FA
:105B3000D10BCE0105960E94AB1EA5019401609188
:105B4000D20B7091D30B8091D40B9091D50B0E9406
:105B50007EEA181664F48092D20B9092D30BA09236
:105B6000D40BB092D50BCE0101960E94AB1E0E94C1
:105B700031242C960FB6F894DEBF0FBECDBFDF9157
:105B8000CF911F910F91FF90EF90DF90CF90BF903A
:105B9000AF909F908F907F906F905F904F900895FF
:105BA00050E040E030E820E477CFCF92DF92EF92F0
:105BB000FF920F931F936A01E090D20BF090D30BEA
:105BC0000091D40B1091D50BFB01208131814281D2
:105BD0005381FC0160817181828193810E94192D22
:105BE0001F910F91FF90EF90DF90CF900895CF928B
:105BF000DF92EF92FF920F931F936B01FC01E08005
:105C0000F18002811381EAECFBE024813581468139
:105C1000578160817181828193810E94192D1F912A
:105C20000F91FF90EF90DF90CF900895AF92BF92C9
:105C3000CF92DF92EF92FF920F931F93CF93DF9358
:105C400000D000D0CDB7DEB7FC01E080F18002814A
:105C50001381611112C0A090D20BB090D30BC090F1
:105C6000D40BD090D50B9501A601B701C8010E94B5
:105C700004E287FF02C07501860120E030E048E4BD
:105C800053E4B701C8010E9404E287FD04C0E12C7F
:105C9000F12C08E413E4C701D80189839A83AB830C
:105CA000BC8367ED71E0CE0101960E94F72D0F9045
:105CB0000F900F900F90DF91CF911F910F91FF9058
:105CC000EF90DF90CF90BF90AF9008958F929F920A
:105CD000AF92BF92CF92DF92EF92FF921F93CF933A
:105CE000DF93CDB7DEB760970FB6F894DEBF0FBE77
:105CF000CDBF182F80E00E94F2284B015C018092FA
:105D00008E0490928F04A0929004B092910481E04E
:105D10000E94F2286B017C01C0929204D0929304FD
:105D2000E0929404F092950482E00E94F22860933D
:105D300096047093970480939804909399041D8619
:105D40001E861F86188A89829A82AB82BC82CD8287
:105D5000DE82EF82F88669877A878B879C8783E06B
:105D60000E94F2286D877E878F87988BCE010196DF
:105D70000E9452241E3FD9F480E1FE013196AAEC24
:105D8000BBE001900D928A95E1F760960FB6F8940A
:105D9000DEBF0FBECDBFDF91CF911F91FF90EF907F
:105DA000DF90CF90BF90AF909F908F90089584E048
:105DB000189FF0011124DF01A653B44F81E090E059
:105DC0008C0F9D1FE80FF91F408151816281738103
:105DD0004D935D936D937C931397D7CF0C9483B4BD
:105DE000CF930E94F72D8091660BC82FC47082FD5F
:105DF0000CC01092660B82E00E94662E0E94EE2E6E
:105E000081E0C11180E0CF9108950E94017D882337
:105E100081F3F9CFCF93DF93CDB7DEB72C970FB6D1
:105E2000F894DEBF0FBECDBF0E94FFB40E944C2786
:105E30009CE0EBE2F5E0DE01119601900D929A955F
:105E4000E1F781110E94A273CE0101960E947BCCE2
:105E50002C960FB6F894DEBF0FBECDBFDF91CF9169
:105E600008952F923F924F925F926F927F928F92FE
:105E70009F92AF92BF92CF92DF92EF92FF920F93D9
:105E80001F93CF93DF9300D01F92CDB7DEB78090E2
:105E9000CA0B9090CB0BA090CC0BB090CD0B409048
:105EA000CE0B5090CF0B6090D00B7090D10BC09068
:105EB000D20BD090D30BE090D40BF090D50B0E9476
:105EC000AF230E94D11506EE1BE088E291E09B8390
:105ED0008A838AED282E8BE0382E198289810E94D0
:105EE0004629C8010E94D16EEA81FB8161937193BA
:105EF00081939193FB83EA83C1010E94D16EEA8171
:105F0000FB816087718782879387F981FF5FF983BF
:105F10000C5F1F4F84E0280E311CF330F9F60E940D
:105F200045730E94FD23A50194016091CA0B7091F5
:105F3000CB0B8091CC0B9091CD0B0E9404E2811190
:105F40001CC0A30192016091CE0B7091CF0B809188
:105F5000D00B9091D10B0E9404E281110EC02091D0
:105F6000D20B3091D30B4091D40B5091D50BC7017C
:105F7000B6010E9404E28823B9F00F900F900F90B1
:105F8000DF91CF911F910F91FF90EF90DF90CF9015
:105F9000BF90AF909F908F907F906F905F904F9049
:105FA0003F902F900C940A2F0F900F900F90DF913D
:105FB000CF911F910F91FF90EF90DF90CF90BF9006
:105FC000AF909F908F907F906F905F904F903F9099
:105FD0002F9008952F923F924F925F926F927F92EF
:105FE0008F929F92AF92BF92CF92DF92EF92FF92E9
:105FF0000F931F93CF93DF93CDB7DEB7C358D1096B
:106000000FB6F894DEBF0FBECDBFCDB6DEB641E011
:1060100064E070E0CE0187589F4F0E94C9B441E010
:1060200062E070E0CE0183589F4F0E94C9B443E004
:1060300050E0BE0167587F4F8FED91E00E941AEB50
:10604000892B31F181E08093AD049091AD0481E022
:1060500089270FB6F894DEBE0FBECDBECD57DF4FF9
:106060000FB6F894DEBF0FBECDBFDF91CF911F9169
:106070000F91FF90EF90DF90CF90BF90AF909F90E7
:106080008F907F906F905F904F903F902F900895EA
:10609000E9961CAE1DAE1EAE1FAEE997109212130C
:1060A00010921113CE018F579F4F0E944C1EADB618
:1060B000BEB6CF57DF4F0881C158D04010E00D5F0A
:1060C0001F4F000F111F000F111F8DB79EB7801BB0
:1060D000910B0FB6F8949EBF0FBE8DBFEDB7FEB704
:1060E0003196CE57DF4FF983E883C258D040801BEA
:1060F000910B0FB6F8949EBF0FBE8DBFEDB7FEB7E4
:1061000031964F01801B910B0FB6F8949EBF0FBEC6
:106110008DBFEDB7FEB731967F01B801CE57DF4F87
:1061200088819981C258D0400E94511E4091EB0253
:1061300081E0482764E070E087ED91E10E94C9B4F6
:10614000B801C4010E94511EB801C7010E94511E2E
:106150001091EB02111153C0CF57DF4F8881C15806
:10616000D04090E00296A7ECB1E170E060E030E052
:1061700020E042E45CE0821793070CF498C0CE570D
:10618000DF4FE881F981C258D040E60FF71F408009
:106190005180628073804D925D926D927D928217E4
:1061A00093070CF48AC0F401E60FF71F20803180BA
:1061B0000281E3812101602E7E2E50964D925D92E8
:1061C0006D927C925397821793070CF480C0F7016D
:1061D000E60FF71F208031800281E3812101602ECC
:1061E0007E2E90964D925D926D927C9293972F5F4A
:1061F0003F4F6C5F7F4F2430310509F0BCCF8BEFF0
:1062000091E10E941C1E8FEF91E10E941C1E83E011
:1062100092E10E941C1E87E092E10E941C1E8BE00E
:1062200092E10E941C1E41E0412760E170E08AED8E
:106230009BE00E94C9B4CE018B589F4F0E941C1E48
:106240000FB6F894BEBE0FBEADBE85E495E00E94C9
:10625000441ECE0183599F4F0E94241E8E010F5F62
:106260001F4FC8010E941C1ECE018B589F4F0E94D9
:106270001C1ECE018B589F4F0E941C1EC8010E94FD
:106280004C1ECE0183599F4F0E944C1EE980AE9652
:106290008FADAE97E89E70011124F1E0EF1AF1087E
:1062A00000F1CE018B589F4F0E941C1EF6CFFA01C1
:1062B00045905590659074906ECFE2E3FCE0459078
:1062C0005590659074901201062DE72D73CFE2E290
:1062D000FCE045905590659074901201062DE72DD5
:1062E0007DCF8BE393E10E94441E8AE0F82EFA945E
:1062F000CE01FF2029F08B589F4F0E941C1EF7CF24
:1063000081589F4F0E944C1ECE0180589F4F0E9483
:106310004C1EC158DF4F8881CF57D040853009F0DF
:106320008AC1C058DF4F8881C058D040853009F0FD
:1063300082C18091EB02811102C00E94B37283EE90
:1063400092E00E943C1E8BED92E00E943C1E409128
:10635000EB0281E0482764E670E087E792E00E9464
:10636000C9B4C8010E94341ECE0183599F4F0E94B8
:10637000241E4091EB02FF24F3944F2564E070E06B
:10638000C8010E94C9B483E495E00E94341E409184
:10639000EB024F256CE070E08CE79BE00E94C9B4F3
:1063A0004091EB024F2564E170E0C8010E94C9B43E
:1063B000F090EB02F11038C089809A80AB80BC80ED
:1063C000A5019401C501B4010E94FCEA81112CC011
:1063D0008092051390920613A0920713B0920813AF
:1063E0002CEA35EC47E25EE36D817E818F819885F2
:1063F0000E946AE26093091370930A1380930B134F
:1064000090930C132CEA35EC47E25EE369857A85BC
:106410008B859C850E947EE960930D1370930E130B
:1064200080930F1390931013C8010E942C1EC80173
:106430000E94141EF11038C089809A80AB80BC8005
:10644000A5019401C501B4010E94FCEA81112CC090
:106450008092700B9092710BA092720BB092730BA2
:106460002CEA35EC47E25EE36D817E818F81988571
:106470000E946AE26093740B7093750B8093760BA5
:106480009093770B2CEA35EC47E25EE369857A85D9
:106490008B859C850E947EE96093780B7093790BC5
:1064A00080937A0B90937B0BC8010E94141EC80145
:1064B0000E94241EC8010E942C1EF11004C0898174
:1064C0009A810E94216B85E0F80111928A95E9F783
:1064D0004091EB02FF24F3944F2565E070E0C80182
:1064E0000E94C9B4C8010E94341E4091EB024F259E
:1064F00060E270E0C8010E94C9B4CE0183599F4F89
:106500000E94341E4091EB024F2569E070E0C80103
:106510000E94C9B44091EB0241110FC08981809360
:1065200076028A819B81AC81BD81809372029093B7
:106530007302A0937402B0937502FF24F3944F2565
:1065400060E270E0C8010E94C9B44091EB024F259F
:1065500060E470E0C8010E94C9B44091EB024F258D
:1065600060E170E0C8010E94C9B44091EB024F2580
:1065700060E170E0C8010E94C9B4C8010E941C1EFD
:106580004091EB024F256CE070E0C8010E94C9B455
:106590004091EB024F256CE670E0C8010E94C9B43F
:1065A00019821A821B821C821D821E821F821886FB
:1065B00019861A861B861C86C8010E94141E4091EB
:1065C000EB024F2568E070E0C8010E94C9B4409119
:1065D000EB024F256CE070E0C8010E94C9B4CE0107
:1065E00081589F4F0E94241ECE0183599F4F0E94C5
:1065F0001C1E8091C80B9091C90B8134934069F4A3
:106600001092AD042091111330911213EF968EADBC
:106610009FADEF972817390719F081E08093AD04FB
:106620008091EB02811111CD8091AD0481110DCDCE
:106630000E94312F0ACDC8010E943C1ECE01835911
:106640009F4F0E943C1EC158DF4FE880CF57D0407B
:10665000C058DF4F8881C058D040E89E7001112497
:1066600081E0E81AF10808F47CCECE018B589F4FE8
:106670000E941C1EF5CF84E690E09093C90B809396
:10668000C80B10921213109211130C94EA2F8091E0
:106690004105811105C08091B00B882309F461C0C8
:1066A00080918D04329B57C0816080938D048091CE
:1066B0008D04339B52C0826080938D0480918D0441
:1066C000349B4DC0846080938D0480911E0580FFB3
:1066D00010C08091420580FF0CC080918D0480FF26
:1066E00008C08091660B81608093660B80E00E94F9
:1066F0009BCC80911E05869580FF11C0809142053C
:10670000869580FF0CC080918D0481FF08C0809128
:10671000660B82608093660B81E00E949BCC809127
:106720001E058695869580FF1CC080914205869542
:10673000869580FF16C08091B00B882391F08091E0
:106740008D0482FF0EC08091660B84608093660B7F
:1067500082E00C949BCC8E7FA8CF8D7FADCF8B7FBA
:10676000B2CF0895CF93DF9300D000D0CDB7DEB77E
:1067700084EF91E0A0E0B0E089839A83AB83BC838F
:10678000BE016F5F7F4F8CE30E94FD748FE698E03F
:106790000E94F37686B169E678E082FB882780F96B
:1067A0000E94382086B163E678E083FB882780F971
:1067B0000E94382086B16DE578E0829581700E9454
:1067C0003820349909C00E9437750F900F900F90B0
:1067D0000F90DF91CF9108950E941C750F900F903C
:1067E0000F900F90DF91CF91089580914105811115
:1067F00004C08091B00B882331F062E070E080E04B
:1068000090E00C94BF730895CF93DF93CDB7DEB7BC
:106810002C970FB6F894DEBF0FBECDBFA7ECB1E149
:1068200090E080E0FC01EA5CF34F45915591659161
:1068300074914D935D936D937D93FC01EA5DF34FED
:10684000459155916591749150964D935D936D93DB
:106850007C935397FC01EA5EF34F45915591659106
:10686000749190964D935D936D937C93939704965A
:1068700080319105B9F680E29EE4A0E0B0E080931B
:10688000D7119093D811A093D911B093DA1180E069
:1068900090E8ABE3B4E48093FB119093FC11A093D8
:1068A000FD11B093FE1180E090E0AAE7B4E480937C
:1068B000FF1190930012A0930112B093021280E096
:1068C00090E0A6E9B3E48093031290930412A0939E
:1068D0000512B0930612109207121092081210922D
:1068E000091210920A1210920B1210920C121092AE
:1068F0000D1210920E1280E090E0A0E2B1E48093BD
:10690000DA0B9093DB0BA093DC0BB093DD0B80E0F4
:1069100090E0A0EAB0E48093DE0B9093DF0BA093AD
:10692000E00BB093E10B4AE959E969E97EE3409352
:10693000E20B5093E30B6093E40B7093E50B8093B1
:10694000E60B9093E70BA093E80BB093E90B109242
:106950004D0510924E0510924F0510925005109261
:10696000490510924A0510924B0510924C05109261
:1069700045051092460510924705109248050E9461
:1069800001738CE0E6E7F1E0DE01119601900D92D3
:106990008A95E1F789819A81AB81BC8180933B1311
:1069A00090933C13A0933D13B0933E138D819E8131
:1069B000AF81B88580933F1390934013A093411308
:1069C000B093421389859A85AB85BC858093431328
:1069D00090934413A0934513B093461384EB90E037
:1069E00090937D0B80937C0B86E490E090937F0BDB
:1069F00080937E0B1092810B1092800B80EF90E0C1
:106A00009093830B8093820B8EE690E09093850B9E
:106A10008093840B1092870B1092860B86E696E685
:106A2000A6E8B1E48093051390930613A09307138F
:106A3000B09308138CE993E5A9E4BEE380930913AE
:106A400090930A13A0930B13B0930C1380EE95EB65
:106A5000A5EAB3E480930D1390930E13A0930F1344
:106A6000B093101383EC95E9ACE2B4E48093700B1F
:106A70009093710BA093720BB093730B80E29BE128
:106A8000A2E9B1E48093740B9093750BA093760BFD
:106A9000B093770B87EF9CEDABECB5E48093780B6C
:106AA0009093790BA0937A0BB0937B0B83EC90E0DF
:106AB0000E94216B1092760280E090E0A0EEBFE38E
:106AC0008093720290937302A0937402B093750244
:106AD00010924105109240050E94F5332C960FB696
:106AE000F894DEBF0FBECDBFDF91CF910C94312F54
:106AF0000C9404343F924F925F926F927F928F92E8
:106B00009F92AF92BF92CF92DF92EF92FF920F933C
:106B10001F93CF93DF9300D000D0CDB7DEB7382ED0
:106B200080E090E0A0E2B1E489839A83AB83BC83E8
:106B3000C0904313D0904413E0904513F090461357
:106B400020E030E0A901C701B6010E9404E287FFFE
:106B50000CC0A701960160E070E080E291E40E9421
:106B6000FAE869837A838B839C8360E0CE01019687
:106B70000E94162E4090CA0B5090CB0B6090CC0B0D
:106B80007090CD0B8090CE0B9090CF0BA090D00B3F
:106B9000B090D10B332089F10E94447D19821A8272
:106BA0001B821C82E090D20BF090D30B0091D40B8F
:106BB0001091D50BCE0101966C01A5019401C30182
:106BC000B2010E94192D3092B00B0E94F5330F9044
:106BD0000F900F900F90DF91CF911F910F91FF9029
:106BE000EF90DF90CF90BF90AF909F908F907F906D
:106BF0006F905F904F903F9008950E94017DCECF9F
:106C00002F923F924F925F926F927F928F929F92BC
:106C1000AF92BF92DF92EF92FF920F931F93CF93A9
:106C2000DF93CDB7DEB764970FB6F894DEBF0FBE23
:106C3000CDBFD82E282E312CF101E850F84DF4901C
:106C400082E0D81234C08091B00B811103C081E082
:106C50000E947A350E94447D81115AC18AE199E0EF
:106C60000E94D16E20E030E0A9010E9404E2882356
:106C7000F1F06F2DFF0C770B880B990B0E940BE244
:106C80002B013C018AE199E00E94D16E4B015C012D
:106C900020E030E040EA50E40E9404E287FF1BC09D
:106CA000812C912C90EAA92E90E4B92E14C06F2D5E
:106CB000FF0C770B880B990B0E940BE22B013C0118
:106CC000C101880F991F880F991F8E5E964F0E94F1
:106CD000D16E4B015C01A3019201C501B4010E9478
:106CE0006AE24B015C017101EE0CFF1CEE0CFF1C13
:106CF000C7018A5F964F0E94D16E20E030E040ECE1
:106D00005FE30E946AE2A30192010E946AE2AB0182
:106D1000BC0100E010E098018D2D0E94D6B792E0F2
:106D2000D91230C10E94017D20E030E0A901C501E7
:106D3000B4010E9404E200E010E020E431E481119B
:106D400018C08091AF0B84608093AF0B8091A0043A
:106D500084608093A004C7018650974F0E94D16E33
:106D60006093D20B7093D30B8093D40B9093D50B7D
:106D70003DC0B501A40170588D2D0E94D6B7E2E048
:106D8000DE1609F4C0C0A5019401C501B4010E943A
:106D9000FBE8698B7A8B8B8B9C8BF2E0DF12D0C087
:106DA00000E010E020EC30E449895A896B897C8945
:106DB0008D2D0E94D6B782E0D812F0C00E94017DCE
:106DC0008091AF0B84608093AF0B8091A0048460AE
:106DD0008093A004C7018650974F0E94D16EF7019F
:106DE000E653F44F6083718382839383209143132E
:106DF0003091441340914513509146136091D20B4A
:106E00007091D30B8091D40B9091D50B0E94FAE82E
:106E10006093D20B7093D30B8093D40B9093D50BCC
:106E2000F701EF59FD4F10821182128213828D2DCE
:106E30000E9446290E94EE2EF701E653F44F80810E
:106E40009181A281B381F701EF5AFD4F8083918335
:106E5000A283B38392E0D91609F48FC08CE0E2E8F4
:106E6000F1E0DE01119601900D928A95E1F7E1E0E3
:106E7000F0E0EC0FFD1FEE0DFF1D80809180A280E1
:106E8000B38020E030E0A901C501B4010E9404E212
:106E90008823F1F120E030E0A901C501B4010E948E
:106EA0007EEA87FF04C0B7FAB094B7F8B094F70150
:106EB000E653F44F7F01A5019401C301B2010E9482
:106EC0006AE29B01AC01F70160817181828193814B
:106ED0000E94FAE8F7016083718382839383F2E072
:106EE00080E090E0A0E4B1E4DF1621F080E090E0E3
:106EF000A8E4B2E48D879E87AF87B88BCE010D964C
:106F00000E94AB1E05C00E94447D882309F43BCF3C
:106F100064960FB6F894DEBF0FBECDBFDF91CF9160
:106F20001F910F91FF90EF90DF90BF90AF909F90D7
:106F30008F907F906F905F904F903F902F9008952B
:106F4000F101E950F74F6491611107C00E94BB7CC9
:106F500085ED98E00E94F3766AE070E090E080E0D2
:106F60000E9409E29B01AC0160E070E088E492E4D9
:106F70000E947EE98B019C0117CF0E94D76E811180
:106F8000C7CF6CCF20E030E0A901C501B4010E9459
:106F900004E200E010E098018111EBCE81E090E086
:106FA000A0E0B0E00D2C04C0880F991FAA1FBB1FE2
:106FB0000A94D2F72091AF0B282B2093AF0B20918E
:106FC000A004822B8093A004C7018650974F0E9493
:106FD000D16EF701E653F44F60837183828393830C
:106FE0001FCF8091660B882319F01092660B0895CD
:106FF00040E070E060E08DE398E00E948D7D0F93AB
:107000001F938091BB0B813019F50E949CBD0091AC
:10701000890410918A0420918B0430918C04601BA8
:10702000710B820B930B28EE33E040E050E00E949E
:107030004CE860918504709186048091870490915A
:107040008804620F731F841F951F1F910F9108956D
:1070500060914C0270914D0280914E0290914F02CE
:10706000D6CF1092BB0B1092890410928A04109212
:107070008B0410928C0410924C0210924D021092CC
:107080004E0210924F0210928504109286041092C4
:1070900087041092880408958091BB0B8130F1F031
:1070A0008230C9F40E94FF37609385047093860490
:1070B000809387049093880481E08093BB0B0E94A7
:1070C0009CBD6093890470938A0480938B04909391
:1070D0008C0481E008950E943138EECF80E008955D
:1070E0000E9464B561E083E293E00E9401770C9412
:1070F0004C388091BB0B8150823070F41092BB0BE6
:107100000E949CBD60934C0270934D0280934E028E
:1071100090934F0281E0089580E00895CF93DF932C
:10712000EC010E94E11D20E040E070E060E0CE0153
:10713000DF91CF910C94C61E2F923F924F925F9297
:107140006F927F928F929F92AF92BF92CF92DF9277
:10715000EF92FF920F931F93CF93DF9300D000D055
:1071600000D0CDB7DEB71C017A8369832B833C83C3
:107170004D835E832701380181E08093970B0E9445
:10718000E11D83E08093670130927C0420927B04B0
:1071900089819A8190937A04809379048B819C8170
:1071A000AD81BE818093750490937604A09377049B
:1071B000B093780440927104509272046092730408
:1071C00070927404F12CE12CC0929A0BD0929B0B1C
:1071D000E0929C0BF0929D0BB0925F13A0925E1315
:1071E0009092700480926F048B8D80936E0426962B
:1071F0000FB6F894DEBF0FBECDBFDF91CF911F91C8
:107200000F91FF90EF90DF90CF90BF90AF909F9045
:107210008F907F906F905F904F903F902F90089548
:107220002F923F924F925F926F927F928F929F9296
:10723000AF92BF92CF92DF92EF92FF920F931F9384
:10724000CF93DF93CDB7DEB729970FB6F894DEBFA3
:107250000FBECDBF1C017987688769011A83098336
:10726000EB82BA01550F880B990B0E940BE220E0CC
:1072700030E0A9010E94FBE84B015C0120E030E016
:1072800040E05FEC0E947EEA18162CF0812C912CD5
:10729000A12C2FECB22EC501B4010E94F0E92B0104
:1072A0003C01B601DD0C880B990B0E940BE220E03B
:1072B00030E0A9010E94FBE84B015C0120E030E0D6
:1072C00040E05FE40E9404E287FD05C0812C912C20
:1072D000A12C9FE4B92EE885F98560817181072E84
:1072E000000C880B990B0E940BE220E030E0A90112
:1072F0000E94FBE86B017C01C301B2010E940BE21A
:107300009B01AC01C701B6010E94FAE80E94F7E9AF
:107310006C837D838E839F83C501B4010E94F0E955
:107320007B018C01E418F50806091709FB81FF931E
:1073300089809A8087E3A82E84E5B82ECC80DD80F2
:10734000A301920168857985C1010E949C380F9044
:1073500029960FB6F894DEBF0FBECDBFDF91CF9157
:107360001F910F91FF90EF90DF90CF90BF90AF9063
:107370009F908F907F906F905F904F903F902F9055
:10738000089520E040E070E060E085E791E60C942D
:10739000C61E1092020C0E947DC50C94C139E0916A
:1073A0007E04EE2389F0E150E0937E0488E0E89FBC
:1073B000F0011124E25CFB4F6281738127814681D9
:1073C000808191810C94C61E0C94C1398F929F923A
:1073D000AF92BF92CF92DF92EF92FF920F931F93E3
:1073E000CF93DF930E9414BAC091950B85E0982E3D
:1073F0009C0ED6E0DC1B85E0F82EFC1A84E0D82E2B
:10740000DC1A83E0C82ECC1A82E0B82EBC1A81E0C8
:10741000A82EAC1A8C2E8194C11159C08091980B62
:107420008823D1F180916701882359F081E0909100
:10743000980B911180E024E048E358E0682D0E9409
:10744000F8B88091020C80938E0BC43009F0E5C02F
:107450001092AC0B8091980B843009F4C9C08091D4
:107460006701882391F011E08091980B843009F036
:1074700010E080918E0B0E94251900E09C014DE1E7
:1074800058E06D2D812F0E94066DCF5FC911C4CFCA
:1074900087E08093960B0EC08091920B1092920B16
:1074A000882309F4BFCF0E94CF398091970B88239E
:1074B00009F4B8CFDF91CF911F910F91FF90EF901A
:1074C000DF90CF90BF90AF909F908F900895C13084
:1074D000C9F58091980B8130E9F08091670188238C
:1074E000A1F011E08091980B813009F010E08091BB
:1074F0001601909117010E94F01800E09C0142E3F0
:1075000058E06A2D812F0E94066D8091020C8093B5
:107510008E0BBBCF8091920B1092920B8823E9F2D5
:10752000E12C10E000E027EE33E04AE050E066E1B5
:1075300071E082E398E00E9410398091970B8823D4
:1075400061F2B8CFC23009F0C5C08091980B82308B
:10755000C9F0809167018823C1F211E08091980BF6
:10756000823009F010E080910213909103130E9481
:10757000F01800E09C014BE258E06B2D812F0E9437
:10758000066D5FCF8091920B1092920B882309F3C6
:107590000E946DB9E12C0FE61EE123EB31E050E0D3
:1075A00040E062E073E18BE298E00E941039809144
:1075B000970B882371F27ECF8091920B1092920BE1
:1075C000882309F48FC00E946DB9E12C0BE11EEBFA
:1075D0002CE830E050E040E06DE67BE087E298E0A8
:1075E0000E9410398091970B882309F47BC062CFE9
:1075F0008091920B1092920B882309F430CF0E9455
:107600006DB963E779E18DE198E00E94D7BB809185
:10761000970B882309F423CF4DCFC53099F580917E
:10762000980B8530B9F080916701882309F42DCF3C
:1076300011E08091980B853009F010E080912401D1
:10764000909125010E94F01800E09C0148E158E06B
:107650006F2D18CF8091920B1092920B882319F303
:10766000E12C00E519E127EE33E04AE050E064E266
:1076700071E088E198E00E9410398091970B88238F
:1076800091F218CFC63009F000CF8091980B863068
:1076900091F080916701882309F4F7CE81E0909101
:1076A000980B963009F080E023E049E058E06D2F18
:1076B0000E94F8B8EACE8091920B1092920B882328
:1076C00041F38AED92E50E948E388091970B8823D2
:1076D00001F3F0CEC33009F0B4CE8091980B833023
:1076E00009F46ACF80916701882309F40ECF11E075
:1076F0008091980B833009F010E080916D0B909190
:107700006E0B0E94F01800E09C0147E258E06C2DDF
:1077100035CF3F924F925F926F927F928F929F925E
:10772000AF92BF92CF92DF92EF92FF920F931F938F
:10773000CF93DF93D1E08091021390910313892BB3
:1077400009F4D0E00E9414BAC091950B5C2E45E07C
:10775000642E6C0E83E0F82EFC1A82E0982E9C1AA0
:1077600081E0882E8C1A4C2E419459ECC52E59E399
:10777000D52E6CEDA62E67E0B62E86E0782E7C1A0C
:10778000C11194C08091980B882309F46FC0809137
:107790006701882359F081E09091980B911180E066
:1077A00024E044E058E0642D0E94F8B810E000E0C6
:1077B00034E0E32E3C2E351800938E0BCE111FC003
:1077C000F801EE0FFF1FE852F84F859194919093C6
:1077D000AE0B8093AD0B8091980B8C1709F416C1FA
:1077E00080916701882359F081E09091980B9E1158
:1077F00080E023E045EE57E0632D0E94F8B88E2D1F
:107800000F5F1F4F95E0E92E8530B1F680916D0B2B
:1078100090916E0B892B19F4DD2309F417C1C63042
:10782000E9F48091980B863009F401C180916701D9
:107830008823A1F0DF92CF92BF92AF927F9281E036
:107840009091980B963009F080E08F930E944D2024
:107850000F900F900F900F900F900F9087E0D1E056
:10786000CF5FC6118DCF8093960B0EC08091920B87
:107870001092920B882309F48ACF0E94CF3980910D
:10788000970B882309F483CFDF91CF911F910F913C
:10789000FF90EF90DF90CF90BF90AF909F908F9030
:1078A0007F906F905F904F903F900895C13009F0A6
:1078B00060C08091980B813009F43FC080916701CE
:1078C000882309F473CF11E08091980B813009F07F
:1078D00010E080910213909103130E94F01800E0D1
:1078E0009C014DEF57E0682D812F0E94066D80911D
:1078F000020C80938E0BC33009F058CF1092AC0B62
:107900008091980B833009F46CC0809167018823C3
:1079100009F44CCF11E08091980B833009F010E00E
:1079200080918E0B0E94251900E09C014FEE57E0DC
:107930006F2D812F0E94066D39CF8091920B10928E
:10794000920B882309F4BACF0E946DB9E12C01E7AC
:107950001EE123EB31E050E040E062E073E18DEFA7
:1079600097E00E9410398091970B882309F4A6CFE5
:107970008BCFC23009F0BBCF8091980B8230B9F029
:1079800080916701882309F411CF11E08091980B51
:10799000823009F010E080916D0B90916E0B0E9487
:1079A000F01800E09C0149EF57E0692D9DCF8091D0
:1079B000920B1092920B882319F30E946DB9E12C5F
:1079C0000BE11EEB2CE830E050E040E06DE67BE0A0
:1079D00089EF97E00E9410398091970B882381F2FC
:1079E00053CF8091920B1092920B882309F48DCF84
:1079F0000E946DB963E779E18FEE97E00E94D7BBF3
:107A00008091970B882309F480CF3ECF8091920B11
:107A10001092920B882309F4E3CE88E29DE30E9442
:107A20008E388091970B882309F4DACE2DCF809180
:107A3000920B1092920B882309F4F8CE0E94C93958
:107A40008091970B882309F4F1CE1ECF86E008CFF2
:107A50004F925F926F927F928F929F92AF92BF925E
:107A6000CF92DF92EF92FF920F931F93CF93DF930A
:107A700000918E0B0E9414BAC091950B10E0000F7C
:107A8000111F0852184F95E0592E5C0E2EEBE22E76
:107A900027E0F22ED3E0DC1B3BE5C32E30E2D32EF1
:107AA00040EBA42E47E0B42E82E0782E7C1A55EEEF
:107AB000852E57E0952E81E0682E6C1A4C2E41944D
:107AC000C11137C08091980B8823B1F08091670174
:107AD000882359F081E09091980B911180E024E087
:107AE0004CEC57E0642D0E94F8B8CF5F5C12E8CFF1
:107AF00084E08093960B0CC08091920B1092920BB5
:107B0000882321F30E94CF398091970B8823F1F2CB
:107B1000DF91CF911F910F91FF90EF90DF90CF9069
:107B2000BF90AF909F908F907F906F905F904F909D
:107B30000895C13059F5F801859194919093AE0B59
:107B40008093AD0B8091980B813081F0809167011B
:107B5000882359F21F929F928F926F9281E09091A9
:107B6000980B913009F474C080E072C08091920B40
:107B70001092920B882351F380918E0B682F0E94F4
:107B800048BE8091970B882309F3C2CFC23009F019
:107B900042C0F801859194919093AE0B8093AD0B08
:107BA0008091980B8230D1F080916701882309F48D
:107BB0009CCFDF92CF92BF92AF927F9281E0909163
:107BC000980B923009F080E08F930E944D200F9027
:107BD0000F900F900F900F900F9087CF8091920B86
:107BE0001092920B882301F30E945B208091970BE7
:107BF0008823D1F28DCF8091920B1092920B882323
:107C0000C1F060918E0B8FEF0E9448BE8091970B60
:107C1000882379F07DCFC33009F067CFF8018591D3
:107C200094919093AE0B8093AD0B8091980B833021
:107C300011F380916701882309F457CF1F92FF92B7
:107C4000EF92DF9381E09091980B933009F08CCF05
:107C50008F930E944D200F900F900F900F900F90D8
:107C600044CF2F923F924F925F926F927F928F926A
:107C70009F92AF92BF92CF92DF92EF92FF920F93BB
:107C80001F93CF93DF930E9414BAC091950B6C2E73
:107C900085E0582E5C0E98E9C92E97E0D92E23E096
:107CA000E22E4E2C4C1A7724739437EAA32E37E039
:107CB000B32E12E01C1B372C3C1A2C2E219446E7C5
:107CC000842E47E0942E84E0F82EFC1AC1117CC06B
:107CD0008091980B882309F456C08091670188230E
:107CE00059F081E09091980B911180E024E04BEAEB
:107CF00057E0622D0E94F8B88091A0048770873009
:107D000009F0BAC020E030E0A9016091E30270916F
:107D1000E4028091E5029091E6020E9404E2882349
:107D200009F4AAC0D5E0C43009F0A7C0D09171020F
:107D30008091980B843079F48091920B1092920B81
:107D4000882349F0D725E09267010E940E1E80919A
:107D5000970B811126C080916701882391F081E003
:107D60009091980B943009F080E02EE737E0D11124
:107D700002C02AE737E001E041E857E06F2D0E949A
:107D8000066DD5E08EC08091920B1092920B8823E5
:107D900009F4A3CF0E94CF398091970B882309F46F
:107DA0009CCFDF91CF911F910F91FF90EF90DF90CB
:107DB000CF90BF90AF909F908F907F906F905F908B
:107DC0004F903F902F900895C13019F58091980BF6
:107DD000813081F080916701882309F48DCF81E0A3
:107DE0009091980B913009F080E023E040ED57E24C
:107DF000632D80CF8091920B1092920B882351F3C8
:107E00008DE79FE30E948E388091970B882311F3B2
:107E1000C8CFC23009F05BC09091980B923071F0DE
:107E200080916701882309F467CF81E0923009F0DF
:107E300080E020E24DE957E0612F5CCF8091920B0A
:107E40001092920B882361F3B0925205A0925105D3
:107E50008091970B882321F3A4CF8091920B1092ED
:107E6000920B8823E1F1D0925205C0925105809186
:107E7000970B8823A1F195CFD4E0DC1312C0909129
:107E8000980B9D17A9F080916701882351F06C2F02
:107E9000661981E09C1380E020E245E657E00E94ED
:107EA000F8B8CF5FC51112CFDF5FD093960B79CFB3
:107EB0008091920B1092920B882329F39092520595
:107EC000809251058091970B8823E9F26ACFC330E5
:107ED00009F012CF9091980B933009F4BECF8091A6
:107EE0006701882309F408CF81E0933009F080E02E
:107EF00020E24EE857E0642DFDCEDF92EF92FF9234
:107F00000F931F93CF93DF930E9414BAC091950BE8
:107F100085E0E82EEC0ED4E0DC1B13E01C1B02E035
:107F20000C1B81E0F82EFC1ADC2ED194C1112EC05E
:107F30008091980B8823B1F080916701882359F0D4
:107F400081E09091980B911180E024E04EE557E09C
:107F50006D2D0E94F8B8CF5FCE11E8CF85E08093F9
:107F6000960B0CC08091920B1092920B882321F3F8
:107F70000E94CF398091970B8823F1F2DF91CF9146
:107F80001F910F91FF90EF90DF900895C13011F590
:107F90008091980B813079F0809167018823D9F224
:107FA00081E09091980B913009F080E023E041EF5F
:107FB00057E26F2DCECF8091920B1092920B8823B7
:107FC00059F38AE690E20E948E388091970B8823BD
:107FD00019F3D4CFC23009F055C08091980B82308C
:107FE00081F080916701882309F4B5CF81E09091F9
:107FF000980B923009F080E023E04AEE57E2602FC0
:10800000A8CF8091920B1092920B882351F385E6B2
:1080100090E20E948E388091970B882311F3AECFA7
:108020008091980B833081F080916701882309F457
:1080300092CF81E09091980B933009F080E023E09B
:1080400043EE57E2612F85CF8091920B1092920BF5
:10805000882351F380E690E20E948E388091970B3E
:10806000882311F38BCF8091920B1092920B88236F
:1080700091F08FE49FE10E948E388091970B8823C6
:1080800051F07CCFC33061F2C43009F064CF8091ED
:10809000980B843041F380916701882309F45BCF0A
:1080A00081E09091980B943009F080E023E04AED54
:1080B00057E26D2F4ECF0C94CF392F923F924F92B3
:1080C0005F926F927F928F929F92AF92BF92CF9268
:1080D000DF92EF92FF921F93CF93DF93CDB7DEB77E
:1080E0002C970FB6F894DEBF0FBECDBF1C01162F24
:1080F0008091920B1092920B8823E1F01092940BD6
:108100000E94CF392C960FB6F894DEBF0FBECDBFBC
:10811000DF91CF911F91FF90EF90DF90CF90BF90B4
:10812000AF909F908F907F906F905F904F903F9017
:108130002F90089580919A0B90919B0BA0919C0B8E
:10814000B0919D0B8D839E83AF83B887892B8A2B3B
:108150008B2B09F460C080912601882309F4BDC0EF
:10816000809127018111B9C0613009F494C0623057
:1081700009F4A2C08090280190902901A0902A01C2
:10818000B0902B01C0903401D0903501E0903601C1
:10819000F0903701612E712C6D817E818F819885E1
:1081A0000E940BE2209112013091130140911401C1
:1081B000509115010E946AE2D301AA0FBB1FAA0FBA
:1081C000BB1FBC87AB87A653B44FBA87A9872D9135
:1081D0003D914D915C910E94FBE82B013C018D810A
:1081E0009E81AF81B885B7FF8FC0A5019401C301FF
:1081F000B2010E9404E287FD7FC0EB85FC85E65357
:10820000F44F4082518262827382812F0E94E71F65
:1082100081E08093670110929A0B10929B0B109251
:108220009C0B10929D0B80916701882309F46ACF03
:10823000F4E01F9FC0011124FC01E653F44F845465
:10824000944FDC012D913D914D915C916081718144
:10825000828193810E94FBE86B017C01C982DA82F2
:10826000EB82FC822DEC3CEC4CEC5DE36091120166
:108270007091130180911401909115010E947EEA82
:1082800087FD52C0CE0101960E94BB16BC01C10100
:108290000E94876C37CF80902C0190902D01A09088
:1082A0002E01B0902F01C0903801D0903901E0909C
:1082B0003A01F0903B016ECF8090300190903101F7
:1082C000A0903201B0903301C0903C01D0903D01AC
:1082D000E0903E01F0903F015DCF812C30E5932E80
:1082E00033ECA32E37ECB32EC12C40E5D42E43EC57
:1082F000E42E47E4F42E4ECFA985BA858D929D9247
:10830000AD92BC92139781CFA7019601C301B20130
:108310000E947EEA18160CF070CFE985FA85C082BB
:10832000D182E282F38271CF20E030E040E251E47A
:10833000C701B6010E946AE220E030E04AE754E457
:108340000E946AE24B015C0120E030E0A901C70114
:10835000B6010E9404E220E030E040EA50E487FFEA
:1083600004C020E030E040EA50ECC501B4010E94B6
:10837000FBE820E030E040E251E40E947EE90E9408
:10838000F0E96B017C01F7FC62C020EA36E841E0CD
:1083900050E00E946EE8CA01B9012AE030E040E0F6
:1083A00050E00E946EE8605D60939E0BC701B601CD
:1083B00020E137E240E050E00E946EE88AE0882E3B
:1083C000912CA12CB12CCA01B901A50194010E94E4
:1083D0006EE8605D60939F0BC701B60128EE33E045
:1083E00040E050E00E946EE8CA01B901A501940185
:1083F0000E946EE8605D6093A00B8EE28093A10BFB
:10840000C701B60124E630E040E050E00E946EE88B
:10841000CA01B901A50194010E946EE8605D6093F4
:10842000A20BC701B601A50194010E946EE8162FA8
:10843000CA01B901A50194010E946EE8605D6093D4
:10844000A30B105D1093A40B8EE99BE01FCFF0945B
:10845000E094D094C094C11CD11CE11CF11C6DE2CD
:10846000A3CF62E083EE97E20C945D4061E08AEE78
:1084700097E20C945D4060E081EF97E20C945D40E0
:10848000CF93DF9300D000D0CDB7DEB78091920BB1
:108490001092920B882359F01092940B0E94CF39BE
:1084A0000F900F900F900F90DF91CF9108956091F2
:1084B0009A0B70919B0B80919C0B90919D0B611579
:1084C00071058105910561F10E940BE22091120175
:1084D0003091130140911401509115010E946AE2FC
:1084E0002091D60B3091D70B4091D80B5091D90BDE
:1084F0000E94FBE86093D60B7093D70B8093D80B48
:108500009093D90B83E00E94E71F81E0809367017D
:1085100010929A0B10929B0B10929C0B10929D0B39
:1085200080916701882309F4BBCF2091880B30919B
:10853000890B40918A0B50918B0B6091D60B7091F7
:10854000D70B8091D80B9091D90B0E94FAE86983E0
:108550007A838B839C83CE0101960E94BB16BC015B
:108560008AED97E20E94876C9BCF3F924F925F9279
:108570006F927F928F929F92AF92BF92CF92DF9233
:10858000EF92FF920F931F93CF93DF930E9414BA41
:10859000C091950B3C2E85E0482E4C0E94E7C92ED9
:1085A00096E0D92E0EE816E0D4E0DC1B23E4A22EE0
:1085B00026E0B22E3DE9E32E36E0F32E83E0782E5E
:1085C0007C1A44E1842E46E0942E82E0682E6C1AD8
:1085D00081E0582E5C1AC11139C08091980B882314
:1085E000B9F080916701882361F0632D619581E086
:1085F0009091980B911180E024E04EEB56E00E94A0
:10860000F8B8CF5FC411E7CF85E08093960B0CC01C
:108610008091920B1092920B882319F30E94CF390C
:108620008091970B8823E9F2DF91CF911F910F91F1
:10863000FF90EF90DF90CF90BF90AF909F908F9082
:108640007F906F905F904F903F900895C13041F5BB
:108650008091980B813089F080916701882389F29D
:108660001F9288EB96E09F938F935F9281E09091A9
:10867000980B913061F180E02AC08091920B1092AA
:10868000920B882349F386EB95E0909352058093F3
:1086900051050E94C1398091970B8823E9F2C4CF1C
:1086A000C23009F064C08091980B8230C9F080918B
:1086B0006701882309F4A5CF1F928FEA96E09F9364
:1086C0008F936F9281E09091980B9230A1F68F93E7
:1086D0000E944D200F900F900F900F900F9091CF10
:1086E0008091920B1092920B882309F3909252057D
:1086F000809251050E94C1398091970B8823B9F26D
:1087000093CF8091980B833081F08091670188230B
:1087100009F477CF1F92FF92EF927F9281E09091C0
:10872000980B933009F0A7CFD2CF8091920B109283
:10873000920B882351F3B0925205A09251050E94EA
:10874000C1398091970B882301F36ECF8091920BF2
:108750001092920B8823A1F0D0925205C09251053D
:108760000E94C1398091970B882351F05DCFC330AF
:1087700041F2C43009F045CF8091980B843031F339
:1087800080916701882309F43CCF1F921F930F93B8
:10879000DF9381E09091980B943009F06CCF97CFE4
:1087A0007F928F929F92AF92BF92CF92DF92EF9281
:1087B000FF920F931F93CF93DF930E94D11D182F29
:1087C0000E9414BAC091950B0C2F85E0782E7C0E78
:1087D00085E0F82EFC1A86E0E82EEC1A84E0D82E0C
:1087E000DC1A83E0C82ECC1A82E0982E9C1A9AE7F5
:1087F000A92E94E0B92E81E0882E8C1AC1114AC0AE
:108800008091980B882361F180916701882361F042
:10881000602F619581E09091980B911180E024E0A8
:1088200049EE54E00E94F8B8111193C1C53009F027
:1088300022C18091980B853009F4BBC080916701FB
:10884000882361F081E09091980B953009F080E0E9
:1088500023E04FEA54E06F2D0E94F8B8D7E07AC1C8
:108860008091920B1092920B882371F20E94CF3963
:108870008091970B882341F2DF91CF911F910F9147
:10888000FF90EF90DF90CF90BF90AF909F908F9030
:108890007F900895C13079F58091980B8130D1F0A7
:1088A00080916701882309F4BFCF1F9288ED94E07F
:1088B0009F938F938F9281E09091980B913009F064
:1088C00080E08F930E944D200F900F900F900F909B
:1088D0000F90AACF8091920B1092920B882301F3F4
:1088E000B0925205A09251050E94C1398091970B18
:1088F0008823B1F2C1CFC23009F00EC18091980B2C
:108900008230A1F080916701882361F081E090912D
:10891000980B923009F080E023E04FEC54E0692D91
:108920000E94F8B8112309F499CF13C18091920BDA
:108930001092920B882331F385EF96E40E948E38D3
:108940008091970B8823F1F297CF8091980B833019
:1089500081F080916701882309F4F8C081E090914B
:10896000980B933009F080E023E042EC54E06C2D4A
:10897000D7CF8091920B1092920B882351F385EC04
:1089800098E40E948E388091970B882311F374CF5E
:108990008091920B1092920B882309F4C8C082EC4C
:1089A0009BE40E948E388091970B882309F4BFC006
:1089B00063CF8091920B1092920B882309F43ECFE3
:1089C00088EA9DE40E948E388091970B882309F4F1
:1089D00035CF52CF8091920B1092920B882309F4DD
:1089E00052C08BE29FE40E948E388091970B8823BF
:1089F00009F449C041CF8091920B1092920B8823C9
:108A000009F4AFC08AE590E50E948E388091970BFB
:108A1000882309F4A6C030CF8091920B1092920B5C
:108A2000882309F44BC08EED91E50E948E38809129
:108A3000970B882309F442C01FCF8091920B1092AC
:108A4000920B882309F453C00E94E11D20E040E00E
:108A500070E060E086EA90E2DF91CF911F910F9184
:108A6000FF90EF90DF90CF90BF90AF909F908F904E
:108A70007F900C94C61EC63009F0F0CE8091980B02
:108A8000863009F4A7CF80916701882309F4E6CEE8
:108A900081E09091980B963009F080E023E046EA5F
:108AA00054E06E2D0E94F8B8D7E081E08D0F8C1352
:108AB00015C08091980B8C1709F4AECF8091670197
:108AC000882361F06C2F601B81E09091980B9C13C0
:108AD00080E023E041E954E00E94F8B882E08D0F85
:108AE0008C1313C09091980B9C1709F4A6CF80911A
:108AF0006701882351F06C2F601B81E09C1380E09C
:108B000023E04FE754E00E94F8B8CF5FC71176CE5C
:108B1000DD5FD093960BB0CEC33009F416CFC430CE
:108B200009F082CE8091980B843009F431CF809186
:108B30006701882359F081E09091980B943009F0F7
:108B400080E023E04DEB54E06D2DEACE112309F4D3
:108B500092CFD5E0DC13A9CF8091980B8D1709F443
:108B60004ACF80916701882309F49FCF6C2F601B47
:108B700081E09091980B9C1380E023E04AE954E057
:108B80000E94F8B892CF6F927F928F929F92AF928D
:108B9000BF92CF92DF92EF92FF920F931F93CF93EA
:108BA000DF930E9414BAC091950B6C2E85E0782E4D
:108BB0007C0E92E5E92E95E7F92E23E0C22E25E002
:108BC000D22ED5E0DC1B3CE1A32E35E7B32E14E01A
:108BD0001C1B03E00C1B82E0982E9C1A81E0882E5F
:108BE0008C1AC11136C08091980B8823B9F08091FE
:108BF0006701882361F0662D619581E09091980B63
:108C0000911180E024E040E355E00E94F8B8CF5F86
:108C1000C711E7CF86E08093960B0CC08091920B32
:108C20001092920B882319F30E94CF398091970BF1
:108C30008823E9F2DF91CF911F910F91FF90EF9080
:108C4000DF90CF90BF90AF909F908F907F906F906C
:108C50000895C13029F58091980B8130A1F0809161
:108C600067018823A1F28DE695E79F938F9385E1B5
:108C700095E09F938F938F9281E09091980B913024
:108C800049F180E027C08091920B1092920B8823CB
:108C900031F30E946D758091970B882301F3CACF41
:108CA000C23009F085C08091980B8230E9F0809144
:108CB0006701882309F4ABCF8DE190E29F938F93F6
:108CC0008BE095E09F938F939F9281E09091980B1A
:108CD0009230B9F68F930E944D200F900F900F9015
:108CE0000F900F900F9093CF8091920B1092920B58
:108CF0008823E9F20E941D208091970B8823B9F206
:108D000099CF8091980B8330A9F0809167018823D7
:108D100009F47DCF87E395E79F938F938CEF94E0E1
:108D20009F938F930F9381E09091980B933009F06C
:108D3000A8CFD0CF8091920B1092920B882329F369
:108D40000E9437758091970B8823F9F273CF809139
:108D5000980B843099F080916701882309F457CFEC
:108D6000BF92AF9287EF94E09F938F931F9381E020
:108D70009091980B943009F084CFACCF8091920BF6
:108D80001092920B882339F30E941C758091970BE7
:108D9000882309F34FCF8091920B1092920B882376
:108DA00099F00E9452758091970B882369F042CF09
:108DB000C33009F4A6CFC43051F2C53009F027CF33
:108DC0008091980B853039F380916701882309F4ED
:108DD0001ECFFF92EF92DF92CF92DF9381E09091CE
:108DE000980B953009F04DCF75CF7F928F929F925F
:108DF000AF92BF92CF92DF92EF92FF920F931F93A9
:108E0000CF93DF930E9414BAC091950B65E0862E34
:108E10008C0ED6E0DC1B85E0D82EDC1A84E0C82E50
:108E2000CC1A83E0B82EBC1A82E0A82EAC1A81E0DE
:108E3000982E9C1A7C2E7194C11134C08091980B8D
:108E40008823B1F080916701882359F081E09091E7
:108E5000980B911180E024E04AE554E0672D0E94D0
:108E6000F8B8CF5FC811E8CF87E08093960B0CC0AD
:108E70008091920B1092920B882321F30E94CF399C
:108E80008091970B8823F1F2DF91CF911F910F9181
:108E9000FF90EF90DF90CF90BF90AF909F908F901A
:108EA0007F900895C130E9F58091980B8130E9F009
:108EB000809167018823A9F211E08091980B81309D
:108EC00009F010E06091EB117091EC118091ED11BF
:108ED0009091EE110E94D41B00E09C0145EA53E002
:108EE000692D812F0E94066DBCCF8091920B10924C
:108EF000920B8823E9F20E946DB9E12C1CE3F12E5C
:108F00000CE116E420E030E040E85FE36BEE71E155
:108F100085EA93E00E946ABA8091970B882341F218
:108F2000B3CFC23009F006C18091980B8230D9F0DE
:108F300080916701882309F494CF11E08091980B08
:108F4000823009F010E06091EF117091F011809182
:108F5000F1119091F2110E94D41B00E09C014EE9A6
:108F600053E06A2DBECF8091920B1092920B882312
:108F7000F9F20E946DB9E12C1CE3F12E0CE116E42C
:108F800020E030E040E85FE36FEE71E18EE993E0CE
:108F90000E946ABA8091970B882351F275CF809115
:108FA000980B8330D9F080916701882309F459CF59
:108FB00011E08091980B833009F010E06091F3117B
:108FC0007091F4118091F5119091F6110E94D41BCB
:108FD00000E09C0147E953E06B2D83CF8091920B19
:108FE0001092920B8823F9F20E946DB9E12C1CE3D8
:108FF000F12E0CE116E420E030E040E85FE363EF9F
:1090000071E187E993E00E946ABA8091970B882307
:1090100051F23ACF8091980B8430D9F0809167015A
:10902000882309F41ECF11E08091980B843009F059
:1090300010E06091F7117091F8118091F911909101
:10904000FA110E94D41B00E09C0140E953E06C2D12
:1090500048CF8091920B1092920B8823F9F20E94D4
:109060006DB9E12C1CE3F12E0CE116E420E030E0B8
:1090700040E85FE367EF71E180E993E00E946ABA3C
:109080008091970B882351F2FFCE8091980B853009
:10909000D9F080916701882309F4E3CE11E0809133
:1090A000980B853009F010E060910712709108125A
:1090B0008091091290910A120E94D41B00E09C0139
:1090C0004BE853E06D2D0DCF8091920B1092920BD7
:1090D0008823F9F20E946DB9E12C1CE3F12E0CE11A
:1090E00016E420E030E0A90167E072E18BE893E04C
:1090F0000E946ABA8091970B882359F2C5CE80915D
:10910000920B1092920B882329F10E946DB9E12CE9
:109110001CE3F12E0CE116E420E030E0A9016BE045
:1091200072E181E893E00E946ABA8091970B8823EC
:1091300089F0AACEC33009F432CFC43009F46ACF23
:10914000C53009F4A2CFC63009F08BCE8091980BC0
:109150008630A9F280916701882309F482CE11E05C
:109160008091980B863009F010E060910B1270919D
:109170000C1280910D1290910E120E94D41B00E0EF
:109180009C0141E853E06D2FACCE2F923F924F925D
:109190005F926F927F928F929F92AF92BF92CF9287
:1091A000DF92EF92FF920F931F93CF93DF93CDB790
:1091B000DEB72C970FB6F894DEBF0FBECDBFC090C0
:1091C000CB11D090CC11E090CD11F090CE118091C8
:1091D000CF119091D011A091D111B091D2118C15D5
:1091E0009D05AE05BF0510F4D701C601C090C7119B
:1091F000D090C811E090C911F090CA11BC01CD0106
:109200006C157D058E059F0510F4C701B6010E94FF
:1092100009E22B013C010E9414BA2091950B2B8787
:109220002E83822F8B5F8D8387E0922F821B8F830B
:1092300086E0821B888785E0821B898784E0821B09
:109240008A8783E0282E221A82E0382E321A9195DE
:109250009C872B85211142C08091980B8823C9F0EF
:1092600080916701882359F081E09091980B9111CA
:1092700080E024E04AE554E06C850E94F8B88B85D4
:109280008F5F8B879D819813E4CF88E08093960B46
:109290000CC08091920B1092920B882309F30E94CC
:1092A000CF398091970B8823D9F22C960FB6F8947A
:1092B000DEBF0FBECDBFDF91CF911F910F91FF9009
:1092C000EF90DF90CF90BF90AF909F908F907F9066
:1092D0006F905F904F903F902F9008958B858130D5
:1092E00009F08BC08091980B8130F9F08091670173
:1092F000882329F211E08091980B813009F010E069
:109300006091FB117091FC118091FD119091FE1103
:109310000E94D41B61E02E81621B00E09C014BED9A
:1093200053E0812F0E94066DAACF8091920B10927C
:10933000920B8823D9F20E946DB92AE037ED43E2FF
:109340005DE3C301B2010E946AE220E030E0A901BE
:109350000E94FBE84B015C0120E030E040E05FE46C
:109360000E9404E287FD05C0812C912CA12C3FE4D2
:10937000B32E2AE037ED43E25DE36091FB1170917B
:10938000FC118091FD119091FE110E946AE220E093
:1093900030E0A9010E94FBE820E030E040E85FE314
:1093A0000E94FAE80E94F7E969837A838B839C83A1
:1093B000C501B4010E94F0E97B018C0121E0E21AB1
:1093C000F108010911091F92912C812C25E2A22E8E
:1093D00024E5B22EC980DA8021E030E040E050E0A0
:1093E0006BEF71E18BED93E00E949C380F908091C0
:1093F000970B882309F47ACF58CF8B85823009F0F8
:1094000090C18091980B8230D9F0809167018823B8
:1094100009F435CF11E08091980B823009F010E00B
:109420006091FF11709100128091011290910212CF
:109430000E94D41B00E09C0141ED53E0632D71CFED
:109440008091920B1092920B8823F9F20E946DB9D1
:109450006091D3117091D4118091D5119091D61152
:109460000E9409E27B018C0120E030E048EC52E4EC
:109470006FEF71E181ED93E00E946ABA8091970BE2
:10948000882319F212CF8091980B8330D9F0809104
:109490006701882309F4F3CE11E08091980B8330A3
:1094A00009F010E06091031270910412809105128E
:1094B000909106120E94D41B00E09C0148EC53E0FE
:1094C000622D2FCF8091920B1092920B8823F9F28C
:1094D0000E946DB92AE037ED43E25DE3C301B201BA
:1094E0000E946AE220E030E0A9010E94FBE84B0103
:1094F0005C0120E030E040E05FE40E9404E287FD90
:1095000005C0812C912CA12C9FE4B92E2AE037EDC7
:1095100043E25DE3609103127091041280910512A1
:10952000909106120E946AE220E030E0A9010E94B8
:10953000FBE820E030E040E85FE30E94FAE80E94A8
:10954000F7E969837A838B839C83C501B4010E9408
:10955000F0E97B018C0121E0E21AF108010911090F
:109560001F92912C812C85E2A82E84E5B82EC9800B
:10957000DA8021E030E040E050E063E072E188EC26
:1095800093E00E949C380F908091970B882309F4F8
:109590007ECF8BCE8091980B8430E9F0809167016B
:1095A000882309F46CCE11E08091980B843009F087
:1095B00010E06091C7117091C8118091C91190910C
:1095C000CA110E9409E20E94BC1900E09C0141EC12
:1095D00053E06A85A6CE8091920B1092920B88235D
:1095E000E9F20E946DB90FE214E224E630E040E0B7
:1095F00050E067EC71E181EC93E00E9409BB80913F
:10960000970B882359F251CE8091980B8530E9F061
:1096100080916701882309F432CE11E08091980B84
:10962000853009F010E06091CB117091CC118091E0
:10963000CD119091CE110E9409E20E94BC1900E068
:109640009C014AEB53E069856CCE8091920B10929D
:10965000920B8823E9F20E946DB90DE214E224E630
:1096600030E040E050E06BEC71E18AEB93E00E9467
:1096700009BB8091970B882359F217CE8091980BE4
:109680008630E9F080916701882309F4F8CD11E074
:109690008091980B863009F010E06091CF117091A5
:1096A000D0118091D1119091D2110E9409E20E94B3
:1096B000BC1900E09C0143EB53E0688532CE8091F9
:1096C000920B1092920B8823E9F20E946DB90BE283
:1096D00014E22AE030E040E050E06FEC71E183EB0F
:1096E00093E00E9409BB8091970B882359F2DDCD4E
:1096F0008091920B1092920B882339F10E946DB9E0
:1097000009E214E224E630E040E050E063ED71E16C
:109710008CEA93E00E9409BB8091970B8823A9F003
:10972000C4CD2B85233009F4AECE243009F432CFDA
:10973000253009F469CF263009F4A0CF273009F08D
:109740009ECD8091980B873099F280916701882394
:1097500009F495CD11E08091980B873009F010E065
:109760006091D3117091D4118091D5119091D6113F
:109770000E9409E20E94BC1900E09C014CEA53E0FF
:109780006F81CFCD3F924F925F926F927F928F9277
:109790009F92AF92BF92CF92DF92EF92FF920F9380
:1097A0001F93CF93DF930E9414BAC091950BA5E04D
:1097B0004A2E4C0ED4E0DC1B83E0782E7C1A82E02B
:1097C000682E6C1A81E0582E5C1A3C2E3194C1111F
:1097D00038C08091980B8823B1F08091670188236D
:1097E00059F081E09091980B911180E024E04AE5D6
:1097F00054E0632D0E94F8B8CF5FC411E8CF85E034
:109800008093960B0CC08091920B1092920B882340
:1098100021F30E94CF398091970B8823F1F2DF91D9
:10982000CF911F910F91FF90EF90DF90CF90BF905D
:10983000AF909F908F907F906F905F904F903F90F0
:109840000895C13009F05DC08091980B8130E9F036
:1098500080916701882381F211E08091980B81301B
:1098600009F010E06091DA0B7091DB0B8091DC0B5A
:109870009091DD0B0E94071C00E09C0149EF53E032
:10988000652D812F0E94066DB7CF8091920B1092AB
:10989000920B8823E9F20E946DB920E030E0A90123
:1098A0006091DA0B7091DB0B8091DC0B9091DD0BFA
:1098B0000E94FBE820E030E040E85FE30E94FAE825
:1098C0000E94F7E91F92912C812CE9E1AE2EE4E58C
:1098D000BE2E6B011DEDE12E13E0F12E00E010E035
:1098E00021E030E040E050E06AED7BE089EF93E07A
:1098F0000E949C380F908091970B882309F4A8CF81
:109900008ECFC23009F0FEC08091980B8230D9F022
:1099100080916701882309F46FCF11E08091980B43
:10992000823009F010E06091DE0B7091DF0B8091C6
:10993000E00B9091E10B0E94071C00E09C0141EFBD
:1099400053E0662D9ECF8091920B1092920B88234C
:10995000F9F20E946DB920E030E0A9016091DE0BC0
:109960007091DF0B8091E00B9091E10B0E94FBE87E
:1099700020E030E040E85FE30E94FAE80E94F7E967
:109980001F92912C812C49E1A42E44E5B42E6B0149
:109990001DEDE12E13E0F12E00E010E021E030E0BB
:1099A00040E050E06EED7BE081EF93E00E949C3858
:1099B0000F908091970B882309F4AACF30CF809124
:1099C000980B8330D9F080916701882309F414CF74
:1099D00011E08091980B833009F010E06091E20B68
:1099E0007091E30B8091E40B9091E50B0E94D519E7
:1099F00000E09C0149EE53E0672D43CF8091920B2C
:109A00001092920B8823F9F20E946DB920E030E0A9
:109A100048EC52E46091E20B7091E30B8091E40B0F
:109A20009091E50B0E946AE220E030E0A9010E94DB
:109A3000FBE820E030E040E251E40E94FAE80E94B6
:109A4000F7E91F92912C812C23E1A22E24E5B22E5E
:109A50006B011EEAE12E12E8F12E01E010E02AE08F
:109A600030E040E050E062EE7BE089EE93E00E945F
:109A70009C380F908091970B882309F4A4CFCFCE08
:109A80008091920B1092920B882309F446C00E9499
:109A90006DB920E030E048EC52E46091E60B709143
:109AA000E70B8091E80B9091E90B0E946AE220E0BD
:109AB00030E0A9010E94FBE820E030E040E251E400
:109AC0000E94FAE80E94F7E91F92912C812C83E111
:109AD000A82E84E5B82E6B011EEAE12E12E8F12EC5
:109AE00001E010E02AE030E040E050E066EE7BE08C
:109AF00081EE93E00E949C380F908091970B882311
:109B000061F08DCEC33009F45ACFC43009F074CE61
:109B10008091980B843009F4B3CF8091670188233A
:109B200009F46ACE11E08091980B843009F010E0BE
:109B30006091E60B7091E70B8091E80B9091E90B37
:109B40000E94D51900E09C0141EE53E06D2F99CEA3
:109B50004F925F926F927F928F929F92AF92BF923D
:109B6000CF92DF92EF92FF920F931F93CF93DF93E9
:109B70000E9414BAC091950B65E0562E5C0ED3E09E
:109B8000DC1B82E0782E7C1A81E0682E6C1A4C2E49
:109B90004194C11137C08091980B8823B1F0809116
:109BA0006701882359F081E09091980B911180E032
:109BB00024E04AE554E0642D0E94F8B8CF5FC51157
:109BC000E8CF84E08093960B0CC08091920B1092AA
:109BD000920B882321F30E94CF398091970B882321
:109BE000F1F2DF91CF911F910F91FF90EF90DF90F5
:109BF000CF90BF90AF909F908F907F906F905F902D
:109C00004F900895C13009F061C08091980B813068
:109C1000E9F080916701882389F211E08091980B27
:109C2000813009F010E060913B1370913C138091FA
:109C30003D1390913E130E948B1A00E09C014FE16E
:109C400054E0662D812F0E94066DB8CF8091920B53
:109C50001092920B8823E9F220E030E040E251E4D8
:109C600060913B1370913C1380913D1390913E1392
:109C70000E946AE220E030E0A9010E94FBE820E0B7
:109C800030E84BEB54E40E94FBE80E94F7E91F9296
:109C9000912C812C4DE0A42E44E5B42E6B0118EBE1
:109CA000E12E1BE0F12E00E010E024E23AEF4FEF4E
:109CB0005FEF6BE373E18FE194E00E949C380F90BB
:109CC0008091970B882309F4A4CF8BCFC23009F081
:109CD0009FC08091980B8230D9F0809167018823D2
:109CE00009F46CCF11E08091980B823009F010E0FC
:109CF00060913F13709140138091411390914213F2
:109D00000E948B1A00E09C0140E154E0672D9ACF3D
:109D10008091920B1092920B8823F9F220E030E0B0
:109D200040E251E460913F137091401380914113E0
:109D3000909142130E946AE220E030E0A9010E9463
:109D4000FBE820E030E84BEB54E40E94FBE80E9483
:109D5000F7E91F92912C812C2DE0A22E24E5B22E42
:109D60006B0118EBE12E1BE0F12E00E010E024E285
:109D70003AEF4FEF5FEF6FE373E180E194E00E9411
:109D80009C380F908091970B882309F4A6CF29CF98
:109D90008091920B1092920B882309F441C020E02D
:109DA00030E04AE754E4609143137091441380918A
:109DB0004513909146130E946AE220E030E0A90129
:109DC0000E94FBE820E030EA4CE056E40E94FBE809
:109DD0000E94F7E91F92912C812C8DE3A82E84E537
:109DE000B82E6B0110E5E12E16E4F12E00E010E034
:109DF00028ED3CED4FEF5FEF63E473E181E094E029
:109E00000E949C380F908091970B882349F0E9CEEF
:109E1000C33009F0D3CE8091980B833009F4B8CFCA
:109E200080916701882309F4C9CE11E08091980BD5
:109E3000833009F010E060914313709144138091D6
:109E40004513909146130E94CC2000E09C0141E014
:109E500054E06D2FF7CEBF92CF92DF92EF92FF9238
:109E60000F931F93CF93DF930E9414BAC091950B69
:109E700085E0C82ECC0ED4E0DC1B13E01C1B82E076
:109E8000F82EFC1A81E0E82EEC1ABC2EB194C11118
:109E900030C08091980B8823B1F0809167018823AE
:109EA00059F081E09091980B911180E024E04AE50F
:109EB00054E06B2D0E94F8B8CF5FCC11E8CF85E05D
:109EC0008093960B0CC08091920B1092920B88237A
:109ED00021F30E94CF398091970B8823F1F2DF9113
:109EE000CF911F910F91FF90EF90DF90CF90BF9097
:109EF0000895C130B9F58091980B8130F1F08091CF
:109F000067018823C9F2DD24D3948091980B8130B6
:109F100009F0D12C6091DB117091DC118091DD1181
:109F20009091DE110E940C1B00E09C014FE454E074
:109F30006E2D8D2D0E94066DBFCF8091920B1092D9
:109F4000920B8823E1F20E946DB947E254E26BED77
:109F500071E18FE494E00E948BBB8091970B882382
:109F600071F2BDCFC23009F07FC08091980B823072
:109F7000E1F080916701882309F49ECFDD24D3941A
:109F80008091980B823009F0D12C6091DF11709193
:109F9000E0118091E1119091E2110E940C1B00E010
:109FA0009C0144E454E06F2DC4CF8091920B109239
:109FB000920B8823F1F20E946DB945E254E26FEDF5
:109FC00071E184E494E00E948BBB8091970B88231D
:109FD00081F285CF8091980B8330E1F08091670109
:109FE000882309F469CFDD24D3948091980B8330C2
:109FF00009F0D12C6091E3117091E4118091E51189
:10A000009091E6110E940C1B00E09C0149E354E092
:10A01000612F8FCF8091920B1092920B8823F1F2D7
:10A020000E946DB943E254E263EE71E189E394E08A
:10A030000E948BBB8091970B882381F250CF809137
:10A04000920B1092920B8823C9F00E946DB941E2E5
:10A0500054E267EE71E18EE294E00E948BBB809146
:10A06000970B882359F03BCFC33009F4B3CFC430EA
:10A0700009F022CF8091980B843009F38091670119
:10A08000882309F419CFDD24D3948091980B843070
:10A0900009F0D12C6091E7117091E8118091E911DC
:10A0A0009091EA110E940C1B00E09C014EE254E0EA
:10A0B0006D2F3FCF2F923F924F925F926F927F9280
:10A0C0008F929F92AF92BF92CF92DF92EF92FF92C8
:10A0D0000F931F93CF93DF9300D000D000D0CDB764
:10A0E000DEB70E9414BA7090950B7E8285E0870DD2
:10A0F0008D8384E0682E671823E0322E232C2718E6
:10A1000082E0582E571881E0482E4718711041C040
:10A110008091980B8823C1F080916701882361F0BA
:10A120006E81619581E09091980B911180E024E01F
:10A130004AE554E00E94F8B873948D817812E6CF16
:10A1400085E08093960B0CC08091920B1092920B3D
:10A15000882311F30E94CF398091970B8823E1F275
:10A1600026960FB6F894DEBF0FBECDBFDF91CF911C
:10A170001F910F91FF90EF90DF90CF90BF90AF9025
:10A180009F908F907F906F905F904F903F902F9017
:10A19000089581E078122DC09091980B9130B9F01C
:10A1A00080916701882341F281E0913009F080E0DD
:10A1B00090913D0525E733E0911102C021E733E09E
:10A1C00001E048E753E0642D0E94066DB5CF809111
:10A1D000920B1092920B882319F380913D058725ED
:10A1E00080933D05309267018091970B8823C1F2DF
:10A1F000B7CF82E07812A0C08091980B8230C1F076
:10A2000080916701882309F497CF11E08091980B22
:10A21000823009F010E080912201909123010E9488
:10A22000F01800E09C014AE653E0652D812FCCCF69
:10A230008091920B1092920B882311F3E12C10E085
:10A2400000E023EB31E050E040E062E271E08AE6BA
:10A2500093E00E9410398091970B882389F280CF78
:10A260008091980B8330B9F080916701882309F4BD
:10A2700063CF11E08091980B833009F010E080915A
:10A280002001909121010E94F01800E09C0143E61A
:10A2900053E0622DCBCF8091920B1092920B8823CA
:10A2A00019F3E12C10E000E023EB31E050E040E056
:10A2B00060E271E083E693E00E9410398091970B91
:10A2C000882391F24DCF8091920B1092920B8823AC
:10A2D00009F43EC020E030E048EC52E460911C01FB
:10A2E00070911D0180911E0190911F010E946AE2F0
:10A2F00020E030E0A9010E94FBE80E94F7E91F92EC
:10A30000912C812C81E3A82E84E5B82E6B0118EEE8
:10A31000E12E13E0F12E00E010E020E030E0A90192
:10A320006CE171E08BE593E00E949C380F90809186
:10A33000970B882369F014CF83E0781609F490CF47
:10A3400084E07812F9CE8091980B843009F4BBCF69
:10A3500080916701882309F4EFCE11E08091980B7A
:10A36000843009F010E0C0901C01D0901D01E090F5
:10A370001E01F0901F0120E030E0A901C701B601E5
:10A380000E9404E22DEB37E346E055EB87FD04C065
:10A390002DEB37E346E055E3C701B6010E94FBE829
:10A3A00069837A838B839C83CE0101960E94371741
:10A3B00000E09C014BE553E0662D38CF4F925F9251
:10A3C0006F927F928F929F92AF92BF92CF92DF92C5
:10A3D000EF92FF920F931F93CF93DF930E9414BAD3
:10A3E000C091950B35E0632E6C0E43E0542ED1E006
:10A3F000DC1B4C2E419482E0782E7C1AC1113FC0A8
:10A400008091980B8823F1F080916701882359F09F
:10A4100081E09091980B911180E024E04AE554E0AE
:10A42000642D0E94F8B880917602882309F4C0C098
:10A43000C23009F457C083E0CF5FC611DFCF8093ED
:10A44000960B0CC08091920B1092920B8823E1F234
:10A450000E94CF398091970B8823B1F2DF91CF9181
:10A460001F910F91FF90EF90DF90CF90BF90AF9032
:10A470009F908F907F906F905F904F900895C13024
:10A4800091F68091980B8130C9F080916701882303
:10A4900051F281E09091980B913009F080E0909119
:10A4A000760225E733E0911102C021E733E001E0B5
:10A4B00041E553E06D2F0E94066DB5CF8091760285
:10A4C0009091920B1092920B9923F9F28C27809322
:10A4D0007602509267010E94D1158091970B8823D4
:10A4E000A1F2BCCF8091980B8230F1F0809167018E
:10A4F000882309F4A0CF11E08091980B823009F0F5
:10A5000010E06091720270917302809174029091D8
:10A5100075020E94CC2000E09C0147E453E0672DC7
:10A52000812F0E94066D87CF8091920B1092920B23
:10A530008823E1F20E946DB920E030E04AE754E45C
:10A540006091720270917302809174029091750211
:10A550000E946AE220E030E0A9010E94FBE820E0CE
:10A5600030E84BEB54E40E94FAE80E94F7E91F92AE
:10A5700081ED882E85E1982E9DE3A92E94E5B92ED4
:10A580006B0116EDE12E16E0F12E00E010E02CED4F
:10A5900035E040E050E062E772E087E493E00E943B
:10A5A0009C380F908091970B882309F49FCF56CF4A
:10A5B00082E042CFCF92DF92EF92FF92CF93DF9370
:10A5C0008091920B1092920B882351F01092940B71
:10A5D000DF91CF91FF90EF90DF90CF900C94CF3927
:10A5E00081E08093940B80919A0B90919B0BA091AA
:10A5F0009C0BB0919D0B0097A105B10509F44BC0D0
:10A600002AE0289FE001299FD00D112410929A0B77
:10A6100010929B0B10929C0B10929D0BBE010D2E65
:10A62000000C880B990B0E940BE220910B0C3091CF
:10A630000C0C40910D0C50910E0C0E946AE220917E
:10A6400043133091441340914513509146130E9497
:10A65000FBE86B017C0120E030E040E151EC0E941E
:10A660007EEA87FD18C020E030E040E151E4C701F8
:10A67000B6010E9404E2181674F0CE010E94D5BD06
:10A68000C0924313D0924413E0924513F0924613C4
:10A6900082E08093670180916701882379F083E4E9
:10A6A00093E10E9479B9BC0188E393E0DF91CF91F7
:10A6B000FF90EF90DF90CF900C94876CDF91CF915B
:10A6C000FF90EF90DF90CF9008950F931F93CF935B
:10A6D000DF93FC01EB0180919A0B90919B0BA09171
:10A6E0009C0BB0919D0BB7FF08C010929A0B109273
:10A6F0009B0B10929C0B10929D0B8091710490917A
:10A700007204A0917304B091740440919A0B50911B
:10A710009B0B60919C0B70919D0B84179507A6076E
:10A72000B70744F480939A0B90939B0BA0939C0BD8
:10A73000B0939D0B809167018823E1F060919A0BA3
:10A7400070919B0B80919C0B90919D0B00917504D7
:10A75000109176042091770430917804600F711F76
:10A76000821F931F0995BC0180917B0490917C040A
:10A770000E94876C8091920B811108C080916E04B9
:10A780008823D1F1809167018823B1F18091790408
:10A7900090917A040097B1F040919A0B50919B0BE5
:10A7A00060919C0B70919D0B009175041091760443
:10A7B0002091770430917804400F511F621F731F5E
:10A7C000FE010995E0916F04F0917004309741F01B
:10A7D00080916E04811103C08091920B81110995C3
:10A7E0008091920B1092920B882331F0DF91CF91E0
:10A7F0001F910F910C94CF39DF91CF911F910F9141
:10A8000008956CE779E185E999E10C94655368E571
:10A810007CE181E79CE10C9465536FE37CE180E887
:10A820009CE10C94655368EA7CE181EC9CE10C941A
:10A83000655363EE7CE186EF9CE10C9465536FEF0A
:10A840007CE18AE19DE10C94655369E27DE182E45B
:10A850009DE10C94655360ED7CE181E59DE10C94F4
:10A8600065536FE87CE18AE59DE10C94655369E9E5
:10A870007DE18CEA9DE10C94655368EB7DE18FEFFF
:10A8800090E20C946553CF93DF93CDB7DEB78D8103
:10A8900090915002891768F0809350029E01285FC2
:10A8A0003F4F4E815F816AE270E080E292E00E9459
:10A8B000CBE1DF91CF9108950F931F93CF93DF9357
:10A8C0008C016F3F19F41092500260E02091500209
:10A8D000862F062E000C990B2817190609F04CF547
:10A8E0006093500260E08CEC92E00E940177C80116
:10A8F0000E94F3768AE00E944776C8010E9451E1E7
:10A90000800F911FEC01C01BD10BCB32D1053CF065
:10A910000197FC012491207C2038D1F3F3CFDD276F
:10A92000AE01B80180E292E00E9472E1C05EDD4FAC
:10A930001882DF91CF911F910F910895DF92EF92CE
:10A94000FF920F931F93CF93DF93CDB7DEB7C65817
:10A95000D1090FB6F894DEBF0FBECDBFC358DF4F8D
:10A96000188219821A821B82CD57D040809105022D
:10A9700090910602A0910702B0910802CF57DF4FD5
:10A9800088839983AA83BB83C158D04084E690E032
:10A990009093C90B8093C80B10921213109211134D
:10A9A0001092AD0464E070E0CE018F579F4F0E947B
:10A9B00034BD8091C80B9091C90B02969093C90B3E
:10A9C0008093C80B109212131092111381E0CA5792
:10A9D000DF4F8883C658D040CE018A579F4F0E94D0
:10A9E000671E68E470E087EC91E10E9434BD60E18D
:10A9F00070E08AED9BE00E9434BD8AE097EDA3EA07
:10AA0000BCE3C358DF4F88839983AA83BB83CD57A8
:10AA1000D040CE0183589F4F0E945F1E85E495E091
:10AA20000E946B1E7E018DE6E80EF11C8FEFD701B0
:10AA30008C93C7010E94671E19821A821B821C8296
:10AA40008E010F5F1F4FC8010E945F1E19821A827C
:10AA50001B821C82C8010E945F1EC358DF4F1882F0
:10AA600019821A821B82CD57D04083E0F701808380
:10AA70008983CE0183589F4F0E945F1EC7010E94A9
:10AA8000671EC8010E94671E4AE0D42EDA94DD20BA
:10AA900031F0CE0183589F4F0E945F1EF7CF8BE3AA
:10AAA00093E10E946B1EC358DF4F188219821A82ED
:10AAB0001B82CD57D0403AE0D32EDA94DD2031F01E
:10AAC000CE0183589F4F0E945F1EF7CF85E0D82E9E
:10AAD000D982D701DC92C8010E94671EC7010E947B
:10AAE000671E68E070E083EE92E00E9434BD68E08B
:10AAF00070E08BED92E00E9434BD64E670E087E781
:10AB000092E00E9434BD19828FEFF7018083C80163
:10AB10000E94631EC7010E94671E64E070E08BED17
:10AB200091E00E9434BD809143058983C8010E9451
:10AB3000631E6CE070E08CE79BE00E9434BD198AD4
:10AB40001A8A1B8A1C8A80E090E0A0E8BFE38D8708
:10AB50009E87AF87B88B8091051390910613A091C3
:10AB60000713B091081389839A83AB83BC832CEAC3
:10AB700035EC47E25EE36091091370910A1380910E
:10AB80000B1390910C130E947EE96D837E838F835B
:10AB900098872CEA35EC47E25EE360910D137091E3
:10ABA0000E1380910F13909110130E946AE269872F
:10ABB0007A878B879C8764E170E0C8010E9434BD6E
:10ABC00084E190E09A838983C8010E94571E809196
:10ABD000700B9091710BA091720BB091730B8983E4
:10ABE0009A83AB83BC832CEA35EC47E25EE3609149
:10ABF000740B7091750B8091760B9091770B0E947E
:10AC00007EE96D837E838F8398872CEA35EC47E25B
:10AC10005EE36091780B7091790B80917A0B909143
:10AC20007B0B0E946AE269877A878B879C87C801C1
:10AC30000E945B1E8CE0EEE8F1E0D80101900D92DD
:10AC40008A95E1F7C8010E945B1E1982C8010E9423
:10AC5000671E80914001909141019A838983C801C8
:10AC60000E94571EEAE9F1E0D80101900D92DA94B2
:10AC7000E1F765E070E0C8010E9434BD1982C801A7
:10AC80000E94631E80E2EFE9F1E0D80101900D928D
:10AC90008A95E1F760E270E0C8010E9434BDD701F7
:10ACA0001C92C7010E94631E86E792E00E94631E09
:10ACB00082E792E00E945F1EC358DF4F188219821C
:10ACC0001A821B82CD57D040CE0183589F4F0E94DD
:10ACD0005F1E80E2F80111928A95E9F760E270E068
:10ACE000C8010E9434BDFE01F99688E0DF011D9283
:10ACF0008A95E9F744E650E060E070E049835A83C2
:10AD00006B837C834D835E836F83788783E090E0E1
:10AD1000A0E0B0E089879A87AB87BC874D875E87C4
:10AD20006F87788B498B5A8B6B8B7C8B8D8B9E8B33
:10AD3000AF8BB88F898F9A8FAB8FBC8F8D8F9E8F83
:10AD4000AF8FB8A38EE190E0A0E0B0E089A39AA312
:10AD5000ABA3BCA38DA39EA3AFA3B8A789A79AA7B3
:10AD6000ABA7BCA78DA79EA7AFA7B8AB89AB9AAB83
:10AD7000ABABBCAB8DAB9EABAFABB8AF60E470E040
:10AD8000C8010E9434BD90E1D92EF8018D2D119299
:10AD90008A95E9F760E170E0C8010E9434BDD801EE
:10ADA0001D92DA94E9F760E170E0C8010E9434BDB9
:10ADB000C358DF4F188219821A821B82CD57D040A8
:10ADC000CE0183589F4F0E945F1E2CE0D22EF801C7
:10ADD0008D2D11928A95E9F76CE070E0C8010E9410
:10ADE00034BD8CE6D8011D928A95E9F76CE670E0D7
:10ADF000C8010E9434BD81EA94E00E945B1EF70105
:10AE00001082118212821382148215821682178296
:10AE100068E070E0C7010E9434BDF7011192DA9436
:10AE2000E9F7CB57DF4F1882C558D04080E090E05B
:10AE3000A0E4B0E4ED968CAF9DAFAEAFBFAFED97A1
:10AE4000C7010E946B1ECE018B579F4F0E94671E49
:10AE5000CE0187589F4F0E945F1E8091AD048111E3
:10AE600024C00091C80B1091C90B809111139091CF
:10AE70001213D7018D939C9384E690E09093C90BB5
:10AE80008093C80B64E070E08FED91E00E9434BDC8
:10AE9000C7010E94571E91E00134134009F490E06D
:10AEA0008091AD04892B8093AD048091AD04811114
:10AEB00005C060E082EF9BE00E945C549091AD047D
:10AEC00081E08927CA57DF4F0FB6F894DEBF0FBE67
:10AED000CDBFDF91CF911F910F91FF90EF90DF9049
:10AEE000089581E08093EB020E943B331092EB02C5
:10AEF00081110C943B330E9404340E949E540E94A2
:10AF0000BB7C82E09CE00E94F37680E008950C9484
:10AF100071570C949E542F923F924F925F926F9272
:10AF20007F928F929F92AF92BF92CF92DF92EF92D9
:10AF3000FF920F931F93CF93DF9300D01F92CDB753
:10AF4000DEB70E94D11DF82E0E9414BA2091950BF5
:10AF50002A83722E2B5F298383E0382E371882E0F4
:10AF6000682E671881E0582E5718472C419499E8AD
:10AF7000C92E97E5D92E2DE5A22E25E0B22E38E771
:10AF8000832E35E3932E8A818111F8C08091980B2E
:10AF9000882309F4CFC080916701882359F081E0AC
:10AFA0009091980B911180E024E041EB55E0642DE5
:10AFB0000E94F8B8F11055C18A81833009F054C15C
:10AFC0008091980B833009F42CC180916701811125
:10AFD00039C194E09B83EB80E39410E000E02A8089
:10AFE00027189A819E1122C0F801EE0FFF1FE85228
:10AFF000F84F859194910093AC0B9093AE0B809396
:10B00000AD0B8091980B2A81821709F472C180914F
:10B010006701882359F081E09091980B9E1180E0A0
:10B0200023E04CE655E0622D0E94F8B8EB82E394F1
:10B030000130110509F05AC18A81E81220C08091BF
:10B04000980B9A81891709F465C18091670188235B
:10B05000B1F0DF92CF92BF92AF928A8187198F931E
:10B0600081E09091980B2A81921380E08F930E9447
:10B070004D200F900F900F900F900F900F908B819D
:10B080008E5FF1104EC09A81891323C08091980B76
:10B09000891709F44EC1809167018823D1F087E8B0
:10B0A00097E59F938F938FE495E09F938F938A8189
:10B0B00087198F9381E09091980B2A81921380E0F9
:10B0C0008F930E944D200F900F900F900F900F9034
:10B0D0000F908B818D5F9A81891321C08091980B8D
:10B0E000891709F435C1809167018823C1F09F92C7
:10B0F0008F928EE395E09F938F938A8187198F9328
:10B1000081E09091980B2A81921380E08F930E94A6
:10B110004D200F900F900F900F900F900F908B81FC
:10B120008C5F9A819F5F9A83298192132CCF8093A1
:10B13000960B0EC08091920B1092920B882309F40B
:10B140002ACF0E94CF398091970B882309F423CF0F
:10B150000F900F900F90DF91CF911F910F91FF9063
:10B16000EF90DF90CF90BF90AF909F908F907F90A7
:10B170006F905F904F903F902F9008959A819130FB
:10B1800049F58091980B8130B1F080916701882357
:10B1900009F410CF81E09091980B913009F080E094
:10B1A00023E04FE955E0652D0E94F8B8FF2009F42F
:10B1B0005BC023E054C08091920B1092920B8823C5
:10B1C00021F380ED93E40E948E388091970B8823C1
:10B1D000E1F2BECF2A81223009F0ECCE8091980BAB
:10B1E000823081F080916701882309F4C0C081E03A
:10B1F0009091980B923009F080E023E040E955E00F
:10B20000662DD6CE8091920B1092920B882351F32B
:10B210008AED92E50E948E388091970B882311F376
:10B2200097CF8091920B1092920B882309F4CDCE88
:10B2300083EC95E40E948E388091970B882309F463
:10B24000C4CE86CF81E09091980B933009F080E0D6
:10B2500023E048E855E0632D0E94F8B824E02B83F2
:10B26000BACE83E08B8302C094E09B832B818A81DA
:10B270002813B1CE8091980B8217E1F0809167017D
:10B28000882309F4A8CEEA80E71811E08091980B92
:10B290009A81891310E080914001909141010E94B0
:10B2A000F01800E09C014BE755E06E2D812F0E94C5
:10B2B000066D91CE8091920B1092920B8823F1F241
:10B2C000EE24E39408EA19E12FEF30E048E750E07C
:10B2D00060E471E08BE795E00E9410398091970B54
:10B2E000882361F235CF83E08B8375CE01E010E0D7
:10B2F00078CE8091920B1092920B882309F487CE1E
:10B300008BEB99E50E948E388091970B882309F486
:10B310007ECE1ECF8091920B1092920B882309F45F
:10B3200094CE0E949E548091970B882309F48DCE71
:10B330000FCF8091920B1092920B882309F4ABCE21
:10B340000E9471578091970B882309F4A4CE00CFF7
:10B350008091920B1092920B882309F4C4CE0E9424
:10B3600004348091970B882309F4BDCEF1CEF110FF
:10B37000BACF84E077CF2F923F924F925F926F9235
:10B380007F928F929F92AF92BF92CF92DF92EF9275
:10B39000FF920F931F93CF93DF93CDB7DEB729971B
:10B3A0000FB6F894DEBF0FBECDBF2091AC0B29873E
:10B3B0000E9414BA3091950B3887E9858E2F90E062
:10B3C000880F991F9C012852384F3B832A8336E00F
:10B3D000E39FC0011124FC01E258F44F1F019C01BE
:10B3E0002458344F69016884362D3B5F398311E05E
:10B3F000412E4618562C5194DD82CC82F6013496AB
:10B40000FF83EE8339E8A32E37E5B32E85E0F82ECF
:10B41000F618460122E0820E911C82E0782E761802
:10B42000388531115BC01123D9F08091980B181623
:10B43000BCF040919A0B50919B0B60919C0B7091CA
:10B440009D0B4F5F5F4F6F4F7F4F40939A0B509311
:10B450009B0B60939C0B70939D0B8F5F8093980B5D
:10B4600080916701882341F0EA81FB8165917491A5
:10B4700043E0852D0E949BB8EE81FF8180818093FF
:10B480008E0BF885F23009F07BC029852093AC0B38
:10B490008091980B823009F460C080916701882305
:10B4A00091F011E08091980B823009F010E08091CA
:10B4B0008E0B0E94251900E09C0146E255E0672DA5
:10B4C000812F0E94066D10E028852F5F2887398123
:10B4D0002313A6CF86E08093960B19C08885813010
:10B4E00059F68091980B813031F08091670181117C
:10B4F00027C010E0C1CF8091920B1092920B88234D
:10B50000A1F30E94CF398091970B882371F329967C
:10B510000FB6F894DEBF0FBECDBFDF91CF911F9164
:10B520000F91FF90EF90DF90CF90BF90AF909F90E2
:10B530008F907F906F905F904F903F902F900895E5
:10B5400081E09091980B913009F080E024E040E395
:10B5500055E0642D0E94F8B8CCCF8091920B1092E8
:10B56000920B882309F499CF6EEA79E186E295E09F
:10B570000E94D7BB8091970B882309F48ECFC7CF49
:10B580003885333099F58091980B8330C1F08091E4
:10B590006701882309F497CF11E08091980B8330DD
:10B5A00009F010E0EC81FD81808191810E94F0180A
:10B5B00063E0661900E09C014FE155E081CF809186
:10B5C000920B1092920B882311F3E12C10E000E013
:10B5D00023EB31E045E050E0B6018FE195E00E94B9
:10B5E00010398091970B882391F291CFF885F43030
:10B5F00091F58091980B8430B9F080916701882390
:10B6000009F461CF11E08091980B843009F010E0CB
:10B61000F401808191810E94F01864E0661900E0D5
:10B620009C014BE155E04CCF8091920B1092920B14
:10B63000882319F3E12C10E000E02CE830E045E02D
:10B6400050E0B1018BE195E00E9410398091970B99
:10B65000882399F25CCFF885F53009F035CF8091D9
:10B66000980B8530E1F080916701882309F42BCF96
:10B67000BF92AF928DE595E09F938F93FF9281E00B
:10B680009091980B953009F080E08F930E944D20A7
:10B690000F900F900F900F900F900F9014CF8091FC
:10B6A000920B1092920B8823F1F20E949E5480918B
:10B6B000970B8823C1F22BCF0E9404340E949E5422
:10B6C0000C94C139CF9380913604811109C088E16F
:10B6D00093E0909384048093830481E08093360404
:10B6E0000E94E11D20E040E070E060E08FEB90E21E
:10B6F0000E94C61EC1E0C093940B0E943124109298
:10B70000940B0E94CF39C093940B8091B10B81119F
:10B7100007C048E053E06FE073E084E00E9490B51A
:10B7200060E08FE798E20E945C5461E082E093E081
:10B73000CF910C9401772F923F924F925F926F922C
:10B740007F928F929F92AF92BF92CF92DF92EF92B1
:10B75000FF920F931F93CF93DF9300D000D01F92DF
:10B76000CDB7DEB72091BB0B2D830E9414BA809118
:10B77000950B8C83582E8B5F898359E1252E57E7D3
:10B78000352E00EF16E060E7E62E68E3F62E7BEF3D
:10B79000C72E76E0D72E81E0482E451883E0782E1C
:10B7A000751882E085198A83E2E6AE2EEBE5BE2E9F
:10B7B000F8E18F2EF7E09F2E952D91959B832C819C
:10B7C00021113EC08091980B8823B1F080916701D0
:10B7D000882359F081E09091980B911180E024E04A
:10B7E00043E357E06B810E94F8B88D81813009F006
:10B7F000ABC024E0622EDBC08091920B1092920BC2
:10B80000882321F30E94CF398091970B8823F1F28E
:10B810000F900F900F900F900F90DF91CF911F918D
:10B820000F91FF90EF90DF90CF90BF90AF909F90DF
:10B830008F907F906F905F904F903F902F900895E2
:10B840008D81813009F080C09C81913061F58091BB
:10B85000980B8130D9F0809167018823A1F0BF92C5
:10B86000AF929F928F924F9281E09091980B91307E
:10B8700009F080E08F930E944D200F900F900F9061
:10B880000F900F900F9094E0692EAAC08091920BB8
:10B890001092920B8823F9F20E94625B8091970BC1
:10B8A0008823C9F2B5CF2C81223031F58091980BD5
:10B8B000823099F080916701882361F081E0909156
:10B8C000980B923009F080E023E04DE057E06A8168
:10B8D0000E94F8B884E0682E9EC08091920B10926E
:10B8E000920B882339F38DE890E20E948E38809184
:10B8F000970B8823F9F28CCF8C81833009F079CFB4
:10B900008091980B833089F080916701882311F32F
:10B9100081E09091980B933009F080E023E048E0BB
:10B9200057E0672D0E94F8B8AECF8091920B10922D
:10B93000920B882349F386EE99E30E948E3880911A
:10B94000970B882309F364CF8091BB0B823009F0F9
:10B95000AFC09C8132E0632E913009F0ABC0809182
:10B96000980B813009F480C08091670181118BC0F0
:10B9700042E0642E81E0860D9C81891316C080917F
:10B98000980B891709F4C6C080916701882369F074
:10B990006C81651981E09091980B2C81921380E065
:10B9A00023E049EE56E00E94F8B8639463948C81DA
:10B9B000681216C08091980B861509F4BCC080915E
:10B9C0006701882369F06C81651981E09091980B7B
:10B9D0002C81921380E023E04DED56E00E94F8B8F0
:10B9E00081E0860D9C81891316C08091980B891780
:10B9F00009F4B2C080916701882369F06C816519F0
:10BA000081E09091980B2C81921380E023E04FEC21
:10BA100056E00E94F8B882E0860D9D819130D9F001
:10BA20002C81821316C08091980B821709F4A5C04F
:10BA300080916701882369F06C81651981E090919C
:10BA4000980B2C81921380E023E044E257E00E949F
:10BA5000F8B883E0860D9C819F5F9C8329819213B7
:10BA6000AECE8093960BD4CE8091920B1092920B17
:10BA7000882309F479CF0E9470388091970B88232E
:10BA800009F472CFC5CEFF92EF92DF92CF924F9220
:10BA900081E09091980B913009F080E08F930E94A3
:10BAA0004D200F900F900F900F900F900F9060CF40
:10BAB000662463942C8162125DCF8091980B861569
:10BAC000E1F080916701882309F454CF3F922F92CF
:10BAD0001F930F938C8185198F9381E09091980B20
:10BAE0002C81921380E08F930E944D200F900F9035
:10BAF0000F900F900F900F903DCF8091920B10926E
:10BB0000920B8823F1F20E9419778091970B88237A
:10BB1000C1F27ECE8091920B1092920B882309F491
:10BB200033CF81E39EE30E948E388091970B882368
:10BB300009F42ACF6DCE8091920B1092920B88233C
:10BB400009F43DCF89E89BE30E948E388091970BE2
:10BB5000882309F434CF5CCE8091920B1092920B23
:10BB6000882309F447CF8BE897E50E948E388091AF
:10BB7000970B882309F43ECF4BCE8091920B109205
:10BB8000920B882309F454CF85EB92E40E948E38FF
:10BB90008091970B882309F44BCF3ACE61E08AED70
:10BBA00092E00E9401770E9479388091B10B811157
:10BBB00007C04FEE52E067EF72E085E00E9490B55B
:10BBC00060E081EE92E00E945C540C94C1390F93C6
:10BBD0001F930E949CBD0091320410913304209168
:10BBE000340430913504601B710B820B930B97FD6D
:10BBF0000CC089B183FB882780F991E089274A9B93
:10BC00008260309B84608093310480913104817024
:10BC10009091310491FD826090913004981749F021
:10BC2000813009F148F0823079F0833091F08093CF
:10BC300030041F910F910895913079F09230B9F747
:10BC400090912F0491500CC0992339F09330C1F397
:10BC5000EECF9130A9F3923051F790912F049F5F6E
:10BC600090932F04E4CF992359F3933001F7F5CF44
:10BC70004F925F926F927F928F929F92AF92BF92FC
:10BC8000CF92DF92EF92FF920F931F93CF93DF93A8
:10BC900000D000D0CDB7DEB70E949CBD4B015C0147
:10BCA000809110018F3FF1F10E949CBDC0901F0454
:10BCB000D0902004E0902104F09022046C197D09BA
:10BCC0008E099F0997FD2EC080914C1390914D13C2
:10BCD0008F5F8F70891731F1E0911001E43008F027
:10BCE000E2C024E0E29FF0011124E953FE4F80817D
:10BCF0009181A281B38189839A83AB83BC83C12C58
:10BD0000D12C76018E010F5F1F4F26ED3BE042EDF7
:10BD10005BE06EEC7BE08AEC9BE00E9421B48FEF4D
:10BD2000809310010E94E75D8091310482FFC4C0BE
:10BD300080912E0481111DC091E090932E0480917A
:10BD40001F0289278093920B10921F0283E0809339
:10BD50006701109231040E949CBD6C507E4F8F4F42
:10BD60009F4F609332047093330480933404909314
:10BD7000350480912A0490912B04A0912C04B09159
:10BD80002D04A5019401281B390B4A0B5B0BDA012A
:10BD9000C901B7FF05C080917D04882309F4D4C18F
:10BDA000D501C4018C599F4FAF4FBF4F80932A04D8
:10BDB00090932B04A0932C04B0932D0460912F0436
:10BDC000062E000C770B77FF03C071956195710902
:10BDD00090912F0480912904981371C0633008F06A
:10BDE0006EC010922F0480912F0480932904653037
:10BDF00008F077C08091920B8111F5C080915E139D
:10BE000090915F138557914641F4809111018823E9
:10BE100009F4FBC08150809311010E944C27C0900F
:10BE2000FE0BD090FF0BE090000CF090010C811104
:10BE30000E94A273D701C6013AE0B695A7959795DF
:10BE400087953A95D1F7009741E0A407B10520F016
:10BE50008FEF9FEFA0E0B0E0969587952091670166
:10BE60002111E5C030917D0431119CC180915E1398
:10BE700090915F138557914609F47BC18091940B93
:10BE8000811177C18091250490912604A091270407
:10BE9000B0912804881A990AAA0ABB0AB7FC77C18C
:10BEA0000E94C13974C18091680190916901A0918B
:10BEB0006A01B0916B011FCF10922E045ACF8DEF03
:10BEC000860F823008F08FCF80912F0491E087FD9C
:10BED0009FEF892F880F880F890F80932F0465E0CB
:10BEE00082CF8091AA0B21E030E040E050E088232F
:10BEF00009F456C0C090A60BD090A70BE090A80BF9
:10BF0000F090A90BC114D104E104F104E9F170E04F
:10BF100090E080E00E9409E220E030E040EA50E456
:10BF20000E947EE92B013C01C501B4016C197D0919
:10BF30008E099F090E9409E29B01AC01C301B20175
:10BF40000E947EE920E030E04AE754E40E946AE281
:10BF50006B017C0120E030E042E053E40E947EEA85
:10BF600024E630E040E050E087FF12C020E030E0FF
:10BF700040EA52E4C701B6010E947EEA2AE030E0BE
:10BF800040E050E087FF04C021E030E040E050E0B6
:10BF90008092A60B9092A70BA092A80BB092A90B2F
:10BFA000A0912F040A2E000CBB0B0E9498E825E0FC
:10BFB00030E040E050E00E946EE880919A0B909152
:10BFC0009B0BA0919C0BB0919D0B820F931FA41F04
:10BFD000B51F80939A0B90939B0BA0939C0BB093EF
:10BFE0009D0B10922F04D501C4018856954CAF4F7C
:10BFF000BF4F8093250490932604A0932704B09309
:10C00000280481E080936701F9CE8CE080931101D0
:10C010008091230490912404009729F00197909334
:10C0200024048093230481E080936701F6CE009777
:10C0300041F040912304509124044817590708F017
:10C0400015CF80917D0481111DC0223038F024303D
:10C0500008F44CC0243011F41092670180919D13B4
:10C06000811105C081E080939D130E943ABF8091A9
:10C070006613909167130E9413BF81E08093990B20
:10C0800080937D0483E00E94106B81E08093841391
:10C09000E0915E13F0915F1309951092990B8091D6
:10C0A0007D04811127C01092920B80915E139091B4
:10C0B0005F138557914609F0E1CE0E949CBDDC01DB
:10C0C000CB0188199909AA09BB09C0902304D09013
:10C0D0002404F12CE12CC816D906EA06FB0608F068
:10C0E000C5CE9093240480932304C0CE81E0809336
:10C0F0006701B4CF84E693E10E9475C291E081119B
:10C1000001C090E090937D04882369F280915E13D2
:10C1100090915F1385579146B9F40E949CBDDC0154
:10C12000CB0188199909AA09BB09C0902304D090B2
:10C130002404F12CE12CC816D906EA06FB0620F4EB
:10C1400090932404809323040F900F900F900F90EE
:10C15000DF91CF911F910F91FF90EF90DF90CF90E3
:10C16000BF90AF909F908F907F906F905F904F9017
:10C17000089548E9840E4AE3941EA11CB11C8092E4
:10C18000250490922604A0922704B092280480915E
:10C190007D048111D9CF809167018130A9F6109279
:10C1A0006701D2CF009709F46DCF43CFCF93809131
:10C1B000F00381114EC010929B1310929C131092A9
:10C1C0009D13109269131092681310926B131092C2
:10C1D0006A1310926D1381E080936C1382E2809356
:10C1E0006E131092731310927213E7E8F3E18FEF5E
:10C1F000819393E1E539F907D9F7C1E0C09384133E
:10C200002FE633EA30937A1320937913C0937B138C
:10C2100010927C1310927D1390E490937E131092F1
:10C220007F132DE433EA309396132093951328E07F
:10C2300031E030936713209366139CE19093891348
:10C240009EE190938813809387130E943ABFC09316
:10C25000F00380914001909141010E94216B81E0A7
:10C2600080931E0289E192E09093F9128093F81274
:10C270001092FB121092FA1253985B9A52985A9AA3
:10C280003898409A0E94E75D10922F04CF9108954C
:10C29000FC01A081B1811C92A281B3818C918F5F3E
:10C2A0008C930280F381E02D90818CE0989F800D2B
:10C2B0001124E0E6F3E113AE84AF0895FC0180E0C1
:10C2C0009491992331F0907C903809F08F5F3196EA
:10C2D000F7CF0895FC0180E09191992329F0907C9B
:10C2E0009038D1F38F5FF8CF08954F925F926F929D
:10C2F0007F928F929F92AF92BF92CF92DF92EF92F6
:10C30000FF920F931F93CF93DF9300D000D01F9223
:10C31000CDB7DEB71092AA0B8091920B1092920BC0
:10C320008823E9F020E040E070E060E08BE99BE5E5
:10C330000F900F900F900F900F90DF91CF911F9162
:10C340000F91FF90EF90DF90CF90BF90AF909F90B4
:10C350008F907F906F905F904F900C94C61E2091AD
:10C3600016013091170140919A0B50919B0BCA0115
:10C37000820F931F2436310509F0CEC34730510593
:10C3800044F006978A3091050CF0D5C38AE090E01E
:10C39000DCC306964A3F5F4FACF38091990B88232C
:10C3A00009F494C12091BC0B3091BD0B4091BE0BA0
:10C3B0005091BF0B6091CA0B7091CB0B8091CC0B4D
:10C3C0009091CD0B0E94FBE84B015C012091C00BCA
:10C3D0003091C10B4091C20B5091C30B6091CE0BB9
:10C3E0007091CF0B8091D00B9091D10B0E94FBE804
:10C3F00069837A838B839C832091C40B3091C50B16
:10C400004091C60B5091C70B6091D20B7091D30B2A
:10C410008091D40B9091D50B0E94FBE82B013C013D
:10C4200020E030E040E251E40E946AE220E030E0A7
:10C4300048EC52E40E946AE26B017C0120E030E0AB
:10C44000A901C301B2010E9404E220E030E040EA09
:10C4500050EC87FD04C020E030E040EA50E4C70122
:10C46000B6010E94FBE820E030E040E251E40E9487
:10C470007EE90E94F0E92B013C0180E277FE09C0D1
:10C480007094609450944094411C511C611C711C28
:10C490008DE280939E0B60E2F0E14F16F7E25F06BB
:10C4A000610471048CF0C301B20120E137E240E085
:10C4B00050E00E946EE8CA01B9012AE030E040E095
:10C4C00050E00E946EE8605D60939F0B60E228EE92
:10C4D000421623E05206610471048CF0C301B201DC
:10C4E00028EE33E040E050E00E946EE8CA01B90156
:10C4F0002AE030E040E050E00E946EE8605D60932A
:10C50000A00BC301B20124E630E040E050E00E94FD
:10C510006EE86AE0C62ED12CE12CF12CCA01B901DB
:10C52000A70196010E946EE8605D6093A10BC301B4
:10C53000B201A70196010E946EE86D83CA01B9019C
:10C54000A70196010E946EE8CD80CC2009F40DC3AE
:10C550008EE28093A20B605D6093A30B2C2D205D77
:10C560002093A40B6EE97BE087E194E00E9413EB3B
:10C5700020E030E0A901C501B4010E9404E220E0FE
:10C5800030E040E05FEB87FD04C020E030E040E0B9
:10C590005FE3C501B4010E94FBE80E94F0E9CB0112
:10C5A0000E947118BC0182E194E00E9413EB20E02C
:10C5B00030E0A90169817A818B819C810E9404E22B
:10C5C00020E030E040E05FEB87FD04C020E030E099
:10C5D00040E05FE369817A818B819C810E94FBE866
:10C5E0000E94F0E9CB010E947118BC018DE094E03B
:10C5F0000E9413EB40914B024F7749830E94FF3713
:10C600006D83972E5C01162F80910F01C9808C15C8
:10C61000C1F0C0920F0128E4C29EB001112490E045
:10C6200080E00E9409E22AE037ED43E25CE30E94E9
:10C630006AE20E94F7E960930C04C110A8C210924C
:10C64000070480910E01181709F440C0CD80C092F4
:10C650000E016C2D792DC50120E13EE040E050E057
:10C660000E944CE869015CE3452E512C612C712C31
:10C670006D81792DC501A30192010E944CE8CA0188
:10C68000B901A30192010E944CE824E6C216D1042C
:10C6900008F0A0C27F936F93DF92CF9283E292E083
:10C6A0009F938F9387EF93E09F938F930E949BE1DB
:10C6B0000FB6F894DEBF0FBECDBF85E0982F990F5F
:10C6C000990F891B880F80588093F6030E949CBDA8
:10C6D0000091F2031091F3032091F4033091F503DC
:10C6E0006B017C01C01AD10AE20AF30A97018601A4
:10C6F00037FD11C02091F10320952093F1036A5476
:10C700007C4F8F4F9F4F6093F2037093F30380939E
:10C71000F4039093F503D090F103D98281E00E9455
:10C72000106B80919813843158F480919A1388305B
:10C7300038F028EA32E04CE068E080E50E94B2BFC1
:10C74000809198138431A0F480919A13823080F004
:10C75000E980EE2031F08091020C22E732E0811175
:10C7600002C02CE332E042E162E088E60E94B2BF00
:10C77000809198138C3108F0E8C0E0900013F0909D
:10C780000113883028F580910213909103130E94C1
:10C79000F018FC01808193E0803229F4818192E0DD
:10C7A000803209F491E043E050E0491B51094E0FFB
:10C7B0005F1F892F880F880F981B892F67E0815F83
:10C7C0000E94C46D69E070E080E090E00E94526BCE
:10C7D000809198138C3130F580919A13843110F147
:10C7E000C7010E94F018FC01808193E0803229F497
:10C7F000818192E0803209F491E043E050E0491BEE
:10C8000051094E0F5F1F892F880F880F981B892FA2
:10C810006CE1815F0E94C46D69E070E080E090E0AF
:10C820000E94526BE0906B0BF0906C0B8091981310
:10C83000883028F580916D0B90916E0B0E94F01856
:10C84000FC01808193E0803229F4818192E0803282
:10C8500009F491E043E050E0491B51094E0F5F1F7E
:10C86000892F880F880F981B892F67E0865A0E94AE
:10C87000C46D69E070E080E090E00E94526B8091AE
:10C8800098138C3130F580919A13843110F1C701DF
:10C890000E94F018FC01808193E0803229F48181AC
:10C8A00092E0803209F491E043E050E0491B5109E5
:10C8B0004E0F5F1F892F880F880F981B892F6CE1FF
:10C8C000865A0E94C46D69E070E080E090E00E94AA
:10C8D000526B809198138C31C0F580919A138431FA
:10C8E000A0F19091020C292F30E02115310569F15A
:10C8F000F980F11084C18091580187FD83C1989F10
:10C9000090011124220F232F221F330B31954AE26D
:10C910004D8344E6429FC001439F900D11248158EE
:10C920009F4F6FEF70E00E94DDE8CB010E94F0188E
:10C93000AC016CE187E60E94C46DCD806C2DCC0CFF
:10C94000770B880B990B0E94526B8091981385335B
:10C9500030F480919A13813310F00E9474C080915A
:10C960009813843368F480919A13823348F002E07C
:10C9700020910C0442E367E384E693E10E94B1C096
:10C98000809198138033D8F480919A138832B8F04C
:10C9900080910704882361F047E054E060E387E377
:10C9A0000E94C46D65E270E080E090E00E94526BEE
:10C9B00047EF53E060E38091F6030E94C46D8091DD
:10C9C0009813873208F055C080919A138F3108F47C
:10C9D00050C083E080939B1326E2D22ED0929C130A
:10C9E00068E570E080E090E00E94526B8BE08093FD
:10C9F0009B13D0929C13E980EE2009F406C182E1DA
:10CA000094E00E94836C88E280939B13F6E2F0939B
:10CA10009C1369E570E080E090E00E94526B80E337
:10CA200080939B1396E2C92EC0929C13D980DD207F
:10CA300009F40CC18DE094E00E94836C8DE4809336
:10CA40009B13F6E2F0939C136AE570E080E090E0BF
:10CA50000E94526B85E580939B1386E2C82EC0929C
:10CA60009C13D980DD2009F414C187E194E00E9471
:10CA7000836C80919813833338F580919A138B32AD
:10CA800018F183E00E94106B83E080939B1383E393
:10CA900080939C1366E070E080E090E00E94526B0F
:10CAA00081E00E94106B80911601909117010E9405
:10CAB000F018AC0163E38CE00E94C46D65E270E0A5
:10CAC00080E090E00E94526B80919813813408F0CE
:10CAD00009C180919A13863308F404C110929B1304
:10CAE0008EE380939C1380E292E00E946A618983C6
:10CAF00060E870E080E292E00E94256CF981F531F7
:10CB000008F0F0C060E270E080E090E00E94526BBC
:10CB100029812F5F2983F2CF243631054CF48536E5
:10CB2000910504F58A30910534F48AE090E009C05B
:10CB300084369105BCF0883EE3E09E0714F087EE52
:10CB400093E02817390709F428CC909317018093B4
:10CB5000160110929A0B10929B0B10929C0B109244
:10CB60009D0B1BCC84E690E0F0CF662351F08EE263
:10CB70008093A20B605D6093A30B80E28093A40B73
:10CB8000F1CC80E28093A30B8093A20BF6CF498176
:10CB900081E3443608F480E28093A20B698190E23D
:10CBA0006A3040F02AE0862F622F0E94AFE80E9490
:10CBB000AFE8905D9093A30B89816AE00E94AFE893
:10CBC000905D9093A40B62EA7BE087E094E00E9482
:10CBD00013EB37CD7F936F93DF92CF9289E192E091
:10CBE0009F938F9387EF93E09F938F930E949BE196
:10CBF0000FB6F894DEBF0FBECDBF86E05FCD65E215
:10CC00006D8387CE85E28D8384CE87E00E9466297E
:10CC100080FF13C002E114E0F80161918F016623E7
:10CC200009F4F1CE6F320CF06FE3062E000C770B97
:10CC3000880B990B0E94526BEFCF8091AF0B80FD58
:10CC4000DECE87E392E00E94216CDDCE87E00E9479
:10CC50006629869580FF13C00DE014E0F80161910C
:10CC60008F01662309F4EACE6F320CF06FE3062ED3
:10CC7000000C770B880B990B0E94526BEFCF8091C1
:10CC8000AF0B869580FDD6CE87E392E00E94216CA3
:10CC9000D5CE87E00E9466298695869580FF17C0CD
:10CCA00087E194E09A838983E981FA816191FA832B
:10CCB000E983662309F4DDCE6F320CF06FE3062EB4
:10CCC000000C770B880B990B0E94526BEDCF809173
:10CCD000AF0B8695869580FDC8CE8FE292E00E94CC
:10CCE000216CC7CE0F900F900F900F900F90DF9197
:10CCF000CF911F910F91FF90EF90DF90CF90BF9059
:10CD0000AF909F908F907F906F905F904F9008951D
:10CD1000AF92BF92CF92DF92EF92FF920F931F9349
:10CD2000CF93DF93EC015B018A01FB01099587FD3D
:10CD300016C0C82ED12CF12CE12C2196F801C0820E
:10CD4000D182E282F382CE01DF91CF911F910F91C8
:10CD5000FF90EF90DF90CF90BF90AF900895982F05
:10CD6000907E903CA9F48F7190E0B0E0A0E06C015F
:10CD70007D0156E0CC0CDD1CEE1CFF1C5A95D1F752
:10CD8000CE010196F50109958F73C82A2296D6CF58
:10CD9000982F907F903E11F58F7090E0B0E0A0E06A
:10CDA0006C017D0136E0CC0CDD1CEE1CFF1C3A95BD
:10CDB000D1F7CE010196F50109958F73C82A46E097
:10CDC000CC0CDD1CEE1CFF1C4A95D1F7CE0102965F
:10CDD000F50109958F73C82A2396B0CF982F987FB5
:10CDE000903F79F5877090E0B0E0A0E06C017D01A4
:10CDF00086E0CC0CDD1CEE1CFF1C8A95D1F7CE0121
:10CE00000196F50109958F73C82A96E0CC0CDD1CBC
:10CE1000EE1CFF1C9A95D1F7CE010296F5010995FB
:10CE20008F73C82A26E0CC0CDD1CEE1CFF1C2A9553
:10CE3000D1F7CE010396F50109958F73C82A249680
:10CE40007DCF982F907C903841F4807C803869F4B5
:10CE50002196CE01F5010995F8CF8E7F8D3F28F000
:10CE60002196CE01F5010995F8CFC12CD12C760180
:10CE700065CFAF92BF92CF92DF92EF92FF920F9366
:10CE80001F93CF93DF9300D000D0CDB7DEB77C01E6
:10CE9000062F6A01122F86E0A82EB12C11160CF075
:10CEA00040C0AE014F5F5F4F68E07EE1C7010E9466
:10CEB00088667C0169817A818B819C81611571050D
:10CEC0008105910571F16D3371058105910509F4B5
:10CED00050C06E3771058105910509F44AC06A3268
:10CEE00071058105910569F507FF12C08FE092E099
:10CEF0000E3F11F08BE092E026E01202B001112407
:10CF00000E94C36B66E070E00E94DDE8161B61C002
:10CF100065E470E080E090E00E94526B115059F59A
:10CF200010E0812F0F900F900F900F90DF91CF9115
:10CF30001F910F91FF90EF90DF90CF90BF90AF9037
:10CF40000895643271058105910579F4C114D10405
:10CF500061F026E01202B0011124C6010E94C36BE9
:10CF6000B5010E94DDE8161B99CF0E94526B11504B
:10CF700095CF07FDBBCF61E089819A81AB81BC81F0
:10CF8000CD97A105B10509F460E0600F6A30ACF0FF
:10CF90001150862F6AE00E94BBE8092F682F880F86
:10CFA000770B605D7F4F072E000C880B990B0E945A
:10CFB000526B112309F4B4CF602F062E000C770BAF
:10CFC000605D7F4F072E000C880B990B0E94526BFF
:10CFD0001150112309F4A4CF86E01802B0011124E6
:10CFE000C7010E94C36B66E070E00E94DDE8161B7B
:10CFF00098CF0F931F93CF93DF938C0160E08AE269
:10D0000093E00E940177C8010E944E76F8010190DA
:10D010000020E9F73197EF01C01BD10BCB32D105CE
:10D020002CF08291807C8038E1F3F5CFDD27AE01D2
:10D03000B80180E292E00E9428EBC05EDD4F1882CA
:10D04000DF91CF911F910F910895EF92FF920F936F
:10D050001F93CF93DF93CDB7DEB762970FB6F894E7
:10D06000DEBF0FBECDBF0E946629882309F448C0E9
:10D0700049E152E082FF02C04CE152E029E132E096
:10D0800081FF02C029E032E080FD37C089E192E0F3
:10D090005F934F933F932F939F938F9383EC98E0ED
:10D0A0009F938F938E010F5F1F4F1F930F930E94CB
:10D0B0009BE10E94BB7CC8010E944E760FB6F8949B
:10D0C000DEBF0FBECDBF80915002811103C0C801E9
:10D0D0000E94F9670FB6F894DEBF0FBECDBF81E0A6
:10D0E00062960FB6F894DEBF0FBECDBFDF91CF9131
:10D0F0001F910F91FF90EF9008958BE092E0C8CFC1
:10D1000080E0EECF089590E080E00895282F909180
:10D110000C05833021F495FD0FC094FD0FC0892FBD
:10D1200090E0B0E0A0E004C0B695A79597958795EC
:10D130002A95D2F78170089581E0089580E00895DE
:10D140002F923F924F925F926F927F928F929F9217
:10D15000AF92BF92CF92DF92EF92FF920F931F9305
:10D16000CF93DF93CDB7DEB72E970FB6F894DEBF1F
:10D170000FBECDBFE82ED62E042F122F282F30E061
:10D180003C872B87462F50E05A87498765E0F62E6B
:10D19000F29EC001F39E900D11249E878D87FA01A7
:10D1A000E80FF91FEE0FFF1FEE0FFF1FE958FD4FAD
:10D1B00060817181828193819B01AC010E94FCEAB4
:10D1C000882309F434C1E00E612F6D0DFE9CF0013F
:10D1D0001124A985BA85AE0FBF1FAA0FBB1FAA0FC6
:10D1E000BB1FA958BD4FAC901196BC9011971296D9
:10D1F000CC9012971396DC90E00EFE9CA0011124B7
:10D20000A985BA85A40FB51FAA0FBB1FAA0FBB1F04
:10D21000A958BD4FEC901196FC90119712960C9165
:10D22000129713969C90862F90E0AD85BE85A80F2F
:10D23000B91FAA0FBB1FAA0FBB1FA958BD4F8C90C7
:10D2400011967C90119712966C90129713965C90A1
:10D25000610F70E0AD85BE85A60FB71FAA0FBB1F7B
:10D26000AA0FBB1FA958BD4F4C9011963C90119727
:10D2700012961C91129713962C90E80FF91FEE0F3F
:10D28000FF1FEE0FFF1FE958FD4FB081B9832181C9
:10D290002A8332813B8383818C83FA01E60FF71F57
:10D2A000EE0FFF1FEE0FFF1FE958FD4F90819D838A
:10D2B000A181AE83B281BF83238128879701402F4C
:10D2C000592DB701802F992D0E94FCEA882321F067
:10D2D000E12CF12C00E0912C9501A601B501C601CD
:10D2E0000E94FCEA882319F05701C02ED92C242D66
:10D2F000332D412F522D642D732D812F922D0E949D
:10D30000FCEA882321F0412C312C10E0212C282D1F
:10D31000372D462D552D682D772D862D952D0E9464
:10D32000FCEA882321F0842C732C612E522C2D8151
:10D330003E814F8158856D817E818F8198850E94C5
:10D34000FCEA882321F01D821E821F821886298113
:10D350003A814B815C8169817A818B819C810E94B9
:10D36000FCEA882341F03D8139834E814A835F8105
:10D370005B8388858C8385E0EB85FC858E9FD0015F
:10D380008F9FB00D112429853A85A20FB31FAA0FD4
:10D39000BB1FAA0FBB1FA958BD4FBA87A98795010C
:10D3A000A601B501C6010E94FBE89701402F592D47
:10D3B0000E94FAE86B017C01282D372D462D552D52
:10D3C000682D772D862D952D0E94FBE8242D332D79
:10D3D000412F522D0E94FAE89B01AC01C701B60112
:10D3E0000E94FBE86B017C0129813A814B815C81C1
:10D3F00069817A818B819C810E94FBE82D813E812D
:10D400004F8158850E94FAE89B01AC01C701B60123
:10D410000E94FBE820E030E040E450E40E947EE916
:10D42000A985BA856D937D938D939C9313972E96C2
:10D430000FB6F894DEBF0FBECDBFDF91CF911F9125
:10D440000F91FF90EF90DF90CF90BF90AF909F90A3
:10D450008F907F906F905F904F903F902F900895A6
:10D46000DF92EF92FF920F931F93CF93DF93EC0124
:10D47000D62E1CAD0BAD7C0184E0E80EF11CE98DCD
:10D48000FA8DC7010995412F480F2D2D602FC70137
:10D490000E94FFC29BAD890F8BAF81E090E0DF91CE
:10D4A000CF911F910F91FF90EF90DF900895EF9231
:10D4B000FF920F931F93CF937C0100910F05109162
:10D4C0001005C0E0F701EC0FF11D6081662351F0FB
:10D4D000062E000C770BC8010E9408EB892B49F43B
:10D4E000CF5FF0CF80E0CF911F910F91FF90EF9031
:10D4F000089581E0F8CFCF93DF9300D000D0CDB76F
:10D50000DEB780E090E0A0EAB0E489839A83AB8341
:10D51000BC8361E0CE0101960E94162E0F900F9001
:10D520000F900F90DF91CF91089580910205909117
:10D530000305009731F04AE050E070E060E00C94A1
:10D5400031E060E070E0CB01089580910205909198
:10D550000305009731F04AE050E070E060E00C9481
:10D5600003DF60E070E0CB0108950E94A56A97FD9B
:10D570000CC00E94A56A6F3F71058105910509F0F5
:10D5800034F40E94A56A862F089580E008958FEFF5
:10D5900008958091020590910305892B41F00E9426
:10D5A000B56A91E0811101C090E0892F089591E062
:10D5B000FCCF9CE0899F802D112491E0980F9093DF
:10D5C00015052CE0280F2093AB0B30E02E5F3F4F6A
:10D5D000409198134217130619F014F080E0089553
:10D5E00020919A139217D0F7662341F08E5F0E9424
:10D5F0005BC08091AB0B8E5F0E945BC08091AB0BD8
:10D6000090919813891750F320919A1390911505D2
:10D61000291720F310929B1380939C1381E00895A7
:10D6200020911405022E000C330B8217130641F0D3
:10D630008093140569E077E184E693E10C94A7C236
:10D6400008951F93CF93DF931F92CDB7DEB78F3F1F
:10D65000910519F014F08FEF90E08837910514F4DC
:10D6600088E790E09093410180934001182F8091CA
:10D670009D13811105C081E080939D130E943ABFE4
:10D68000609166137091671319839E012F5F3F4F5E
:10D690004FE084E693E10E940FBF0F90DF91CF919E
:10D6A0001F910895CF92DF92EF92FF920F931F93F5
:10D6B000CF93DF93CDB7DEB72C970FB6F894DEBFCC
:10D6C0000FBECDBF6F3F71058105910509F0D0F404
:10D6D00080E693E10E94306AE0916813F09169134B
:10D6E0003196849190E02C960FB6F894DEBF0FBE71
:10D6F000CDBFDF91CF911F910F91FF90EF90DF9001
:10D70000CF900895F0909B13E0909C1320911E02FF
:10D7100021110FC049EE56E16E2D8F2D0E946BC373
:10D7200090E080E0F80EF0929B13E0929C13992712
:10D73000DACFC0906813D090691324E633E13A83BE
:10D7400029832F2D30E03C832B832E2D30E03E8328
:10D750002D8318861F822FEF3FEF3A8729871C867B
:10D760001B8607E311E29E012F5F3F4FAB01BC0117
:10D77000C6010E94AAB2B60184E693E10E94A7C244
:10D780008F819885CFCFCF92DF92EF92FF920F9348
:10D790001F93CF93DF93CDB7DEB72C970FB6F894D6
:10D7A000DEBF0FBECDBFF0909B13E0909C13209185
:10D7B0001E0221111DC049EC56E16E2D8F2D0E94D5
:10D7C0006BC390E080E0F80EF0929B13E0929C1304
:10D7D00099272C960FB6F894DEBF0FBECDBFDF9110
:10D7E000CF911F910F91FF90EF90DF90CF90089510
:10D7F000C0906813D090691324E633E13A832983FB
:10D800002F2D30E03C832B832E2D30E03E832D8363
:10D8100018861F827A8769871C861B8607E311E2B8
:10D820009E012F5F3F4F48E05EE1BC01C6010E94B0
:10D830006EB3B60184E693E10E94A7C28F819885FA
:10D84000C2CF6FEF7FEF0C94C36BCF92DF92EF925A
:10D85000FF920F931F93CF93DF93CDB7DEB72C9733
:10D860000FB6F894DEBF0FBECDBFF0909B13E090D3
:10D870009C1320911E0221111DC049EA56E16E2D14
:10D880008F2D0E946BC390E080E0F80EF0929B1306
:10D89000E0929C1399272C960FB6F894DEBF0FBE2A
:10D8A000CDBFDF91CF911F910F91FF90EF90DF904F
:10D8B000CF900895C0906813D090691324E633E1A7
:10D8C0003A8329832F2D30E03C832B832E2D30E0AB
:10D8D0003E832D8318861F827A8769871C861B8664
:10D8E00007E311E29E012F5F3F4F4BE05EE1BC0179
:10D8F000C6010E946EB3B60184E693E10E94A7C2FE
:10D900008F819885C2CF6FEF7FEF0C94256CAF921B
:10D91000BF92CF92DF92EF92FF920F931F93CF931C
:10D92000DF935C016B010E945E61E82EC6010E94DC
:10D930006A61F12C03E110E0081B1109C5E20E1524
:10D940001F050CF4CFE18C2F90E09C012E5F3F4F20
:10D95000409198134217130609F0CCF509972091CE
:10D960009A13281719069CF14091AD0B5091AE0BFC
:10D970006091AC0B10929B13C0939C1325E1C501E1
:10D980000E943967D1E0C114D104B1F06AE370E0BC
:10D9900080E090E00E94526B0E151F05D4F4C45F26
:10D9A00080919813C81740F020919A134C2F49503A
:10D9B000550B241715067CF4DF91CF911F910F9121
:10D9C000FF90EF90DF90CF90BF90AF900895D0E0A0
:10D9D000DACFDD2389F3802F880F080F000F009323
:10D9E0009B13C0939C1360E270E080E090E00E9483
:10D9F000526BC601DF91CF911F910F91FF90EF9075
:10DA0000DF90CF90BF90AF900C94836C8F929F92D9
:10DA1000AF92BF92CF92DF92EF92FF920F931F933C
:10DA2000CF93DF93CDB7DEB72C970FB6F894DEBF58
:10DA30000FBECDBF982F862F5A017901D02E692FA6
:10DA40000E94D96A882309F489C0C701002391F193
:10DA50000E945E61C82E8090681390906913809137
:10DA60001E02811145C01FEF23E12C194091AD0B1F
:10DA70005091AE0B6091AC0BC5010E943967CC2070
:10DA800009F46CC0B6E08B9F500111246AE370E08A
:10DA900080E090E00E94526B57E0A516B10408F4B4
:10DAA00044C060E270E080E090E00E94526BA81AEF
:10DAB000B90AF2CF0E946A61C82E809068139090D4
:10DAC000691380911E02882371F2FE0133968AE069
:10DAD000DF011D928A95E9F784E693E19A838983B1
:10DAE0000EE011E29E012F5F3F4F4BE05EE112C05E
:10DAF000FE0133968AE0DF011D928A95E9F784E6FC
:10DB000093E19A8389830EE011E29E012F5F3F4FDC
:10DB100048E05EE1B701C4010E946EB3B40184E63F
:10DB200093E10E94A7C21F819FCF4091AB0B212F91
:10DB300030E0A6E0CA9EC00111242E5F3F4F281797
:10DB400039070CF49C0180E8821B80939B1340935F
:10DB50009C13C701DD20A9F00E94216C2C960FB602
:10DB6000F894DEBF0FBECDBFDF91CF911F910F9113
:10DB7000FF90EF90DF90CF90BF90AF909F908F90ED
:10DB800008950E94836CEACFE0E6F3E183AF64AFCF
:10DB9000CA010C94836C0F931F93CF9310920E05C0
:10DBA00010920D052FE32093130510921205109289
:10DBB00011059C01F90190812F5F3F4F9032D1F305
:10DBC0009E34C9F4818190ED980F9A3020F08D3207
:10DBD00011F08B3281F432969F012F5F3F4F80818D
:10DBE00080538A3008F468C09F012F5F3F4F8081C7
:10DBF000803209F463C0F093BA0BE093B90B8F0144
:10DC00000F5F1F4FC0816AE270E0C8010E9408EBFD
:10DC1000009731F0FC01319780818032E1F311826D
:10DC2000CD3429F0C43519F0C73409F041C0F801EA
:10DC300080810F5F1F4F8032D1F380538A30C0F54F
:10DC4000C093130530E020E06AE0AF014F5F5F4F03
:10DC5000629FC001639F900D11249C0120533109E4
:10DC60008081280F311D87FD3A95FA01808180530C
:10DC70008A3058F33093120520931105CA01FC0134
:10DC8000019640814032D9F3F0931005E0930F05DF
:10DC9000CD3401F52E31310539F090F427313105BD
:10DCA00019F02C313105B1F4F0930E05E0930D0518
:10DCB000CF911F910F910895F9018ECFF90194CF63
:10DCC0002537310538F02737310570F3203A83E0E6
:10DCD000380751F350E040E0CF01019660816623A0
:10DCE00009F45AC0613291F4CD3481F42032310507
:10DCF00069F490930E0580930D0563E270E00E9435
:10DD000008EB0097A9F2FC011082D2CFFC01DF01E1
:10DD10008D91803271F090ED980F9A3008F18E322B
:10DD200051F4918190539A30D8F041155105E1F4A6
:10DD300014C0FD01ECCF8D3211F08B3259F491817A
:10DD400060ED690F6A3060F09E3221F49281905349
:10DD50009A3030F04115510519F4AF014150510985
:10DD600081548A3108F4B8CFDF01FD018D918823F9
:10DD700009F4B2CF90ED980F9A30B8F393ED980F65
:10DD8000923098F38B3289F3CF0101966081603233
:10DD900009F0A2CFFC01F8CF50930E0540930D057A
:10DDA00087CFFC016591759185919491089580913B
:10DDB000B00B882319F080E00E947A3580E0089546
:10DDC0004F925F926F927F928F929F92AF92BF928B
:10DDD000CF92DF92EF92FF92CF93DF93CDB7DEB772
:10DDE00028970FB6F894DEBF0FBECDBF5C01DB01F4
:10DDF000CD90DD90ED90FC90E0914713F0914813A9
:10DE0000FE83ED8384819581A681B78189839A837E
:10DE1000AB83BC839C01AD01C701B6010E94FAE847
:10DE20002B013C01F50180809180A280B380AD81FF
:10DE3000BE818D919D910D90BC91A02D8D839E836F
:10DE4000AF83B88727E137EB41ED58EBC301B2014F
:10DE50000E947EEA87FDD0C027E030E046E153E42F
:10DE6000C301B2010E9404E218160CF4C5C02D8152
:10DE70003E814F815885C501B4010E94FAE82B010B
:10DE80003C0127E137EB41ED58EB0E947EEA87FD2C
:10DE9000B3C027E030E046E153E4C301B2010E9481
:10DEA00004E218160CF4A8C020E030E0A9016D814E
:10DEB0007E818F8198850E94FBE82B013C0120E048
:10DEC00030E040E450E40E9404E287FF05C0412CAA
:10DED000512C30E4632E762C27E137EB41ED58E3EB
:10DEE000C301B2010E94FAE89B01AC01C501B40173
:10DEF0000E947EEA87FD80C020E030E046E153E4E6
:10DF00006D817E818F8198850E94FBE82B013C0109
:10DF100020E030E043E153E40E947EEA181634F436
:10DF2000412C512C23E1622E23E4722E27E137EBA2
:10DF300041ED58E3C301B2010E94FBE89B01AC0133
:10DF4000C501B4010E9404E218160CF455C020E08B
:10DF500030E0A90169817A818B819C810E94FBE874
:10DF60004B015C0120E030E040E951E40E9404E212
:10DF700087FF06C0812C912C90E9A92E91E4B92E3F
:10DF800027E137EB41ED58E3C501B4010E94FAE8FF
:10DF90009B01AC01C701B6010E947EEA87FD2CC03F
:10DFA00020E030E046E153E469817A818B819C81F5
:10DFB0000E94FBE84B015C0120E030E044E053E4C8
:10DFC0000E947EEA181634F4812C912C84E0A82E4D
:10DFD00083E4B82E27E137EB41ED58E3C501B401E6
:10DFE0000E94FBE89B01AC01B1E0B983C701B60117
:10DFF0000E9404E218160CF41982898128960FB643
:10E00000F894DEBF0FBECDBFDF91CF91FF90EF90B0
:10E01000DF90CF90BF90AF909F908F907F906F9048
:10E020005F904F9008950E94A56ACB0108950F93C9
:10E030001F93CF9380910205909103050097E9F01B
:10E04000FC018F01C1912C2F2F7D81F0C53411F07F
:10E05000C536B9F7F801108270E060E00E94A5DDD6
:10E06000F801C083CF911F910F91089570E060E097
:10E07000CF911F910F910C94A5DD60E070E0CB0172
:10E08000F1CF682F880F770B80910F0590911005C5
:10E090000E9408EBFC0181E0309709F480E03097A2
:10E0A00081F0918120ED290F2A3030F09E3251F419
:10E0B000928190539A3098F43196F0930305E0934F
:10E0C000020508959D3211F09B3249F4928120EDB2
:10E0D000290F2A3088F39E3211F49381EACFF0E0C1
:10E0E000E0E0EBCF0E944170882341F081E0209175
:10E0F000020530910305232B09F480E00895CF93A6
:10E10000DF93EB010E947270882321F0DF91CF91A1
:10E110000C941370CE01DF91CF910895CF93C62F49
:10E120000E947270882319F0CF910C94B56A8C2FDD
:10E13000CF910895CF92DF92EF92FF926A017B0117
:10E140000E947270882331F0FF90EF90DF90CF90A3
:10E150000C941770C701B601FF90EF90DF90CF903D
:10E160000895CF93DF93C82FD62F0E947270882313
:10E1700021F0DF91CF910C94C96A8C2F0E944170DD
:10E18000811101C08D2FDF91CF9108954F925F9241
:10E190006F927F928F929F92AF92BF92CF92DF92B7
:10E1A000EF92FF920F931F93CF93DF93EC01209197
:10E1B000DB023091DC024091DD025091DE02688189
:10E1C00079818A819B810E94FAE86B017C01209110
:10E1D000DF023091E0024091E1025091E2026C8155
:10E1E0007D818E819F810E94FAE84B015C01A7012D
:10E1F0009601609144017091450180914601909192
:10E2000047010E9404E2882309F450C0C0924401EF
:10E21000D0924501E0924601F09247012091FA0424
:10E220003091FB044091FC045091FD04C701B601FC
:10E230000E946AE22B013C010E9426EA6B017C01EC
:10E2400020E030E0A9010E9404E287FD70C020E0D8
:10E2500030E040E450E4C701B6010E947EEA18169F
:10E260002CF4C12CD12CC0E4EC2EFE2CA70196017D
:10E27000C301B2010E94FAE86093F2047093F304C0
:10E280008093F4049093F504C701B6010E94F0E96D
:10E290006093F004062E000C770B6F5F7F4F6430A5
:10E2A000710514F064E070E06093EE04D0914201D7
:10E2B0001091F004A5019401609148017091490109
:10E2C00080914A0190914B010E9404E2811133C078
:10E2D000D11381C02091D6043091D7044091D80445
:10E2E0005091D9046091F2047091F3048091F40488
:10E2F0009091F5040E946AE22091DA043091DB04E7
:10E300004091DC045091DD040E94FBE8DF91CF9145
:10E310001F910F91FF90EF90DF90CF90BF90AF9043
:10E320009F908F907F906F905F904F900895C12C39
:10E33000D12C76019BCF8092480190924901A09206
:10E340004A01B0924B012091FE043091FF044091AC
:10E35000000550910105C501B4010E946AE24B011C
:10E360005C010E9426EA6B017C0120E030E0A901FB
:10E370000E9404E287FDF3C020E030E040E450E476
:10E38000C701B6010E947EEA18162CF4C12CD12CCC
:10E39000B0E4EB2EFE2CA7019601C501B4010E944A
:10E3A000FAE86093F6047093F7048093F80490936E
:10E3B000F904C701B6010E94F0E96093F104062E4A
:10E3C000000C770B6F5F7F4F6430710514F064E0D1
:10E3D00070E06093EF04C091F104D11305C0809107
:10E3E00043018C1709F470C08091F0049091F104FE
:10E3F00090934301809342010C2E000CDD0B25E02D
:10E400001203C0011124FC01EC0FFD1FEE0FFF1FD2
:10E41000EE0FFF1FE958FD4F20813181428153816A
:10E420002093EA043093EB044093EC045093ED0402
:10E430000091EF04002E000C110BFC01E00FF11F06
:10E44000EE0FFF1FEE0FFF1FE958FD4F6081718136
:10E45000828193810E94FAE86093E6047093E70456
:10E460008093E8049093E9042091EE0435E02303BF
:10E47000F0011124CE0FDF1FCC0FDD1FCC0FDD1FED
:10E48000C958DD4F288139814A815B812093E2049C
:10E490003093E3044093E4045093E504E00FF11F4C
:10E4A000EE0FFF1FEE0FFF1FE958FD4F60817181D6
:10E4B000828193810E94FAE86093DE047093DF0406
:10E4C0008093E0049093E1048090F6049090F70428
:10E4D000A090F804B090F9042091E6043091E7048C
:10E4E0004091E8045091E904C501B4010E946AE238
:10E4F0002091EA043091EB044091EC045091ED043A
:10E500000E94FBE86B017C01C092DA04D092DB042C
:10E51000E092DC04F092DD042091DE043091DF040F
:10E520004091E0045091E104C501B4010E946AE207
:10E530002091E2043091E3044091E4045091E50419
:10E540000E94FBE8A70196010E94FAE86093D604B6
:10E550007093D7048093D8049093D904BBCEC12C78
:10E56000D12C760118CF1F93CF93DF93CDB7DEB7B1
:10E570002C970FB6F894DEBF0FBECDBF182F88239F
:10E5800079F020E030E0A9016091E3027091E402AB
:10E590008091E5029091E6020E9404E28823F9F05E
:10E5A000809171028117D9F00E9431248CE0E3EE52
:10E5B000F1E0DE01119601900D928A95E1F7CE010E
:10E5C00001960E94C67080917102882391F08AECB6
:10E5D0009BE00E946A24109271020E94EE2E2C96FB
:10E5E0000FB6F894DEBF0FBECDBFDF91CF911F9164
:10E5F000089581E0809371028AEC9BE00E9452248E
:10E60000ECCF80E00E94B3721092DF021092E00221
:10E610001092E1021092E2021092DB021092DC02F0
:10E620001092DD021092DE021092E7021092E802D0
:10E630001092E9021092EA021092E3021092E402B0
:10E640001092E5021092E602E7E7F2E02BED32E0ED
:10E6500080E090E0A0ECBFE780839183A283B38346
:10E6600084839583A683B78380879187A287B387A6
:10E6700084879587A687B787808B918BA28BB38B76
:10E6800074962E173F0741F708958F929F92AF928D
:10E69000BF92CF92DF92EF92FF92C090E302D090B0
:10E6A000E402E090E502F090E60220E030E0A9010B
:10E6B000C701B6010E9404E28823E1F1A701960197
:10E6C00060E070E080E89FE30E947EE96B017C01DE
:10E6D0008090E7029090E802A090E902B090EA02F0
:10E6E00020E030E0A901C501B4010E9404E28823C2
:10E6F00029F1A501940160E070E080E89FE30E94A9
:10E700007EE9C092FA04D092FB04E092FC04F092FD
:10E71000FD046093FE047093FF04809300059093C2
:10E720000105FF90EF90DF90CF90BF90AF909F904A
:10E730008F900895C12CD12C7601CACF60E070E093
:10E74000CB01DFCFEFE6F0E0808182608083089527
:10E750008091B60B9091B70B892B79F48091B60B11
:10E760009091B70B892B49F42091B60B3091B70BE0
:10E7700081E0232B19F480E0089581E00895CF9281
:10E78000DF92EF92FF926B017C0183E3C816D10404
:10E79000E104F10470F082E3C81AD108E108F1083D
:10E7A00062E370E080E090E00E9401BD0E945DC8DD
:10E7B000ECCFC701B6010E9401BDFF90EF90DF9042
:10E7C000CF900C945DC85E9A8091AF0B8E7F809342
:10E7D000AF0B5E9A8091AF0B8D7F8093AF0B159A34
:10E7E0008091AF0B8B7F8093AF0B5E9A089581E091
:10E7F0000895DC01EC918E2F90E0FC01EE0FFF1FDD
:10E80000E80FF91FED5EFC4E80818F7780830895BD
:10E810001092900082E080939100109295001092E7
:10E820009400C19AE1E7F0E08081826080830895DE
:10E830007F928F929F92AF92BF92CF92DF92EF9290
:10E84000FF920F931F93CF93DF93EC017B0188819D
:10E850008C3008F0C4C090E0FC01EE0FFF1FE80F01
:10E86000F91FED5EFC4E80818F770E94C1B3198243
:10E870001A8288812CE0622F0E94AFE8829FB0014B
:10E88000112430E020E0AB01420F531FFA01EE0FDC
:10E89000FF1FE40FF51FED5EFC4E908197FD09C050
:10E8A0002F5F3F4F2C30310571F7811102C00E945C
:10E8B00008747880072D10E06801CC0CDD1CF6018F
:10E8C000E00FF11FED5EFC4E80818068808377FC55
:10E8D00086C080E2E81682E0F8060CF03FC08A812C
:10E8E00028E532E0281B310987FD3395220F331FBD
:10E8F000220F331F032E000C440B550B898178E83F
:10E90000872E912C881A910887FD9394880C991C66
:10E91000880C991C092C000CAA08BB0860E070E068
:10E92000CB01F7FC0AC0B701653B710514F064EB3D
:10E9300070E0072E000C880B990B281939094A0939
:10E940005B090E943CE824EB30E040E050E00E948C
:10E950006EE8820E931EA41EB51E74018BE087150F
:10E96000D8F0298188E890E0821B910927FD9395D2
:10E97000880F991F880F991FE816F90604F502976A
:10E980002FB7F894E601C00FD11FCD5EDC4E880F83
:10E99000991F9A8389832FBF62E370E080E090E043
:10E9A000DF91CF911F910F91FF90EF90DF90CF906B
:10E9B000BF90AF909F908F907F900C94BF732A81EF
:10E9C00088E592E0821B910927FD9395880F991F96
:10E9D000880F991FE816F90694F6C701D0CFDF918A
:10E9E000CF911F910F91FF90EF90DF90CF90BF904C
:10E9F000AF909F908F907F900895CF93DF93EB011E
:10EA0000682F70E088E393E10E941874688179812F
:10EA10008A819B81643F21E072078105910520F482
:10EA200064EF71E080E090E00E94BF7386B1829550
:10EA30008170DF91CF910895CF93DF9300D000D004
:10EA4000CDB7DEB78EEE92E0A0E0B0E089839A8386
:10EA5000AB83BC83BE016F5F7F4F8AE50E94FD746C
:10EA60000F900F900F900F90DF91CF910895CF935B
:10EA7000DF9300D000D0CDB7DEB78EEE92E0A0E0FD
:10EA8000B0E089839A83AB83BC83BE016F5F7F4F05
:10EA90008AE00E94FD740F900F900F900F90DF910D
:10EAA000CF910895CF93DF9300D000D0CDB7DEB7DC
:10EAB00084EF91E0A0E0B0E089839A83AB83BC83CC
:10EAC000BE016F5F7F4F8CE30E94FD740F900F902B
:10EAD0000F900F90DF91CF910895CF93DF9300D0E7
:10EAE00000D0CDB7DEB784EF91E0A0E0B0E089833D
:10EAF0009A83AB83BC83BE016F5F7F4F80EA0E9425
:10EB0000FD740F900F900F900F90DF91CF910895AB
:10EB10001F920F920FB60F9211240BB60F922F93E4
:10EB20003F934F935F936F937F938F939F93AF9395
:10EB3000BF93EF93FF938091C00487FF27C010928B
:10EB40009500109294008091C0048F5F8093C00460
:10EB50008091C004082E000C990B209137132817C0
:10EB6000190629F024F08091C0048C30DCF18091EA
:10EB7000940090919500049680349C4908F47DC0DF
:10EB80008091940090919500049679C08091C00482
:10EB9000082E000C990B209137132817190699F2AB
:10EBA00094F2E091C0048E2FEE0F990BFC01EE0F52
:10EBB000FF1FE80FF91FED5EFC4E808187FFC3CF7A
:10EBC000E091C0048E2FEE0F990BFC01EE0FFF1F9A
:10EBD000E80FF91FED5EFC4E808160E08F770E94A8
:10EBE0001BBCB1CF2091940030919500E091C004FE
:10EBF0008E2FEE0F990BFC01EE0FFF1FE80FF91F90
:10EC0000ED5EFC4E81819281820F931F909399005B
:10EC100080939800E091C0048E2FEE0F990BFC01B9
:10EC2000EE0FFF1FE80FF91FED5EFC4E808187FF9E
:10EC300011C0E091C0048E2FEE0F990BFC01EE0F76
:10EC4000FF1FE80FF91FED5EFC4E808161E08F77BA
:10EC50000E941BBCFF91EF91BF91AF919F918F914B
:10EC60007F916F915F914F913F912F910F900BBECC
:10EC70000F900FBE0F901F90189580E49CE9909321
:10EC80009900809398008FEF8093C004E3CF909118
:10EC9000C00095FFFCCF8093C6000895CF93DF930B
:10ECA000EC018991882319F00E944776FACF8DE014
:10ECB0000E9447768AE0DF91CF910C944776CF92FD
:10ECC000DF92EF92FF920F931F93CF93DF93CDB715
:10ECD000DEB7A0970FB6F894DEBF0FBECDBF4423BA
:10ECE00009F445C0611571058105910579F100E0D0
:10ECF000C42ED12CF12CE12CA70196010E944CE8E6
:10ED000011E0100FE1E0F0E0EC0FFD1FE00FF11D4E
:10ED100007FDFA956083B901CA01012F61157105DC
:10ED20008105910549F7115010F1E1E0F0E0EC0F99
:10ED3000FD1FE10FF11D17FDFA95908187E39A30D1
:10ED400008F480E3890F0E944776EDCF80E3A09618
:10ED50000FB6F894DEBF0FBECDBFDF91CF911F91EC
:10ED60000F91FF90EF90DF90CF900C944776A09694
:10ED70000FB6F894DEBF0FBECDBFDF91CF911F91CC
:10ED80000F91FF90EF90DF90CF900895CF92DF9298
:10ED9000EF92FF92CF936B017C01C42F4A3069F44C
:10EDA000F7FE0BC0F094E094D094C094C11CD11C29
:10EDB000E11CF11C8DE20E9447764C2FC701B60181
:10EDC000CF91FF90EF90DF90CF900C945F76CF9330
:10EDD000DF93EC018991882319F00E944776FACFDE
:10EDE000DF91CF910895CF93DF93EC01FE018491E1
:10EDF0002196882319F00E944776F8CFDF91CF91B2
:10EE000008950F931F93CF938C01C62F88E69FE040
:10EE10000E94F376C8010E94F376CC2331F08AE099
:10EE2000CF911F910F910C944776CF911F910F9125
:10EE3000089561E082E79FE00C940177AF92BF9262
:10EE4000CF92DF92EF92FF920F931F93CF93DF93B6
:10EE500085ED9EE00E94F376C0E0D7E0D15021F02E
:10EE600080E20E944776FACF8C2F0E94B3B3CF5F27
:10EE7000C53099F78AE00E94477607E712E0C0E0C4
:10EE800080E20E9447768C2F0E94B3B35801D5E0F0
:10EE900080E20E944776F501C080D180E280F38055
:10EEA000A7019601C701B6010E94FCEA882369F117
:10EEB00080E20E9447768DE30E9447768DE30E94B0
:10EEC00047768DE30E9447768DE30E9447768DE377
:10EED0000E944776D150F4E1AF0EB11CD111D8CFCA
:10EEE0008AE00E944776CF5F0C5F1F4FC53041F626
:10EEF0008AE0DF91CF911F910F91FF90EF90DF900B
:10EF0000CF90BF90AF900C94477620E030E0A901FD
:10EF1000C701B6010E947EEA87FD03C08BE20E9412
:10EF2000477643E0C701B6010E9413C4D3CFCF9206
:10EF3000DF92EF92FF926A017B010E94F37642E03A
:10EF4000C701B601FF90EF90DF90CF900C9413C4EF
:10EF5000CF92DF92EF92FF926A017B010E94F376DB
:10EF60004AE0C701B601FF90EF90DF90CF900C947C
:10EF7000C6762F923F924F925F926F927F928F92BE
:10EF80009F92AF92BF92CF92DF92EF92FF920F9338
:10EF90001F93CF93DF93CDB7DEB7C654D1090FB619
:10EFA000F894DEBF0FBECDBF70E060E085E40E9444
:10EFB0007F70182F8F3F09F483C08823E9F085E81C
:10EFC00096E1CA5BDF4F0FB6F894DEBF0FBECDBF30
:10EFD000DF91CF911F910F91FF90EF90DF90CF9035
:10EFE000BF90AF909F908F907F906F905F904F9069
:10EFF0003F902F900C94F37624EB30E03A832983F2
:10F0000083E50E947270882321F00E9413709A8316
:10F01000898365E070E083E40E947F708AA760E0E6
:10F0200085E50E94B17025968FAF259760E088E74F
:10F0300096E10E945C54A981BA81BD01BB0F880B87
:10F04000990B0E940BE26D837E838F8327969FAF7F
:10F0500027970E949CBD688B798B8A8B9B8B1F3F67
:10F0600009F045C420E030E04CE053E46D817E813E
:10F070008F8127969FAD27970E947EEA18160CF085
:10F08000AAC18DE496E10E94F376CA5BDF4F0FB60A
:10F09000F894DEBF0FBECDBFDF91CF911F910F91CE
:10F0A000FF90EF90DF90CF90BF90AF909F908F90A8
:10F0B0007F906F905F904F903F902F900C9464B52D
:10F0C00046E450E05A8349839BCF1FAEAFC12496DC
:10F0D000EEADFFAD2497808383C2FBEE4F2E512C03
:10F0E000612C712C04C384E190E0A0E0B0E08C8B33
:10F0F0009D8BAE8BBF8BE4E14E2E512C612C712C7D
:10F1000004C34C8A5D8A6E8A7F8AFFC22496EEAD64
:10F11000FFAD24978083D4C389819A81AB81BC8160
:10F1200029A93AA94BA95CA9821B930BA40BB50B87
:10F13000B7FD59C08FAD0E94B7C48AE00E944776E0
:10F1400089819A81AB81BC818053984FAF4FBF4F6B
:10F1500089AB9AABABABBCAB9DA9911177C02EA983
:10F160003FA948AD59ADB101802F26969FAD269796
:10F170000E947EEA18160CF053C020E030E040E018
:10F1800050E4B101802F26969FAD26970E94FBE8A0
:10F190006EAB7FAB88AF99AF2CA53DA54EA55FA503
:10F1A00089819A81AB81BC81280F391F4A1F5B1F5F
:10F1B0002AAF3BAF4CAF5DAF20E030E040EC50E415
:10F1C0006D817E818F8127969FAD27970E94FAE8F7
:10F1D0009101402F26965FAD26970E9404E2881F7A
:10F1E0008827881F8DAB88899989AA89BB89C81609
:10F1F000D906EA06FB0610F4D701C60129813A8137
:10F200004B815C81281B390B4A0B5B0BDA01C9016E
:10F2100081389F44A241B105A8F189E995E10EC268
:10F2200089819A81AB81BC812AAD3BAD4CAD5DAD8E
:10F23000821B930BA40BB50B48E854E267E974E218
:10F24000B7FDD1CF812F0E94ACC5CDCF20E030E0FB
:10F2500040EF51E46D817E818F8127969FAD279786
:10F260000E94FAE89B01AC01B101802F26969FAD68
:10F2700026970E9404E287FFB6CF44E355E264E498
:10F2800075E2E0CF4AA55BA5888D998D481759078F
:10F290000CF09EC003970CF49BC08CE395E10E9498
:10F2A000F3761F3F09F076C0ACE2B5E1BA83A983DB
:10F2B0008BE195E10E94F37689819A810E94F37631
:10F2C000488559856A857B8588E395E10E94977713
:10F2D0008AE00E9447768BE195E10E94F37689816E
:10F2E0009A810E94F37649A15AA16BA17CA184E383
:10F2F00095E10E9497778AE00E9447768BE195E13D
:10F300000E94F37689819A810E94F376B501A40167
:10F3100080E395E10E9497778AE00E9447762596E0
:10F32000FFAD2597FF2391F12CEA35EC47E25EE330
:10F3300069A17AA18BA19CA10E946AE26B017C0168
:10F340002CEA35EC47E25EE3C501B4010E947EE998
:10F35000288539854A855B851F3F09F52093700B09
:10F360003093710B4093720B5093730BC092740BDC
:10F37000D092750BE092760BF092770B6093780B3E
:10F380007093790B80937A0B90937B0B81E0809341
:10F3900059017BCEE7EAF7E2FA83E98389CF20932C
:10F3A0000513309306134093071350930813C0922C
:10F3B0000913D0920A13E0920B13F0920C1360938E
:10F3C0000D1370930E1380930F1390931013DECFD1
:10F3D0000E94385E80C089E396E10E94F3760E9425
:10F3E0007DC58FE780936F0B24EB30E0A8EEB3E090
:10F3F0000E94A0E86CA77DA78EA79FA728893989BE
:10F400004A895B89260F371F481F591F2AAF3BAF18
:10F410004CAF5DAF1092590181E08093520132E010
:10F42000310F3EAF323008F450CE1FAFC888D988B4
:10F43000EA88FB88C9AADAAAEBAAFCAA812C912C3B
:10F44000540189A29AA2ABA2BCA288869986AA86F8
:10F45000BB868FE790E0A0E0B0E08C8B9D8BAE8BFD
:10F46000BF8B1C8690E49A8FACE1AB8FB6E4BC8F67
:10F470001D8E1E8E1F8E18A23FE7432E512C612C2D
:10F48000712C1DAA8EAA9FAAA8AEB9AE1EA21FA259
:10F4900018A619A6E1E0EDA3198E188E212C312CA7
:10F4A00000E026961FAE2697F5E11F02C001112449
:10F4B0009C0124503D4E22963FAF2EAF2297285FED
:10F4C0003F4F24963FAF2EAF24974AA5042E000C41
:10F4D000550B5BA74AA780915201882309F4B0C05D
:10F4E0000E949CBD69837A838B839C8350913E05E7
:10F4F00058AB552309F48BC00E9494C560916B0BE7
:10F5000070916C0B1F3F39F02296AEADBFAD2297C4
:10F5100014966D917C91072E000C880B990B0E941C
:10F520000BE21B01082F26969FAF26972D8D3E8D4F
:10F530004F8D58A126969FAD26970E947EEA1816F9
:10F540003CF42D8E3E8E0F8F2696BFAD2697B8A326
:10F550002C853A8D4B8D5C8DB101802F26969FAD09
:10F5600026970E9404E287FF07C02C863A8E0B8FF5
:10F570002696EFAD2697EC8FFDA19101402F2696A0
:10F580005FAD26976D817E818F8127969FAD2797EE
:10F59000FF2309F45AC00E9404E287FF38C0498162
:10F5A0005A816B817C814C195D096E097F09DB01F1
:10F5B000CA0188589341A109B109B7FD28C08C89B7
:10F5C0009D89AE89BF8984199509A609B709B595A2
:10F5D000A795979587951F3F09F079CD80936F0B7D
:10F5E0004EA35FA368A779A7FD81FD8F2E812E8F83
:10F5F0003F813F8F27964FAD279748A389819A81F6
:10F60000AB81BC81888B998BAA8BBB8B1DA220E020
:10F6100030E040EF51E46D817E818F8127969FAD70
:10F6200027970E94FBE89101402F26965FAD269711
:10F630000E9404E287FF70CD87EB95E10E94F3768C
:10F64000109252010E947DC5A1CE0E947EEA18163A
:10F65000F4F689819A81AB81BC81288939894A89EC
:10F660005B89821B930BA40BB50BAC01BD01485801
:10F6700053416109710977FDCACF488D598D452BDA
:10F6800009F40DC1CEA0DFA0E8A4F9A4C80ED91ECC
:10F69000EA1EFB1E2EA13FA148A559A5281B390B28
:10F6A0004A0B5B0BC301B2010E943CE8A701960123
:10F6B0000E946EE84C885D886E887F88420E531EDB
:10F6C000641E751E54E145165104610471040CF466
:10F6D0000ACD8CEE48165104610471040CF0FDCC87
:10F6E00090E849165104610471040CF40ACD4C8A67
:10F6F0005D8A6E8A7F8A2EEF30E040E050E0241968
:10F7000035094609570929013A014C895D896E89F5
:10F710007F8981E396E10E94A877B301A2018CE280
:10F7200096E10E94A8774C855A8D6B8D7C8D85E281
:10F7300096E10E9497774D8D5E8D6F8D78A18EE159
:10F7400096E10E949777A88DB98D13970CF4A7C006
:10F75000C301B2010E940BE220E030E040E850E437
:10F760000E946AE24B015C012C853A8D4B8D5C8DC9
:10F770006D8D7E8D8F8D98A10E94FAE82BED3FE074
:10F7800049E450E40E946AE220E030E040E05FE3B8
:10F790000E946AE29B01AC01C501B4010E947EE9AE
:10F7A0006C877D878E879F87C701B6010E940BE219
:10F7B0002FE632E143E85AE30E946AE26B017C01E2
:10F7C0001E3F59F02AE939E949E15FE3812C912C88
:10F7D000A12C6EE3B62E1F3F59F42DEC3CEC4CE40B
:10F7E0005EE37BEA872E7AEA972EA92C7EE3B72E7A
:10F7F0006C857D858E859F850E946AE26887798702
:10F800008A879B879B01AC010E94FBE8A7019601B8
:10F810000E947EE969A37AA38BA39CA328853985DE
:10F820004A855B85C701B6010E946AE2A501940181
:10F830000E946AE24B015C014C855D856E857F8587
:10F8400088E196E10E949777B701A60182E196E1EF
:10F850000E9497778AE00E944776BEAD83E096E1EA
:10F86000B23010F084EF95E10E94F3764885598517
:10F870006A857B858EEE95E10E94977749A15AA112
:10F880006BA17CA188EE95E10E949777B501A40158
:10F8900082EE95E10E9497778AE00E9447768C89F4
:10F8A0009D89AE89BF89840D951DA61DB71DB5958F
:10F8B000A795979587951F3F09F028CC80936F0BEC
:10F8C000288D398D2F5F3F4F398F288F3D813C87A1
:10F8D0004E814A8F5F815B8F27968FAD27978C8FE4
:10F8E000C980DA80EB80FC8098A99DA390CEE12EA0
:10F8F000012E000CFF08F70183E0EE0FFF1F8A9531
:10F90000E1F7E15AFE4F668177816F507109072E4A
:10F91000000C880B990B0E940BE29B01AC016D81DE
:10F920007E818F8127969FAD27970E947EEA1816C9
:10F930000CF4A7CB89E396E10E94F3760E947DC583
:10F9400085E18E9DF0018F9DF00D1124E450FD4E58
:10F950008FE7808722E330E049CDCF93DF93EB013F
:10F960000E94F376CE01DF91CF910C94BAB38EEC66
:10F970009EE00C94F37688EC9EE00C94F376CF93A3
:10F9800084E50E947270C0E08823D9F00E94B56AB5
:10F99000C82F1816B4F40E94BB7C8DE40E944776F1
:10F9A00080911105909112050E9475B56C2FCC0FB6
:10F9B000770B88E290E10E94AD7C8AE00E94477656
:10F9C000CFEF8C2FCF9108950E947DC50E9479388A
:10F9D000809144058130A1F40E94B77C81E59EE0CE
:10F9E0000E94F37660E087E49EE00E945C546EE53E
:10F9F00071E080E090E00E94BF7388E0809344054E
:10FA00000895CF92DF92EF92FF921F93CF93DF93EF
:10FA100000D000D0CDB7DEB78EEEC82E82E0D82E53
:10FA2000E12CF12CC982DA82EB82FC82BE016F5F8D
:10FA30007F4F8AE50E94FD7481110EC010E0812F76
:10FA40000F900F900F900F90DF91CF911F91FF902B
:10FA5000EF90DF90CF9008950E946D75C982DA8291
:10FA6000EB82FC82BE016F5F7F4F8AE50E94FD74CE
:10FA7000182F882319F30E94B77C8BE29FE00E9425
:10FA8000F3760E94E47CDBCFCF92DF92EF92FF927D
:10FA90001F93CF93DF9300D000D0CDB7DEB78EEEAB
:10FAA000C82E82E0D82EE12CF12CC982DA82EB82BA
:10FAB000FC82BE016F5F7F4F8AE00E94FD7481115E
:10FAC0000EC010E0812F0F900F900F900F90DF91DC
:10FAD000CF911F91FF90EF90DF90CF9008950E94FB
:10FAE0006D750E941C750E9437750E941C75C98235
:10FAF000DA82EB82FC82BE016F5F7F4F8AE00E9458
:10FB0000FD74182F8823E9F20E94B77C8EEE9EE0E8
:10FB10000E94F3760E94E47CD5CFEC018B01F42E99
:10FB20000E947DC50E94B77C87E29EE00E94F3762A
:10FB30000115110511F407EA17E2209711F4CEE13F
:10FB4000DEE00E94D6601F930F93DF93CF938EE089
:10FB50009EE09F938F93D1E0DF930E9443540E94D5
:10FB6000C139C0916513C695C6958DB79EB70796E6
:10FB70000FB6F8949EBF0FBE8DBF80919D1381116B
:10FB800004C0D0939D130E943ABF80916613909158
:10FB900067130E9413BFDC2FDD0F1D2F1C0F83E0A6
:10FBA0000E94106B40E252E06C2F80E00E94C46D16
:10FBB00010929B13D0939C138FEF9DE00E94216CB9
:10FBC00010929B1310939C1382EF9DE00E94216C76
:10FBD00084E693E10E9475C28111E1CF61E085E185
:10FBE0009EE00E94017789EE93E030E6019729F0CC
:10FBF000232F2A950000E9F7F9CFF89489EE93E0D6
:10FC000038EE019729F0232F2A950000E9F7F9CF64
:10FC10000E947DC5FF2021F00E94E373A895FECFCE
:10FC20005E9AFCCF80910F12909110122FEF3FEF50
:10FC3000981751F0E92FF0E0E15FFD4E228130E0AE
:10FC40009F5F9F7790931012C90108952F923F9262
:10FC50004F925F926F927F928F929F92AF92BF92DC
:10FC6000CF92DF92EF92FF920F931F93CF93DF9388
:10FC700000D000D000D0CDB7DEB7809153058031E1
:10FC800008F051C10E949CBD6B017C01809153051D
:10FC9000811108C080910F1290911012891B8F77EB
:10FCA00009F491C411E601E013C08A3019F08D30D7
:10FCB00009F0FCC01092F712809195129091961263
:10FCC000FC01EF56FD4E1682892BF1F40E945DC8AF
:10FCD00080915305803108F026C180910F129091D8
:10FCE0001012891B8F7709F41EC10E94127E97FFA4
:10FCF000DCCF0E94B77C84ED9DE00E94F37680917A
:10FD00000F1280931012E4CF109296121092951257
:10FD100027E932E13D832C83EC81FD8181918032A2
:10FD200009F44BC08E3409F06DC06FEC7DE08C811E
:10FD30009D810E9481E15C01892B49F06EE470E0B5
:10FD40008C819D8104960E9408EB009711F48C81B0
:10FD50009D814AE050E070E060E001960E9403DF80
:10FD60002B013C018091911290919212A0919312DB
:10FD7000B09194120196A11DB11D481659066A064C
:10FD80007B0629F060E08CE99DE0AB2861F16AE236
:10FD900070E08C819D810E9437EB009739F1282F0C
:10FDA0003C81231BB12C222359F02150EC81FD8191
:10FDB000E20FF11D3081B326F6CFFD83EC83ACCF8B
:10FDC0004AE050E070E060E001960E9403DF8B2C77
:10FDD000912CB12CA12C681579058A059B0551F051
:10FDE00060E08DE79DE00E94FDB372CF60E083E5A7
:10FDF0009DE0F9CF4092911250929212609293122C
:10FE000070929412809144058130E9F067E470E0CB
:10FE10008C819D810E9408EB0097A9F04AE050E098
:10FE200070E060E001960E9403DF62307105810599
:10FE3000910548F48CED9CE00E94F37660E082ED41
:10FE40009CE00E945C54C0920805D0920905E092A3
:10FE50000A05F0920B05809197128B3309F438CF85
:10FE600080915305803108F033CF80915505819FF3
:10FE7000C001112467E972E18A5A9A4F0E9413EB7C
:10FE800080915505189FF0011124EA54FA4F108211
:10FE90008F5F803140F480935505809153058F5FCB
:10FEA0008093530515CF10925505F7CF9091F71217
:10FEB000913009F40DCF9430B0F094509093F71234
:10FEC0008830C9F48091951290919612009709F4A8
:10FED000FFCE019790939612809395128F569D4E68
:10FEE000FC011682F5CE8C35C9F49C5F9093F71215
:10FEF000943009F4EDCE2091951230919612A9011B
:10FF00004F5F5F4F50939612409395122F563D4E80
:10FF1000F90186834F3551051CF4DACE8B3381F617
:10FF20000093F712D5CE0E949CBD6B017C0180919D
:10FF3000040590910505A0910605B091070500976D
:10FF4000A105B10581F14091B20B5091B30B6091C5
:10FF5000B40B7091B50B840F951FA61FB71FA70197
:10FF60009601281B390B4A0B5B0BDA01C901B7FD5F
:10FF70001AC00E94B77C4091B90B5091BA0B5D83B7
:10FF80004C8385E99CE00E94F3768C819D810E94E0
:10FF9000E7768AE00E94477640E070E060E090E01B
:10FFA00080E00E948D7D80914C0190914D01A09147
:10FFB0004E01B0914F01892B8A2B8B2B79F09091B8
:10FFC0004C1380914D13981709F405C1C092B20BE0
:10FFD000D092B30BE092B40BF092B50B0E949CBD93
:10FFE0004B015C0180911F02811108C020914C13CC
:10FFF00090914D1381E0291301C080E020910013FE
:020000021000EC
:100000003091011391E089272A3A31050CF480E000
:1000100091E04091CD045091CE046091CF04709155
:10002000D004452B462B472B09F490E0981789F014
:10003000882309F40AC1D501C40180569444A24F13
:10004000BF4F8093CD049093CE04A093CF04B09380
:10005000D0044090D60B5090D70B6090D80B709086
:10006000D90B2091C9043091CA044091CB0450911E
:10007000CC04C301B2010E9404E2882319F18091EB
:10008000CD049091CE04A091CF04B091D0044092C1
:10009000C9045092CA046092CB047092CC04892B9C
:1000A0008A2B8B2B09F449C0D501C4018056944496
:1000B000A24FBF4F8093CD049093CE04A093CF0462
:1000C000B093D0048091CD049091CE04A091CF0440
:1000D000B091D0040097A105B10579F1881A990A69
:1000E000AA0ABB0AB7FC29C01092CD041092CE0414
:1000F0001092CF041092D00480E89CE00E94F37626
:1001000060E08CE69CE00E945C5480910213909128
:1001100003131816190624F490E080E00E94A3232C
:1001200080916D0B90916E0B1816190634F4109295
:100130006E0B10926D0B0E941BBE8091D1049091AA
:10014000D204A091D304B091D404A7019601281B36
:10015000390B4A0B5B0BDA01C901B7FD14C22091C0
:100160004C1390914D1380915801291709F471C0D7
:10017000E0914D133BE5E39FF0011124E459F34F67
:100180009081899FC0011124880F892F881F990BA6
:100190009195182F0E949CBD112309F4F6C0809000
:1001A000C1049090C204A090C304B090C404811410
:1001B0009104A104B10409F04FC06C597F4F8F4FD7
:1001C0009F4F6093C1047093C2048093C3049093C3
:1001D000C4041FEF47C00E949CBD0091B20B109158
:1001E000B30B2091B40B3091B50B80904C019090E3
:1001F0004D01A0904E01B0904F01080D191D2A1D10
:100200003B1D601B710B820B930B97FF03C0109279
:10021000D504E4CE8091D5048111E0CE81E08093B5
:10022000D5045E9A8091AF0B8E7F8093AF0B5E9A60
:100230008091AF0B8D7F8093AF0B159A8091AF0BA0
:100240008B7F8093AF0B5E9AC9CE80E090E0DC019B
:10025000F8CE9091020C95CF681979098A099B090B
:1002600097FDB7CF412F50E05D834C8384E00E941F
:10027000C1B3111193C060E084E00E941BBC809167
:100280003D05882309F472C10091220110912301D8
:10029000C8010297209102133091031328173907E0
:1002A0000CF464C130904D13212C19821A821B82E8
:1002B00080914C13831509F4DFC0832D90E02BE56A
:1002C000289FF001299FF00D1124EA5EF34F458924
:1002D00056896789708D452B462B472B89F4418DB4
:1002E000528D638D748D452B462B472B49F4458DDC
:1002F000568D678D70A1452B462B472B09F440C0C6
:10030000EBE5E89FA001E99F500D11244A5E534F91
:100310005D834C83FA0161817281838194810E94A3
:10032000BCEA4B015C01EC81FD8161A172A183A15A
:1003300094A10E9409E22B013C01EC81FD8165A1A1
:1003400076A187A190A50E9409E29B01AC01C3019F
:10035000B2010E947EE9A50194010E946AE25B015C
:100360008E839C83222D39814A815B810E947EEAA3
:10037000181634F42A2CB982FE81FA832C812B833F
:100380003394332D3F70332E93CF1092C1041092CB
:10039000C2041092C3041092C40464CF8C819D8166
:1003A0008F3F910511F461E067CFEBE8F7E2E4914C
:1003B000E150EA3008F059C0F0E0EF51FE470C94EC
:1003C000F1E8EB81F081F5810182358235820D8281
:1003D00015821D82298284B5806884BD17BD4FCFE8
:1003E00084B5806284BD18BD4ACF8091800080684A
:1003F00080938000EC81FD81F0938900E093880078
:100400003ECF809180008062809380002C813D816E
:1004100030938B0020938A0032CF8091B0008068A7
:100420008093B0001093B3002ACF8091B000806217
:100430008093B0001093B40022CF80919000806828
:10044000809390004C815D81509399004093980077
:1004500016CF809190008062809390008C819D8166
:1004600090939B0080939A000ACFEC81FD81E03845
:10047000F1050CF098CFFFCEB801110F880B990B46
:100480000E940BE28B018E839C8320911C01309192
:100490001D0140911E0150911F01622D79818A81B9
:1004A0009B810E946AE298014E815C810E94FBE878
:1004B0003B014C01A0902001B09021019B01AC01B7
:1004C000B8018E819C810E947EEA1816A4F0B501C5
:1004D000BB0C880B990B0E940BE28B018E839C83D3
:1004E0009B01AC01B301C4010E947EEA18161CF006
:1004F00083018E829C828090C5049090C604A09057
:10050000C704B090C80498014E815C81C501B40154
:100510000E947EEA1816C4F428E431EE4AE75FE34D
:10052000C501B4010E946AE220E037ED43EA5CE3D2
:100530000E94FBE89B01AC01B8018E819C810E9466
:100540006AE28B018E839C83C801AE81BC8180935B
:10055000C5049093C604A093C704B093C804B8011F
:10056000CD010E94F0E9CB010E94A32344E6C40E12
:10057000D11CE11CF11CC092D104D092D204E092B3
:10058000D304F092D4040E945DC88091440588236E
:10059000E9F126960FB6F894DEBF0FBECDBFDF910E
:1005A000CF911F910F91FF90EF90DF90CF90BF9070
:1005B000AF909F908F907F906F905F904F903F9003
:1005C0002F900C94385E8091080590910905A091B8
:1005D0000A05B0910B05A7019601281B390B4A0BA0
:1005E0005B0BDA01C901885E9340A109B109B7FD2F
:1005F00059CB8CEE9DE00E94F376C0920805D09214
:100600000905E0920A05F0920B054CCB26960FB631
:10061000F894DEBF0FBECDBFDF91CF911F910F9138
:10062000FF90EF90DF90CF90BF90AF909F908F9012
:100630007F906F905F904F903F902F9008952F92F2
:100640003F924F925F926F927F928F929F92AF9262
:10065000BF92CF92DF92EF92FF920F931F93CF93AF
:10066000DF93CDB7DEB763970FB6F894DEBF0FBE4A
:10067000CDBF8091C61183FDA3C189E40E94727031
:10068000882309F48FC10E94B56A90E018161906F4
:1006900014F481E090E026E0289FF001299FF00DFE
:1006A0001124E458F44F828193811A828C38910589
:1006B00014F08CE890E090936E0B80936D0B0E9489
:1006C0001BBE60E081E00E9464C520916D0B3091FB
:1006D0006E0B80916B0B90916C0B821793070CF44F
:1006E00022C18DEF94E160E00E945C5481E0809330
:1006F00052011B821C821D821E8219861A861B864D
:100700001C861E862CE32F873CE1388B46E4498B00
:10071000312C212C50E859838FEB8A8B1B8A91E076
:100720009D87812C912C540100916D0B10916E0BC3
:10073000B801012E000C880B990B0E940BE26B0193
:100740007C01232D322D49815A890E9404E288239D
:1007500089F080916B0B90916C0BAA81A111E6C07E
:10076000B1E0BB8B081719070CF01B8A3C2C2D2C11
:10077000E982FA8A0E949CBD6B017C01DC01CB01FD
:1007800029853A854B855C85821B930BA40BB50BA1
:10079000B7FD2FC0D701C60188519C4FAF4FBF4F47
:1007A00089879A87AB87BC8780E00E94B7C489EFAE
:1007B00094E10E94F37681149104A104B10409F438
:1007C000DFC0C501B40168577C4E8F4F9F4F6C1935
:1007D0007D098E099F0928EE33E040E050E00E9439
:1007E0004CE8CA01B9014AE00E94C6768AE00E943C
:1007F00047760E94267E0E949CBD6093B20B709348
:10080000B30B8093B40B9093B50B60916B0B70910D
:100810006C0B072E000C880B990B0E940BE26F8368
:1008200078878C019B01AC01632D722D89819A8997
:100830000E94FAE82B013C0120E030E0A9010E946F
:100840007EEA87FF04C077FA709477F87094811479
:100850009104A104B10409F097C020E030E040E821
:100860005FE3C301B2010E9404E287FF10C09D85CF
:10087000812C912C5401992331F082E8882E86E056
:10088000982EA12CB12C8C0C9D1CAE1CBF1CAB89CE
:10089000AA2391F12B813C814D815E812115310587
:1008A0004105510541F0D701C601821B930BA40BF2
:1008B000B50BB7FD21C02F813885A8016E857F85D6
:1008C000888999890E94FAE820E030E040E85FE3F7
:1008D0000E9404E287FD2DC0D701C601805A9541D0
:1008E000AF4FBF4F8B839C83AD83BE839F819E8719
:1008F000A885AF87088B198B809152018823C9F096
:1009000081149104A104B10461F0B8E8CB1AB3E1F9
:10091000DB0AE108F108C818D908EA08FB08F7FE65
:1009200008C01D8601CF8CE095E1DDCE08171907C0
:100930000CF580915201882309F442C010925201B3
:1009400063960FB6F894DEBF0FBECDBFDF91CF9197
:100950001F910F91FF90EF90DF90CF90BF90AF90DD
:100960009F908F907F906F905F904F903F902F90CF
:100970000C9464B53C2C2D2CE982FA8A1B8AFACEA1
:100980008FE30E94477632CF20E030E040E450E42D
:10099000C301B2010E947EEA18160CF078CF46011E
:1009A000570175CF83E50E9472708A83811105C05B
:1009B00082E50E947270882319F00E94137076CE2F
:1009C00063960FB6F894DEBF0FBECDBFDF91CF9117
:1009D0001F910F91FF90EF90DF90CF90BF90AF905D
:1009E0009F908F907F906F905F904F903F902F904F
:1009F00008952F923F924F925F926F927F928F92C3
:100A00009F92AF92BF92CF92DF92EF92FF920F939D
:100A10001F93CF93DF93CDB7DEB765970FB6F894EA
:100A2000DEBF0FBECDBF8091C61183FD82C10E9483
:100A3000BF7C8A8787FD7DC189E40E94727088230C
:100A400009F4A8C10E94B56A90E01816190614F4BA
:100A500081E090E026E0289FF001299FF00D11240D
:100A6000E458F44F808191811D8A0E94A32361E0A4
:100A700081E00E9464C5209102133091031380919C
:100A8000001390910113821793070CF038C189EE7F
:100A900094E19F938F9384EF94E19F938F931F92A0
:100AA0000E9443540F900F900F900F900F9031E0E1
:100AB0003C8B0E9482248C89882309F43AC190914E
:100AC0003D059B8B10923D0581E0809352011C8275
:100AD0001D821E821F821B861C861D861E861F8607
:100AE000ACE3A88BBCE1B98B26E42A8B312C212CFA
:100AF00030E83A834FEB4B831982812C912C5401BF
:100B00000091021310910313B801012E000C880B01
:100B1000990B0E940BE26B017C01232D322D4A813F
:100B20005B810E9404E2882389F0809100139091F8
:100B300001135D895111EFC0A1E0A98308171907BE
:100B40000CF019823C2C2D2CEA82FB820E949CBD69
:100B50006B017C01DC01CB012B853C854D855E85DD
:100B6000821B930BA40BB50BB7FD2FC0D701C60199
:100B700088519C4FAF4FBF4F8B879C87AD87BE87F7
:100B80008A850E94B7C48AED94E10E94F3768114AD
:100B90009104A104B10409F4EBC0C501B401605390
:100BA000784F8F4F9F4F6C197D098E099F0928EE52
:100BB00033E040E050E00E944CE8CA01B9014AE04D
:100BC0000E94C6768AE00E9447760E94267E0E9496
:100BD0009CBD6093B20B7093B30B8093B40B909356
:100BE000B50B6091001370910113072E000C880B58
:100BF000990B0E940BE2688779878C019B01AC01FD
:100C0000632D722D8A819B810E94FAE82B013C01A1
:100C100020E030E0A9010E947EEA87FF04C077FA55
:100C2000709477F8709481149104A104B10409F0D0
:100C3000A3C020E030E040E85FE3C301B2010E94BE
:100C400004E287FF10C09C89812C912C54019923C8
:100C500031F08AE9882E82E0982EA12CB12C8C0CE0
:100C60009D1CAE1CBF1CA981AA2391F12C813D8142
:100C70004E815F81211531054105510541F0D701B4
:100C8000C601821B930BA40BB50BB7FD21C02885B1
:100C90003985A8016F85788989899A890E94FAE83F
:100CA00020E030E040EC5FE30E9404E287FD36C0C4
:100CB000D701C601805A9541AF4FBF4F8C839D83AA
:100CC000AE83BF8398859F87A985A88B098B1A8BD4
:100CD00080915201882311F181149104A104B1047F
:100CE00061F0B0EDCB1AB7E0DB0AE108F108C818F3
:100CF000D908EA08FB08F7FE11C01C8A01CF2D892C
:100D00008EED94E1222309F4C4CE5D895C8BD1CEB3
:100D10004C894D8BCECE0817190724F580915201CE
:100D2000882321F0109252010E9464B52B892093F0
:100D30003D0565960FB6F894DEBF0FBECDBFDF91BF
:100D4000CF911F910F91FF90EF90DF90CF90BF90C8
:100D5000AF909F908F907F906F905F904F903F905B
:100D60002F9008953C2C2D2CEA82FB821982EECE26
:100D70008FE30E94477626CF20E030E040E450E445
:100D8000C301B2010E947EEA18160CF06CCF460136
:100D9000570169CF83E50E9472708D8B811107C066
:100DA00082E50E9472708C8B882309F4B1CF0E9477
:100DB00013705BCE2F923F924F925F926F927F9211
:100DC0008F929F92AF92BF92CF92DF92EF92FF925B
:100DD0000F931F93CF93DF93CDB7DEB7ED970FB689
:100DE000F894DEBF0FBECDBF80917102888B87E57E
:100DF0000E944170882309F41BC120E030E0A90162
:100E00006091E3027091E4028091E5029091E60224
:100E10000E9404E2811107C00E94B77C86E190E144
:100E20000E94F37618C18AE50E947270882339F116
:100E30000E9417702091C40B3091C50B4091C60BD6
:100E40005091C70B0E94FAE86B017C0120E030E072
:100E500040E251ECC701B6010E947EEA87FD0AC05C
:100E600020E030E040E251E4C701B6010E9404E214
:100E7000181674F40E94B77C89E090E1D1CFC0903D
:100E8000D20BD090D30BE090D40BF090D50BDECFEB
:100E900040E050E060EC7FE788E50E949A70209186
:100EA000BC0B3091BD0B4091BE0B5091BF0B0E940B
:100EB000FAE82B013C0140E050E060EC7FE789E577
:100EC0000E949A702091C00B3091C10B4091C20BCF
:100ED0005091C30B0E94FAE84B015C016FEF89E46B
:100EE0000E948E70182F6FEF8AE40E948E70082F78
:100EF000A3019201C301B2010E94FCEA81116EC0FC
:100F0000A5019401C501B4010E94FCEA811166C0EB
:100F10008BA19CA1ADA1BEA18BAB9CABADABBEAB7D
:100F20002091DB023091DC024091DD025091DE0223
:100F3000C301B2010E94FAE82B013C0120E030E03D
:100F400040E05FE36BA97CA98DA99EA90E946AE29B
:100F50009B01AC01C301B2010E94FBE82BA93CA993
:100F60004DA95EA90E947EE90E94F0E9162F4FA0CC
:100F700058A469A47AA42091DF023091E002409144
:100F8000E1025091E202C501B4010E94FAE84B016E
:100F90005C0120E030E040E05FE3C301B2010E9469
:100FA0006AE29B01AC01C501B4010E94FBE8A30108
:100FB00092010E947EE90E94F0E9062F812F012E06
:100FC000000C990B97FD2CC0059764F5802F002E1F
:100FD000000C990B97FD28C0059744F51530D8F5FE
:100FE0000530C8F580E00E94B37295E01902F00167
:100FF0001124E00FF11D07FDFA95EE0FFF1FEE0F14
:10100000FF1FE958FD4FC082D182E282F3828889B6
:101010000E94B37288898823F1F00E940A2F1BC0B6
:1010200010E0D4CF14E0D2CF00E0D8CF04E0D6CF88
:101030008AE40E94417081110CC070E060E086E596
:101040000E947F709A8389830597F0F084EE9FE079
:10105000E7CE0E940173ED960FB6F894DEBF0FBE87
:10106000CDBFDF91CF911F910F91FF90EF90DF9057
:10107000CF90BF90AF909F908F907F906F905F9038
:101080004F903F902F90089560E084E40E94B170EB
:101090008F8740E050E0BA018AE50E949A706BA702
:1010A0007CA78DA79EA740E050E86BE376E483E53C
:1010B0000E949A7020E030E040E752E40E947EE90E
:1010C000609368017093690180936A0190936B014A
:1010D0000091471310914813D801CD90DD90ED9009
:1010E000FC9020E030E0A901C701B6010E94FBE8B6
:1010F0006AAF7BAF8CAF9DAF20E030E040E450E4BE
:101100000E9404E287FF06C01AAE1BAEB0E4BCAF7B
:10111000E0E4EDAF20E030E046E153E4C701B60182
:101120000E94FBE86BAB672E8FAB98AF20E030E0FE
:1011300043E153E40E947EEA181634F41BAA612CA2
:10114000F3E1FFAB23E428AFD80114968D909D9076
:10115000AD90BC90179720E030E0A901C501B40123
:101160000E94FBE87B018C0120E030E040E951E483
:101170000E9404E287FF04C0E12CF12C00E911E495
:1011800020E030E046E153E4C501B4010E94FBE8F1
:10119000B62EC72ED82E99AF20E030E044E053E4BD
:1011A0000E947EEA181634F4B12CC12CF4E0DF2E34
:1011B000B3E4B9AF88E40E944170882309F40DC2FA
:1011C0000E9417700E94F0E91B0177FF02C06F5F59
:1011D0007F4F75956795719561957109655B7F4F37
:1011E000072E000C880B990B0E940BE2762E872E9F
:1011F000982EA92E9701A8010E947EEA181624F4C1
:10120000E72CF82C092D1A2D2AAD3BAD4CAD5DAD68
:10121000672D782D892D9A2D0E947EEA181624F0CC
:101220007AAC8BAC9CACADAC872D982DA92DBA2D8A
:101230008B8B9C8BAD8BBE8BC701D8018F8B988F0E
:10124000A98FBA8FB101330C880B990B0E940BE266
:101250001B012C01AC019B01B701C8010E94FBE8F6
:101260007B018C012B2D3C2D4D2D59AD0E9404E2AC
:1012700087FF04C0BE2CCF2CD02E19AFA201910144
:10128000672D782D892D9A2D0E94FBE87B018C011A
:101290002BA9362D4FA958AD0E9404E287FF04C048
:1012A000EBAA6F2C0FAB18AF8BA9962DAFA9B8ADD9
:1012B0008B8F9C8FAD8FBE8F8B2D9C2DAD2DB9AD9F
:1012C0008F8F98A3A9A3BAA3BE01695E7F4FCE01F9
:1012D00043960E94E06E882309F4AEC1BE01615EB0
:1012E0007F4FCE014B960E94E06EE82E882309F4D2
:1012F000A3C12F89388D498D5A8D6F8D78A189A111
:101300009AA10E94FAE820E030E040E85EE30E9403
:101310006AE24B015C012B893C894D895E896B8DAA
:101320007C8D8D8D9E8D0E94FAE820E030E040E8B3
:101330005EE30E946AE26BA37CA38DA39EA38FA2AF
:1013400098A6A9A6BAA689819A811816190674F4D6
:1013500082EB9FE00E94F3768F85882321F088EA54
:101360009FE00E94F3768AE00E9447760E94312433
:101370000E94FA2C80E00E94B37280E090E0A0E22C
:10138000B1E48FA798ABA9ABBAAB60E0CE018F9662
:101390000E94162E2091E3023091E4024091E50272
:1013A0005091E6026BA17CA18DA19EA10E9404E256
:1013B000811130C02091E7023091E8024091E902AA
:1013C0005091EA026FA178A589A59AA50E9404E22E
:1013D000811120C02091DB023091DC024091DD02BE
:1013E0005091DE026B897C898D899E890E9404E27E
:1013F000811110C02091DF023091E0024091E102A2
:101400005091E2026F89788D898D9A8D0E9404E255
:101410008823A9F00E94017388E0FE01B396A3EE31
:10142000B2E001900D928A95E1F788E0FE01739693
:10143000ABEDB2E001900D928A95E1F7188A60E079
:1014400085E40E94B17088248394811102C062E017
:10145000862E1B861C861D861E861A8A9E2C48E7B1
:10146000C42E4FE0D42E56E8A52E5FE0B52E1A8983
:1014700015300CF0EBC06B857C858D859E859B01BE
:10148000AC010E94FCEA8111E1C03324339435E0C1
:10149000232E911005C033243A9422242A9484E008
:1014A00091E09926F12EFF0CFF0CF10EF394898B3D
:1014B00019896A89121509F4C5C0062E000C770B2C
:1014C000880B990B0E940BE22FA138A549A55AA5BC
:1014D0000E946AE22F89388D498D5A8D0E94FBE85F
:1014E0002B013C01612F110F770B880B990B0E9488
:1014F0000BE22BA13CA14DA15EA10E946AE22B89C7
:101500003C894D895E890E94FBE86B837C838D83D7
:101510009E834F82588669867A8689819A81892B33
:1015200089F084E99FE00E94F3768F2D0E94B3B387
:1015300069E170E082E99FE00E94AD7C8FE89FE066
:101540000E94F3761F92E9E1EF931F92FF92DF92E0
:10155000CF92BF92AF921F920E9443542981482D8F
:10156000BE01695F7F4FCE0103960E94DDB52B015E
:101570003C014B865C866D867E860FB6F894DEBF96
:101580000FBECDBFAC019B010E94FCEA811157C088
:1015900009898A8925E0020380011124080F111DA1
:1015A00087FD1A95000F111F000F111F09581D4FBD
:1015B000A30192016BA57CA58DA59EA50E94FBE8C9
:1015C000D8016D937D938D939C931397188A0E94F5
:1015D000267EF3948989830D6ACFA701B80186E43A
:1015E0000E949A701B012C014AAD5BAD6CAD7DADC4
:1015F0008CE40E949A706B8B7C8B8D8B9E8B2F8AD8
:10160000388E498E5A8E4B2D5C2D6D2D79AD82E42E
:101610000E949A706B017C014BA9562D6FA978AD81
:1016200082E50E949A706B8F7C8F8D8F9E8FCF8EFC
:10163000D8A2E9A2FAA248CE88EC9FE0F1CB888933
:101640000E94B3728A898F5F8A8B11CF0E9464B522
:101650000E94D76E882359F088890E94B37280E077
:1016600090E0A0ECBFE78B879C87AD87BE876B853A
:101670007C858D859E859B01AC010E94FCEA8111D1
:101680004DC08F85811126C082E0F82E02E094E0E3
:10169000C92E12E0DC2CD11A21E041E0612F802F0D
:1016A0000E94A06821E04FEF612F8F2D0E94A0685B
:1016B0002FEF41E06D2D802F0E94A0682FEF4FEF9C
:1016C0006D2D8F2D0E94A068115020F70150F394CA
:1016D0000F3FF9F60E941E770E9445738F85811196
:1016E00018C08AEC9BE00E94C6709B01AC0160911F
:1016F000D20B7091D30B8091D40B9091D50B0E949B
:10170000FAE86093D20B7093D30B8093D40B909331
:10171000D50B8F858111E888E09271020E94E12C3F
:101720008091710281110E94EE2E0E947B6A75CC1D
:101730002F923F924F925F926F927F928F929F92E1
:10174000AF92BF92CF92DF92EF92FF920F931F93CF
:10175000CF93DF93CDB7DEB7C254D1090FB6F8945B
:10176000DEBF0FBECDBF21968FAF21972DB73EB7FD
:1017700023963FAF2EAF2397809113058D3409F444
:101780004CC6843511F40C948EA1873491F4809169
:101790001105909112058C31910509F46CC208F085
:1017A00074C08430910509F4F1C130F4029708F453
:1017B00002C10E947BB581C18531910509F47DC1CB
:1017C0004B97B9F787E00E942568811176C119828D
:1017D0001A821B821C821D821E821F82188680E054
:1017E00090E0A0E2B1E489879A87AB87BC8780E567
:1017F0000E94727060E081110E94A56A80E090E012
:10180000A8E4B2E48F8F98A3A9A3BAA380E090E0E4
:10181000A0EAB0E48B8F9C8FAD8FBE8F613009F44E
:10182000EEC1623009F4FFC120E030E040E050E456
:101830006091D20B7091D30B8091D40B9091D50B0A
:101840000E94FBE87B018C0120E030E048E453E497
:101850000E947EEA181624F4E12CF12C08E413E42B
:10186000A984BA84CB84DC849701A801B501C601A0
:101870000E947EEA181614F475018601C701D8018A
:101880008F8B988FA98FBA8FF0C18A32910509F496
:101890002CC408F081C08D31910509F4B7C34E976F
:1018A00009F087CF0091471310914813D8012D916B
:1018B0003D914D915C916091CA0B7091CB0B8091E1
:1018C000CC0B9091CD0B0E94FBE8AB01BC0188E5ED
:1018D0000E949A7069837A838B839C83F8012481A8
:1018E0003581468157816091CE0B7091CF0B8091ED
:1018F000D00B9091D10B0E94FBE8AB01BC0189E5B4
:101900000E949A706D837E838F839887BE016B5F80
:101910007F4FCE0101960E94E06E882309F4CDC06E
:1019200080E00E94B3720E94FA2C61E085E40E947C
:10193000B170182F21E0482FBE016B5F7F4FCE01A1
:1019400001960E94DDB56B017C01AC019B010E94F8
:10195000FCEA811119C049815A816B817C8187E73A
:1019600090E10E9497774D815E816F81788582E753
:1019700090E10E949777B701A6018DE690E10E9461
:1019800097778AE00E9447760E94E12C11110E940D
:101990007B6A0E940A2F91C08B35910509F4C8C457
:1019A0008C35910509F4C8C48A35910509F001CF39
:1019B00010920C0582C080914405813009F07DC0F1
:1019C000E1E5CE2EE2E0DE2EFAECEF2EFBE0FF2E7C
:1019D000ACEBAA2EABE0BA2E10E088E5810F0E9496
:1019E0007270882309F4B6C00E9417702B013C0165
:1019F000812F0E948668882309F4A2C0D7012D9107
:101A00003D914D915C91C301B2010E94FBE8D6016A
:101A10006D937D938D939C9313971F5FF4E0CF0E8E
:101A2000D11C24E0E20EF11C34E0A30EB11C1330F3
:101A3000A1F685E40E947270882309F496C00E9482
:101A400017706B017C0183E00E948668882371F027
:101A50002091D60B3091D70B4091D80B5091D90BD8
:101A6000C701B6010E94FBE86B017C01C0925D02D8
:101A7000D0925E02E0925F02F092600240E050E09D
:101A8000BA0186E40E949A7020E030E0A9010E9429
:101A90007EEA181684F40E94177020E030E040E7D8
:101AA00052E40E947EE960931801709319018093BB
:101AB0001A0190931B010E947C2921962FAD21973A
:101AC00021110C94AC970E949CBD60930805709303
:101AD000090580930A0590930B050091540511E6C2
:101AE000109FF0011124EA54FA4F808181110C9467
:101AF000AC9787ED94E10E94F376019F8001112459
:101B00000A5A1A4FD8018C918E3411F00C94AFA15F
:101B100080E20E9447768EE40E9447760F5F1F4F57
:101B2000F80181918F0190ED980F9A3030F08D324D
:101B300021F08B3211F00C94AFA10E944776F0CFC8
:101B4000F5012081318142815381C301B2010E949C
:101B5000FAE85DCFF70180819181A281B381F6011E
:101B600080839183A283B38358CF8091D60B9091C9
:101B7000D70BA091D80BB091D90B80935D029093B5
:101B80005E02A0935F02B093600278CF80E50E946E
:101B90007270C12CD12C7601882321F00E94956AA5
:101BA0006B017C0183E50E947270882361F00E94C2
:101BB000177020E030E04AE754E40E946AE20E9495
:101BC000F7E96B017C010E94312480912002811190
:101BD00005C060E08BE390E10E945C540E949CBDD4
:101BE000C60ED71EE81EF91E0E949CBD6C197D0909
:101BF0008E099F0997FF61CF0E94267EF5CFBE0117
:101C0000655E7F4FCE0109960E94F72DAE01415EC1
